:1000000000000220657300008D7300008F730000F4
:1000100091730000937300009573000000000000CE
:1000200000000000000000000000000097730000C6
:1000300099730000000000009B7300009D73000096
:100040009F73000035520000297700009D72000068
:10005000917200009F7300009F7300009F73000067
:100060009F7300009F730000B53300009F73000072
:100070009F7300009F7300009F7300009F73000038
:100080009F730000AD7700009F7300009F73000016
:100090009F7300009F7300009F7300009F73000018
:1000A0009F7300009F7300009F7300009F73000008
:1000B0009F7300009F73000000000000000000001C
:1000C0009F7300009F7300009F7300009F730000E8
:1000D0009F7300009F7300009F7300009F730000D8
:1000E0009F730000000000000000000000000000FE
:1000F000000000009F730000000000009F730000DC
:1001000000000000000000000000000000000000EF
:1001100000000000000000000000000000000000DF
:1001200000000000000000000000000000000000CF
:1001300000000000000000000000000000000000BF
:1001400000000000000000000000000000000000AF
:10015000000000000000000000000000000000009F
:10016000000000000000000000000000000000008F
:10017000000000000000000000000000000000007F
:10018000000000000000000000000000000000006F
:10019000000000000000000000000000000000005F
:1001A000000000000000000000000000000000004F
:1001B000000000000000000000000000000000003F
:1001C000000000000000000000000000000000002F
:1001D000000000000000000000000000000000001F
:1001E000000000000000000000000000000000000F
:1001F00000000000000000000000000000000000FF
:1002000010B5054C237833B9044B13B10448AFF350
:1002100000800123237010BD380200200000000080
:10022000ECCB000008B5034B1BB103490348AFF307
:10023000008008BD000000003C020020ECCB000064
:10024000154B002B08BF134B9D46A3F5803A0021A8
:100250008B460F461348144A121A09F029FD0F4B1A
:10026000002B00D098470E4B002B00D09847002061
:10027000002104000D000D48002802D00C48AFF307
:10028000008009F0CDFC2000290007F0A5FA09F054
:10029000A1FC00BF000008000000022000000000D8
:1002A0000000000038020020FC8D0120000000004A
:1002B0000000000010F0010310D104280CD90368DD
:1002C000C3F30F1343B1013B9B001A1DC1180979F9
:1002D00011B101339342F9D1184670470023FBE76F
:1002E000037883B11A0601D40130704703F0C003CC
:1002F000C02B08BF0130024610460132037803F0DC
:10030000C003802BF8D0704708B5002103780BB9E3
:10031000084608BDFFF7E4FF0131F7E738B50022D2
:1003200004460D46411C092003F05EFB40B163000A
:10033000024643F0010342F8043F0023A34200DBDE
:1003400038BD55F8231042F8041F0133F6E70128A1
:1003500038B504DC1C20BDE8384001F07FB80D68DA
:10036000EA0701D41120F6E74868C30706D4042839
:1003700004D9036803F00F03042B01D00E20EAE731
:1003800003F096F96D10002D044603DDFFF7BCFF66
:10039000A84206DA1220DEE72046FFF7A1FF013D62
:1003A0000446012DF8D120787F2808DDDF280ADCFB
:1003B0006378800100F4F86003F03F0318434000C5
:1003C00040F0010038BDEF280ADC637800039B0190
:1003D00080B203F47C630343A07800F03F00EDE7B4
:1003E000F72810DC637880041B0303F47C3300F4EB
:1003F000E0101843E37803F03F030343A078800143
:1004000000F47C60DAE74FF0FF30D8E7486838B591
:10041000C3070D4606D4042804D9036803F00F026D
:10042000092A04D00B20BDE8384001F017B8446811
:10043000C3F30F1364105A1EA2420BD8032194FB7E
:10044000F1F16429A8BF64210329ACBF5918D91C54
:1004500003F006FB0368C3F30F13013B9C4208D271
:10046000A31C013464002A6840F8232044F00104EE
:100470004460002038BD01282DE9F84304DC1C202D
:10048000BDE8F84300F0EABF02284E680CD08C6843
:10049000E70709D56410012CB8BF0124F50705D57D
:1004A0004FF0FF30BDE8F8830124F7E7042EF7D9B9
:1004B00033680D6803F00F02042A2DD1E80706D433
:1004C000042D04D92B6803F00F03042B01D00E2058
:1004D000D6E73046FFF7EEFEA042E1DB304603F000
:1004E000E7F80646284603F0E3F8013C01463019D8
:1004F00009F0ADFF01460028D2D0012433780BB1BA
:100500008E4203D3640044F00100CBE73046FFF78E
:10051000E7FE01340646F1E7092A34D177687F10F7
:10052000BC42BDDCE90725D4042D23D92B6803F098
:100530000F03042B1ED1284603F0BAF8804604F1BD
:10054000010956F829008542DCD0C2070ED40428E0
:100550000CD9036803F00F03042B07D103F0A8F8AC
:100560000146404609F03AFF0028CBD0B9454C4639
:10057000E5DD95E7631C56F82320AA42C2D0BB42B2
:100580001C46F7DD8CE7032A8AD1C3F30F17C3F3A8
:100590004173C3EB8707BC4282DCEB072AD4042DEE
:1005A00028D9286800F00F03032B19D1C0F30F13CB
:1005B000C0F3417005F10408C0EB83003F1A013C11
:1005C00040440336BC423FF76BAF32194346834287
:1005D000194611D317D10134600040F0010061E7E2
:1005E000042B07D1284603F063F880462846FFF71E
:1005F00061FEE3E70F2043E712F8015F09788D42BF
:1006000003F10103E3D00134DCE708B503F034F86B
:10061000400040F0010008BDC30711D404280FD9E1
:10062000026802F00F03032B0AD101F00303C3F1A8
:1006300004035B0703F0C04322F0C042134303608E
:10064000704701282DE9F0470546884604DC1C2048
:10065000BDE8F04700F002BF4C6814F0010701D17B
:100660000D20F5E7022802D08B68DA07F8D5D8F814
:100670000060F30700F1A980042E40F2A6803268E2
:100680006410012C02F00F03B8BF0124092B28D1FC
:100690007668022D4FEA660605D0D8F808305B1060
:1006A0009E42A8BF1E46351B0135012225EAE5758D
:1006B000A918092003F098F9074648B16D000346D0
:1006C00045F00105D8F8002043F8045FA64202DA9D
:1006D0003846BDE8F087013452F8241043F8041F6F
:1006E000F4E7042B43D1304602F0E2FFFFF70CFEA3
:1006F000022D824605D0D8F808305B109842A8BF7A
:100700009A46A24504DA0020BDE8F04703F0E6B9B6
:10071000304602F0CDFF0546A74222DB304602F00C
:10072000C7FFA94606462846FFF7DAFD0134A24571
:100730000546F8DAA0EB0905284603F0CFF907468D
:100740000028C5D002F0B4FF0446D8F8000002F03B
:10075000AFFFA9EB060101442A46204609F084FABE
:10076000B6E72846FFF7BCFD01370546D4E7032B63
:100770002BD1C2F30F13022DC2F34172C2EB8302DD
:1007800005D0D8F808305B109A42A8BF1A46A2429A
:1007900006DA002211460320BDE8F04703F024B931
:1007A000151B0423291D002291FBF3F1032003F004
:1007B0001BF9074600288BD001352946FFF72CFF8F
:1007C000E11C2A4631440430C8E7212040E70028D4
:1007D000F8B504DC1C20BDE8F84000F03FBE0C6812
:1007E00014F001060FD0641024EAE474E11C002226
:1007F0008910032003F0F8F8054610B12146FFF7F1
:100800000BFF2846F8BD042C01D80025F9E7256820
:1008100005F00F05042D19D12046FFF74BFD324698
:10082000C11C074691FBF5F1032003F0DDF80546F6
:100830000028E6D03946FFF7EFFE204602F038FFE9
:100840003A460146281D09F00FFADAE7092DDCD1F6
:1008500067687F100423F91C324691FBF3F10320F3
:1008600003F0C2F805460028CFD03946FFF7D4FE82
:100870000434BE42C5DA54F8043FDA0742BFAA196D
:10088000A3F3480313710136F3E77F2902DC0170FB
:1008900001307047B1F5006F0CDA03468A1162F03F
:1008A0003F0203F8022B01F03F0161F07F0141702C
:1008B00018467047B1F5803F0FDA0B1363F01F0342
:1008C0000370C1F3851301F03F0163F07F0361F012
:1008D0007F014370817003307047B1F5883F0DDAB6
:1008E000F0230370902343708B1101F03F0163F0FC
:1008F0007F0361F07F018370C17004307047000096
:100900000028F7B50F4603DC1C2000F0A7FD0CE023
:100910000A6812F001000AD06C4651102046FFF719
:10092000B4FF011B204603F0E0F8044616E0042A59
:100930003BD9136803F00F03092B36D155681C49C6
:100940006D100124AC420CDD03F0C8F8044628B158
:100950003F6802F0ADFE0126AE421DDD204603B029
:10096000F0BD013452F8243013F0010601D10D20FE
:10097000CBE75B107F2B09DDB3F5006F08DBB3F528
:10098000803F07DB8B42D4BF042600263044D9E7E2
:100990000226FBE70326F9E7013657F82610CB07B6
:1009A000E5D54910FFF771FFD6E72120ADE700BF7D
:1009B000FF0F010010B5044611F0010011D1042908
:1009C0000ED90B6803F00F03042B09D1084602F07F
:1009D0006FFE0146204609F001FDB0FA80F04009A3
:1009E00010BD0020FCE700000128F8B50E4604DC2D
:1009F0001C20BDE8F84000F031BD4D6815F001073E
:100A000006D1042D04D92B6803F00F02092A01D066
:100A10000B20EEE76C6809681F486410C3F30F13DE
:100A2000A34298BF03F1FF34FFF7C4FF40B1012395
:100A3000BC4201DA0020F8BD013745F82730F7E75E
:100A400031681648FFF7B6FF50B1002CF2D0631C96
:100A50000122013C944045F8232014436C60E9E7EF
:100A60003368DA0701D40D20C3E75B10002B0DDDDE
:100A70009C420BDB05EB830305EB84029A4207D112
:100A80000123013C9C4053601C43E7E71220B0E780
:100A9000996843F8041FF1E757B300005BB3000007
:100AA000002310B50B70C3070C4606D50E49421043
:100AB0002046BDE8104009F055BC28B90B49204636
:100AC000BDE8104009F06EBC042801D10849F6E7E2
:100AD00009D9036803F00F03042B04D102F0E8FDE9
:100AE00004490246E4E710BD14BE000060B30000F4
:100AF00066B300006BB300002DE9F04301288FB00E
:100B000081460E4607DC1C2000F0A8FC054628465E
:100B10000FB0BDE8F0830B6813F0010440F0A18032
:100B2000042B40F2D5801B6803F00F03092B40D142
:100B3000274656F8273013F0010806D1042B04D9B4
:100B4000186800F00F00092801D02220DCE75B685C
:100B50000137B94504EB6304EBD10122A11802F07F
:100B600043FF054608B90025D1E7640044F00104BD
:100B70004460424600F1080456F822104B680868A9
:100B80005B10C0F30F10984298BF00F1FF3304319F
:100B90000020834207DC013223EAE373BA4204EB0C
:100BA0008304E9DBB3E751F804CF44F820C00130F7
:100BB000EFE7032B40F08C80274656F8270010F013
:100BC0000108C2D10428C0D9036803F00F02032A28
:100BD00038D1C3F30F12C3F34173C3EB82031C4438
:100BE0000137B945E9D10423E11C002291FBF3F15F
:100BF000032002F0F9FE05460028B4D02146FFF795
:100C00000BFD00F1040956F82840E10720D4042C1C
:100C10001ED9206800F00F03032B19D1C0F30F1366
:100C2000C0F34170C0EB830003344B46A3EB0902D1
:100C3000824211DB08F101080028A8BF8144B845B1
:100C4000E1DB64E7042A80D1FFF734FB0444C7E703
:100C50002046FFF72FFBE7E714F8012F03F8012BDD
:100C6000E4E700252C4656F82500C20732D40428B4
:100C700030D9036803F00F02042A32D1FFF71AFBC0
:100C800004440135A945EED1204602F027FF054670
:100C900000283FF468AF041DB04606EB890958F8F8
:100CA000046BF30728D4042E26D9336803F00F020F
:100CB000042A34D13046FFF7FDFA0746304602F0E9
:100CC000F7FC3A460146204608F0CEFF3C4421E0BE
:100CD0002546C8E701A9FFF7E3FE01A809F088FB54
:100CE000CEE7032A7FF431AFC3F30F12C3F341738E
:100CF000C3EB82031C44C4E701A93046FFF7D0FED2
:100D000001A809F075FB01A906460246204608F035
:100D1000ABFF3444C145C2D100232370F7E6032A58
:100D2000F8D1C3F30F17C3F34173C3EB87073A46F8
:100D3000311DC8E72DE9F04F002893B00F4607DCBE
:100D40001C2000F08BFB0546284613B0BDE8F08F51
:100D50000D6815F0010806D1042D04D92B6803F0A5
:100D60000F03092B01D00B20EBE76E687610002EE5
:100D700003DC404602F0B2FEE5E7012826D04868D1
:100D8000C20723D4042821D9036803F00F03042BDE
:100D90001CD102F08DFC0446204609F029FB0435E5
:100DA000731E8146009303FB00FB05EB860A55F892
:100DB000040FC30771D404286FD9036803F00F022E
:100DC000042A05D1FFF776FA83440AE0384CE3E7BA
:100DD000032A69D1C3F30F12C3F34173C3EB820338
:100DE0009B44AA45E3D1584602F078FE0546002808
:100DF000AAD0D7F800A0B9F1000F03D0786802F0AC
:100E000057FC0446284602F053FC0AF10403074647
:100E10000193019B53F804AF0193504602F048FC44
:100E20001AF001030146029302D1BAF1040F04D86B
:100E300005A95046FFF734FE05A90846039109F0BD
:100E4000D7FADDE9023183468BB9BAF1040F0ED926
:100E5000DAF8000000F00F0CBCF1030F01BFC0F383
:100E60000F13C0F341700AF10401C0EB830B384645
:100E70005A4608F0F9FE5F44B9F1000F08D0009B14
:100E8000434505DD38464A46214608F0EDFE4F440D
:100E900008F101084645BCD156E705A9FFF700FE59
:100EA00005A809F0A5FA8FE702F002FCF9E700BFF8
:100EB000FFB70000002810B511DD0B6813F0010426
:100EC00002D05C1024EAE4740122A118092002F087
:100ED0008BFD18B1640044F00104446010BD00248F
:100EE000F2E70A6838B512F0010436D1042A34D981
:100EF0001368496803F00F00092818D15068C3F33C
:100F00000F134010834298BF03F1FF30151DA0421C
:100F100005DC01330220984205DB002038BD45F88E
:100F2000041F0134F3E742F820100130F3E70328EF
:100F300013D1C80704D41320BDE8384000F08EBA9E
:100F40004910FF29F7D80432C3F30F1302EB8303D0
:100F50009A42E2D202F8011BFAE70B2000F07EFA77
:100F6000DBE700002DE9F0414E6816F001078846E6
:100F700028D1042E26D9346804F00F03092B11D18F
:100F80007568C4F30F146D10AC4200D8651ED8F814
:100F90000010CB071AD54C10002C01DDA54220DA39
:100FA000122034E0042B04D13046FFF783F90546C4
:100FB000EDE7032B08D1C4F30F15C4F34174C4EB60
:100FC0008505E4E70025E2E73D46E0E72848FFF72E
:100FD000F1FCA8B109F05EF990FBF5F404FB1504EF
:100FE0000134002F41D1042E3FD9336803F00F03A1
:100FF000092B12D1013456F824402046BDE8F08177
:10100000D8F800101B48FFF7D5FC20B91120BDE827
:10101000F04100F023BA2C46E3E7042B1DD1304603
:1010200002F046FB012C05460FDCFFF759F9461B81
:10103000304602F053FD04460028DED002F038FBB3
:101040003246294608F010FED7E72B78013C002BEA
:10105000A6D02846FFF744F9E4E7032B05D1344432
:10106000E478640044F00104C7E70B20CFE700BF39
:1010700050B300005BB300002DE9F0414C6814F060
:10108000010688462ED1042C2CD923688F6803F0E2
:101090000F02092A13D16568C3F30F136D10AB4219
:1010A00000D85D1ED8F800102848FFF783FC68B30D
:1010B000236803F00F03092B1ED1012317E0032A35
:1010C00010D1FA0704D41320BDE8F04100F0C6B9EE
:1010D0007E10FF2EF7D8C3F30F15C3F34173C3EB94
:1010E0008505DFE70B20EFE7013344F823709D42CD
:1010F000FADA0020BDE8F081032BFAD10334012392
:101100009D42F6DB04F8016F0133F9E7D8F80010CF
:10111000CB0706D54910002901DD8D4208DA1220DF
:10112000D2E70B48FFF746FC08B91120CCE7294667
:10113000236803F00F03092B03D1013144F8217018
:10114000D7E7032B04BF6418E670D2E757B300005B
:101150005BB30000086808B5C3071BD4042819D97D
:10116000036803F00F02092A01D1406808BD032A71
:1011700009D1C3F30F12C3F34170C0EB82004000EA
:1011800040F00100F2E7042A04D102F091FAFFF7DF
:10119000BBF8F4E70120E9E7024A03480B2104F019
:1011A00013B900BFF8B20000F0B200000020704791
:1011B0000420704701207047002002F08FBC0020FF
:1011C00070470020704700207047002070470020C3
:1011D00070470020704700207047002070470000D3
:1011E000024A03480C2104F0EFB800BFE0B300004E
:1011F00040B400007047037883B11A0601D401306F
:10120000704703F0C003C02B08BF013002461046F0
:101210000132037803F0C003802BF8D07047000040
:10122000F8B511F0010506461446084626D10429F2
:101230003FD90B6803F00F03042B3AD1D30714D422
:10124000042A36D9136803F00F03042B31D102F0BE
:101250002FFA0546204602F02BFA0146284609F0EF
:10126000BDF800282DDB1ED126E002F021FA294628
:101270000A2209F081F90546601011E012F0010719
:1012800015D1042A15D9136803F00F03042B10D1CC
:1012900010464D1002F00CFA0A22394609F06CF99A
:1012A00085420EDB08DD002E09DC00200CE04D102D
:1012B000E2E7064B0F221A700136022EF5D8042001
:1012C00002E0701700F00400F8BD00BF78020020B3
:1012D00010B510F0010402D04410204610BD0428BF
:1012E00012D9026802F00F02042A07D102F0E0F9D5
:1012F0000A222146BDE8104009F03EB9032A03D175
:101300000A2221460430F5E7014B0D221A70E4E76A
:101310007802002010F0010210B516D1042802D97D
:101320000268C2F30F1211F0010310D1042902D98F
:101330000B68C3F30F13934216D1043000EB830202
:101340000331904205D301200BE00022EBE700239C
:10135000F1E710F8014B11F8013F1CB9B3FA83F023
:10136000400910BD9C42ECD00020FAE72DE9F74F70
:10137000804689469A46304F304E6AB102233B7010
:10138000012333603368DFF8D0B00024FC544445B7
:1013900004DB03B0BDE8F08F3260F3E759F82400B6
:1013A0003168C30707EB0105C1F5487105D5244A2B
:1013B0004310284608F0A2FF04E0C8B9214A284695
:1013C00008F09CFF1C4809F013F83060BAF1000FD8
:1013D0000CD008F1FF33A34208DDB0F5487F05D2F9
:1013E000431C20223A540022FA5433600134CEE7E1
:1013F000042801D1144AE2E71BD9026802F00F0366
:10140000042B06D1019102F053F9104A01990346C9
:10141000CFE7092B03D143685A465B10C9E7032B7A
:1014200008D1C2F30F13C2F34172C2EB8303084A1F
:10143000BFE70123074ABCE7790200209C05002092
:1014400014BE000060B3000066B300003FC400009B
:10145000BFB60000CAB60000B0B60000014B18705D
:10146000002070477802002010B501F047FE084CBC
:10147000231D01461F22184608F0D4FF08F0B8FFCC
:1014800004308008000140F004002060204610BDB8
:10149000540200202DE9F04F85B000F118010469D5
:1014A0000291D0E90232824601EB8404BD4F4169CA
:1014B000029800EB8109397803EB820529BB53F8C8
:1014C0002230B94A1E1203F07F03043552F823304C
:1014D000904643F0010318479AF8010004F0C8FB56
:1014E00000238AF8003021E03B7873B92B681E1284
:1014F00003F07F03043558F82330EAE7029B221DEE
:10150000D31AD82B26DD1A233B70DAF808209AF874
:10151000023039789AF80100AA1A921043EA02229E
:1015200004F0ACFB00238AF800303B70DAF8083096
:10153000ED1A029BE41AA9EB0309AD10A4104FEABF
:10154000A903CAF80C50CAF81040CAF8143005B004
:10155000BDE8F08F3B7826600BB11446D5E72B68C9
:101560001E1203F07F03144658F823300435B0E709
:10157000029B221DD31AD82B02DD1A233B70C4E72D
:101580002968216039782B1D11B114461D46BCE72E
:101590006B681E1203F07F03144658F82330083599
:1015A00097E7029B221DD31AD82B02DD1A233B702A
:1015B000ABE73B7805EB860626600BB11446A4E743
:1015C0002B681E1203F07F03144658F823300435AD
:1015D0007FE7029B221DD31AD82B02DD1A233B7012
:1015E00093E7724B53F8263023603B780BB11446D7
:1015F0008BE72B681E1203F07F03144658F8233044
:10160000043566E7694B54F8042D43F826203B78EF
:10161000002B7FF47AAF2B681E1203F07F03043592
:1016200058F8233055E7614B009353F82600FFF735
:101630004FFE834654F8040DFFF74AFE5844009BC2
:10164000400040F0010043F826003B78002B7FF477
:101650005CAF2B681E1203F07F03043558F823306B
:1016600037E7029B221DD31AD82B02DD1A233B70C9
:101670004BE7029B4B4534BF59F80C3C01232360D8
:101680003B780BB1144640E72B681E1203F07F0332
:10169000144658F8233004351BE7029B221DD31A49
:1016A000D82B02DD1A233B702FE7029B4B450FD24C
:1016B00059F80C3C06F180465B10C3EB8373033E84
:1016C000334459F8233023603B782BB114461CE790
:1016D00018233B700023F6E72B681E1203F07F03EC
:1016E000144658F823300435F3E6029B4B4519D2D3
:1016F00059F80C3C54F8042C5B1006F18046C3EBFF
:101700008373033E3344043C49F823203B78002B89
:101710007FF4FBAE2B681E1203F07F03043558F8EC
:101720002330D6E618233B70F0E7029B4B452DD2C1
:1017300059F80C3C06F180465B10033EC3EB837303
:10174000334459F82300FFF7C3FD221F834654F8A2
:10175000040C0092FFF7BCFD59F80C3C009A5B109A
:10176000C3EB837358441E44400040F0010049F825
:10177000260014463B78002B7FF4C7AE2B681E1260
:1017800003F07F03043558F82330A2E618233B709A
:10179000F0E7029B221DD31AD82B09DD1A233B70D8
:1017A000B3E600BF78020020B0B40000C88B01206F
:1017B00059F8263023603B780BB11446A5E62B6818
:1017C0001E1203F07F03144658F82330043580E6D8
:1017D00054F8043D49F826303B78002B7FF495AE51
:1017E0002B681E1203F07F03043558F8233070E68F
:1017F00059F826004FEA600B54F8040DFFF768FD16
:10180000584440003B7840F0010049F82600002B86
:101810007FF47BAE2B681E1203F07F03043558F86B
:10182000233056E6029BA4EB8604A3420BD83B78F8
:10183000002B7FF46AAE2B681E1203F07F03043581
:1018400058F8233045E6C54801F022FF3B78002BCD
:101850007FF45BAE2B681E1203F07F03043558F84B
:10186000233036E6002E05EB8605FFF65FAE3B78AB
:10187000002B7FF44AAE2B681E1203F07F03043561
:1018800058F8233025E654F8043D042B04D1002EEB
:1018900005EB8605FFF64AAE3B78002B7FF435AEAC
:1018A0002B681E1203F07F03043558F8233010E62E
:1018B00054F8043D042B04D0002E05EB8605FFF6FA
:1018C00035AE3B78002B7FF420AE2B681E1203F060
:1018D0007F03043558F82330FBE554F8040CC307A4
:1018E0000BD54010013800280ADB400040F0010011
:1018F00005EB860544F8040C18E6FFF7E9FCF1E770
:101900003B78043C002B7FF400AE2B681E1203F0E2
:101910007F03043558F82330DBE5029B04F10C0209
:10192000D31AD82B02DD1A233B70EEE5730003F4C3
:10193000FF7343F001032360DAF80830EB1A9D10BF
:101940009AF8023043EA05235B0043F00103636029
:10195000029BA9EB03035B1043F00103A360341265
:10196000E6B27F4B8AF8024091463A7853F8363017
:10197000CAF808301AB103F108054C46C5E503F171
:101980000C059B681E1203F07F034C4658F8233069
:101990009FE5029B54F8046C4B452FD1F70720D4E8
:1019A000042E17D9336803F00F03042B13D13046EC
:1019B00001F07EFE08F01CFDB0F5487F28BF4FF413
:1019C00048700630643003F03BFD70B9043DDDF82B
:1019D0000890ABE507D0002E14BF4FF4007007202D
:1019E000F0E70A20EEE70720ECE731469AF801001D
:1019F00004F05BF900238AF80030E8E759F80C3C62
:101A000057495A106FF0030353430C3B09EB03048F
:101A100049F8036059F8083C5A108AF80220D2B2FB
:101A2000C3F3552351F83220CAF8082059F8041C92
:101A30004FEA6109029901EB89093978043402EB14
:101A4000830500297FF461AD52F823301E1203F0A4
:101A50007F03043558F823303BE554F8040CFFF7B6
:101A600037FC1E288346A4EB860425DC00280BDC0B
:101A70003B78002B7FF449AD2B681E1203F07F03E7
:101A8000043558F8233024E501F026FBABF1030BB5
:101A9000344E834401F020FBA0EB0B00B042F9D898
:101AA0003B78002B7FF431AD2B681E1203F07F03CF
:101AB000043558F823300CE501238AF8003001F092
:101AC0000BFB0A385844CAF804002FE554F8040CFC
:101AD000FFF7FEFBA4EB8604061E0BDC3B78002B15
:101AE0007FF413AD2B681E1203F07F03043558F802
:101AF0002330EEE41C4B9E4202DD1D233B7004E5C7
:101B000001238AF8003001F0E7FA4FF47A7303FBFF
:101B100006000A38D7E700233046A4EB8604134EAC
:101B20001A462146FFF722FC3168114801F0DDFF1B
:101B3000104B316818600E4803F05EFF31680C48A6
:101B400004F0B8F83B78002B7FF4DFAC2B681E1252
:101B500003F07F03043558F82330BAE4DCB6000004
:101B6000D08301203F420F0080EE36009C0500200C
:101B700079020020080000203B78A4EB8604002BAB
:101B80007FF4C3AC2B681E1203F07F03043558F8B2
:101B900023309EE4504603F0B7FC3B78002B7FF4E3
:101BA000B4AC2B681E1203F07F03043558F82330C1
:101BB0008FE454F8043C002B44D154F80C0C10F082
:101BC000010B1ED04FEA600B4FEA4B0343F00103B9
:101BD00044F8083CBBF1000F40F388804FEA4B0308
:101BE00043F0010354F80C0C44F8043C54F8083C4E
:101BF000C107CBEB63032AD501335B0043F001033C
:101C000030E004281BD9036803F00F02092A01D130
:101C10004068D7E7042A09D101F04AFD0378002B78
:101C2000D2D0FFF7E8FA0BF1010BF7E7032A06D150
:101C3000C3F30F1BC3F34173C3EB8B0BC4E719232F
:101C40003B7062E44FEA630B0BF1FF3BC2E70428F1
:101C500049D9026802F00F02092A11D103F1020BDF
:101C600050F82B3049F826303B78002B7FF44DACF0
:101C70002B681E1203F07F03043558F8233028E444
:101C8000042A2BD1039309EB8603009301F010FD86
:101C9000039B83465E1C012E12DC5846FFF7ABFA0D
:101CA000A0EB0B06304601F019FF034670B103901C
:101CB00001F0FEFC3246594607F0D6FF039B05E0D3
:101CC0009BF80030013E23B912223A70009A13604B
:101CD000CAE75846FFF78FFA8346DCE7032A02D1AA
:101CE0001844037989E719233B700EE40435BBE7F8
:101CF000029A04EB86039B1AD82B0FDC0123002EDB
:101D000010DC3B78002B7FF400AC2B681E1203F034
:101D10007F03043558F82330FFF7DBBB1A233B70F1
:101D2000FFF7F3BB2360013E0434E8E7029A231D6A
:101D30009B1AD82B03DD1A233B70FFF7E6BB029BEF
:101D40004B452AD254F8040CFFF7C2FA002821DDD3
:101D500059F80C3C5B1083421CDBC3EB83731844C3
:101D600000F180400438A4EB860359F820201A6063
:101D70006FF003003B7800FB06440434002B7FF433
:101D8000C4AB2B681E1203F07F03043558F82330D0
:101D9000FFF79FBB20233B70EAE71823FBE7C04B0C
:101DA0001A68A4EB86036FF003001A603B7800FB0F
:101DB00006440434002B7FF4A8AB2B681E1203F0FA
:101DC0007F03043558F82330FFF783BB54F8043CF5
:101DD000042B3B780CBF05EB8605043C002B7FF4FD
:101DE00094AB2B681E1203F07F03043558F82330A0
:101DF000FFF76FBB54F8043C042B1CBF002344F8CE
:101E0000043C3B78A4F104021CBF05EB8605224686
:101E100013B11446FFF779BB2B681E1203F07F0342
:101E2000144658F823300435FFF753BB4FEA860CAD
:101E3000002EA4EB0C0015DC1C233B70002202607A
:101E40003B786FF0030000FB06440434002B7FF462
:101E50005CAB2B681E1203F07F03043558F8233067
:101E6000FFF737BB036886465B1084445EF8041BAB
:101E700011F0010202D10D233B70E0E749108B42C3
:101E8000A8BF0B46E645F1D15B0043F00102D6E75F
:101E90004FEA860C002EA4EB0C0015DC1C233B70D3
:101EA000002202603B786FF0030000FB064404341C
:101EB000002B7FF42AAB2B681E1203F07F0304353E
:101EC00058F82330FFF705BB036886465B1084444F
:101ED0005EF8041B11F0010202D10D233B70E0E714
:101EE00049108B42B8BF0B46E645F1D15B0043F089
:101EF0000102D6E754F8081C11F0010F4FEA8603DF
:101F00001ED054F8042CD0071AD55210B2EB610F32
:101F1000A4EB0303D4BF002204221A606FF0030075
:101F20003B7800FB06440434002B7FF4EEAA2B68B8
:101F30001E1203F07F03043558F82330FFF7C9BAA7
:101F400054F8042C6FF00100A4EB030BFFF768F9C1
:101F5000CBF80000E2E754F8081C11F0010F4FEA3B
:101F600086031ED054F8042CD0071AD55210B2EBB9
:101F7000610FA4EB0303B4BF002204221A606FF0C8
:101F800003003B7800FB06440434002B7FF4BDAA19
:101F90002B681E1203F07F03043558F82330FFF737
:101FA00098BA54F8042C4FF0FF30A4EB030BFFF762
:101FB00037F9CBF80000E2E754E9020181424FEA29
:101FC000860314D1E31A04221A606FF003003B78F1
:101FD00000FB06440434002B7FF497AA2B681E12E2
:101FE00003F07F03043558F82330FFF772BA042852
:101FF000A4EB030B01D8002315E0C307FBD403684F
:1020000003F00F03042BF6D1CB07F4D40429F2D943
:102010000B6803F00F03042BEDD1FFF77BF90028C9
:102020000CBF00230423CBF80030CEE754E90201B3
:1020300081424FEA860314D1E31A00221A606FF03E
:1020400003003B7800FB06440434002B7FF45DAAB8
:102050002B681E1203F07F03043558F82330FFF776
:1020600038BA0428A4EB030B01D8042315E0C307F6
:10207000FBD4036803F00F03042BF6D1CB07F4D491
:102080000429F2D90B6803F00F03042BEDD1FFF7FD
:1020900041F900280CBF04230023CBF80030CEE721
:1020A0000800002054F8081C11F0010F4FEA8603C5
:1020B0001ED054F8042CD0071AD55210B2EB610F81
:1020C000A4EB0303CCBF002204221A606FF00300CC
:1020D0003B7800FB06440434002B7FF416AA2B68DF
:1020E0001E1203F07F03043558F82330FFF7F1B9CF
:1020F00054F8042C0120A4EB030BFFF791F8CBF864
:102100000000E3E754F8081C11F0010F4FEA8603C2
:102110001ED054F8042CD0071AD55210B2EB610F20
:10212000A4EB0303ACBF002204221A606FF003008B
:102130003B7800FB06440434002B7FF4E6A92B68AF
:102140001E1203F07F03043558F82330FFF7C1B99E
:1021500054F8042C0220A4EB030BFFF761F8CBF832
:102160000000E3E754F8043C042BA4EB860314BFFF
:10217000042200221A606FF003003B7800FB064443
:102180000434002B7FF4C1A92B681E1203F07F03D7
:10219000043558F82330FFF79CB954F8080CFFF7C2
:1021A00097F8834654F8040CFFF792F85844A4EBD0
:1021B0008603400040F0010018606FF003003B7898
:1021C00000FB06440434002B7FF49FA92B681E12E9
:1021D00003F07F03043558F82330FFF77AB954F839
:1021E000080CFFF775F8834654F8040CFFF770F8F5
:1021F000ABEB0000A4EB8603400040F00100186048
:102200006FF003003B7800FB06440434002B7FF49E
:102210007CA92B681E1203F07F03043558F8233085
:10222000FFF757B954F8080CFFF752F8834654F8F3
:10223000040CFFF74DF800FB0BF0A4EB8603400005
:1022400040F0010018606FF003003B7800FB06448B
:102250000434002B7FF459A92B681E1203F07F036E
:10226000043558F82330FFF734B954F8040CFFF75D
:102270002FF88346B8B91F233B70A4EB86036FF099
:102280000300C3F800B03B7800FB06440434002B85
:102290007FF43BA92B681E1203F07F03043558F826
:1022A0002330FFF716B954F8080CFFF711F890FB2C
:1022B000FBFB4FEA4B0B4BF0010BDEE754F8040C31
:1022C000FFF706F88346B8B91F233B70A4EB8603DB
:1022D0006FF00300C3F800B03B7800FB0644043401
:1022E000002B7FF412A92B681E1203F07F03043524
:1022F00058F82330FFF7EDB854F8080CFEF7E8FF64
:1023000090FBFBF303FB1B0B4FEA4B0B4BF0010B5A
:10231000DCE754F8040CFEF7DBFF0028B8BF4042AE
:10232000A4EB8603400040F0010018606FF003004A
:102330003B7800FB06440434002B7FF4E6A82B68AE
:102340001E1203F07F03043558F82330FFF7C1B89D
:10235000A4EB860B012E0096DBF8000026D1FEF7D9
:10236000B7FF0346039307F095FF039B012BB8BF0C
:10237000012390FBF3F202FB1303009A1E446FF05B
:10238000030303FB024476003B7846F00106CBF8DA
:1023900000600434002B7FF4B8A82B681E1203F0F1
:1023A0007F03043558F82330FFF793B8FEF790FF0A
:1023B0000646DBF80400FEF78BFF0130831BD1E7F4
:1023C000A4EB860B5946304601F024FD3B78CBF850
:1023D00000006FF0030000FB06440434002B7FF480
:1023E00094A82B681E1203F07F03043558F823309D
:1023F000FFF76FB854F8080CFEF76AFF834654F8ED
:10240000040CFEF765FF0BEA0000A4EB8603400016
:1024100040F0010018606FF003003B7800FB0644B9
:102420000434002B7FF471A82B681E1203F07F0385
:10243000043558F82330FFF74CB854F8080CFEF771
:1024400047FF834654F8040CFEF742FF4BEA0000B6
:10245000A4EB8603400040F0010018606FF0030019
:102460003B7800FB06440434002B7FF44EA82B6815
:102470001E1203F07F03043558F82330FFF729B804
:1024800054F8080CFEF724FF834654F8040CFEF7BA
:102490001FFF8BEA0000A4EB8603400040F0010020
:1024A00018606FF003003B7800FB06440434002BF7
:1024B0007FF42BA82B681E1203F07F03043558F815
:1024C0002330FFF706B854F8040CFEF701FFC043B1
:1024D000A4EB8603400040F0010018606FF0030099
:1024E0003B7800FB06440434002B7FF40EA82B68D5
:1024F0001E1203F07F03043558F82330FEF7E9BFBE
:1025000054F8080CFEF7E4FE834654F8040CFEF77A
:10251000DFFE0BFA00F0A4EB8603400040F0010060
:1025200018606FF003003B7800FB06440434002B76
:102530007EF4EBAF2B681E1203F07F03043558F8CE
:102540002330FEF7C6BF54F8080CFEF7C1FE8346E1
:1025500054F8040CFEF7BCFE4BFA00F0A4EB860323
:10256000400040F0010018606FF003003B7800FB72
:1025700006440434002B7EF4C8AF2B681E1203F00F
:102580007F03043558F82330FEF7A3BF54F80C0C32
:10259000FEF79EFE834654F8080CFEF799FE8BFB6F
:1025A000002354F8040CCDE90023FEF791FEDDE989
:1025B0000023C0F1200CB0F1200103FA0CFC22FA38
:1025C00000F040EA0C005CBF43FA01F10843A4EBC1
:1025D000860E400040F00100CEF800003B786FF01E
:1025E000030000FB06440434002B7EF48EAF2B68FE
:1025F0001E1203F07F03043558F82330FEF769BF3D
:10260000A4EB860B59463046FEF754FC3B78CBF8DA
:1026100000006FF0030000FB06440434002B7EF43E
:1026200074AF2B681E1203F07F03043558F8233073
:10263000FEF74FBFA4EB860421463046FEF751FC5F
:102640003B78002B7EF461AF2B681E1203F07F03F2
:10265000043558F82330FEF73CBFA4EB860B5946EF
:102660003046FEF77FFC3B78CBF800006FF00300AC
:1026700000FB06440434002B7EF447AF2B681E1287
:1026800003F07F03043558F82330FEF722BFA4EB94
:10269000860421463046FEF7EFFC3B78002B7EF4A3
:1026A00034AF2B681E1203F07F03043558F8233033
:1026B000FEF70FBFA4EB860B59463046FEF74AFDE6
:1026C0003B78CBF800006FF0030000FB06440434B5
:1026D000002B7EF41AAF2B681E1203F07F03043523
:1026E00058F82330FEF7F5BE54F8040C00F0E0FF74
:1026F00054F8083CDA072AD4042B0CD91B6803F0E1
:102700000F03013B082B10D8DFE803F00521272336
:102710000F0F0F0F2500C24907F060FEA4EB8603E0
:10272000002814BF002204221A606FF003003B78D7
:1027300000FB06440434002B7EF4E7AE2B681E1227
:1027400003F07F03043558F82330FEF7C2BEB549C5
:10275000E2E7B549E0E7B549DEE7B549DCE7029BCA
:1027600004F1040BABEB0303D82B03DD1A233B70FE
:10277000FEF7CBBE00F0B8FC3B78400040F0010013
:10278000206013B15C46FEF7C0BE2B681E1203F03A
:102790007F035C4658F823300435FEF79ABE029B4F
:1027A00004F1040BABEB0303D82B03DD1A233B70BE
:1027B000FEF7ABBE00F090FC9E4B03EA40003B7876
:1027C00040F00100206013B15C46FEF79EBE2B680E
:1027D0001E1203F07F035C4658F823300435FEF7E1
:1027E00078BE029B04F1040BABEB0303D82B03DD93
:1027F0001A233B70FEF789BE00F076FC8E4B1B68F7
:1028000098423DBFC3F5830303F63713C018C01ABF
:1028100040003B7840F00100206013B15C46FEF7B9
:1028200074BE2B681E1203F07F035C4658F82330F9
:102830000435FEF74EBE00F057FC7F4B18603B7826
:10284000A4EB8604002B7EF460AE2B681E1203F00E
:102850007F03043558F82330FEF73BBE00F04CFCF4
:10286000B30068B9E41A3B78002B7EF44EAE2B68B7
:102870001E1203F07F03043558F82330FEF729BEFB
:10288000304627466D4EE41A01231A462146FEF7CC
:102890006DFD3068643002F0D3FD18B9043D3C464C
:1028A000FEF744BE9AF801203168654803F015FA36
:1028B00001238AF8003000F00FFC624A3368126886
:1028C000063302FB0300FFF7FEB800F015FCB3006F
:1028D00068B9E41A3B78002B7EF417AE2B681E1201
:1028E00003F07F03043558F82330FEF7F2BD30467D
:1028F0002746524EE41A002201232146FEF736FDF8
:102900003068643002F09CFD0028C7D04C4802F0CB
:102910005FFFCDE7FEF7A8FDA4EB860B3B78CBF875
:1029200000006FF0030000FB06440434002B7EF42B
:10293000ECAD2B681E1203F07F03043558F82330EA
:10294000FEF7C7BD3B78A4EB8604002B7EF4DDAD1B
:102950002B681E1203F07F03043558F82330FEF76E
:10296000B8BDA4EB860B584600F0F3FB3B78CBF8E0
:1029700000006FF0030000FB06440434002B7EF4DB
:10298000C4AD2B681E1203F07F03043558F82330C2
:10299000FEF79FBDA4EB860B584600F0DCFB3B78AE
:1029A000CBF800006FF0030000FB06440434002B5A
:1029B0007EF4ABAD2B681E1203F07F03043558F88C
:1029C0002330FEF786BDA4EB860B5946304600F057
:1029D000C5FB3B78CBF800006FF0030000FB06441A
:1029E0000434002B7EF491AD2B681E1203F07F039C
:1029F000043558F82330FEF76CBDA4EB860420465E
:102A000000F0DEFB3B78002B7EF47FAD2B681E12BE
:102A100003F07F03043558F82330FEF75ABD00BF9A
:102A2000ECB60000F4B60000FBB6000002B70000F0
:102A300007B70000FEFFFF7FA40500209C050020D3
:102A40007902002004000020A4EB860B5946304692
:102A500000F0F0FB3B78CBF800006FF0030000FBC8
:102A600006440434002B7EF450AD2B681E1203F094
:102A70007F03043558F82330FEF72BBDA4EB860402
:102A8000204600F089FC3B78002B7EF43EAD2B689D
:102A90001E1203F07F03043558F82330FEF719BDEA
:102AA0000121304600F046FC3B78002B7EF42DAD32
:102AB0002B681E1203F07F03043558F82330FEF70D
:102AC00008BD0021304600F035FC3B78002B7EF439
:102AD0001CAD2B681E1203F07F03043558F8233019
:102AE000FEF7F7BCA4EB860B584600F0E5FB3B78FD
:102AF000CBF800006FF0030000FB06440434002B09
:102B00007EF403AD2B681E1203F07F03043558F8E2
:102B10002330FEF7DEBCA4EB860B584600F0E0FB4A
:102B20003B78CBF800006FF0030000FB0644043450
:102B3000002B7EF4EAAC2B681E1203F07F030435F1
:102B400058F82330FEF7C5BCA4EB8604204600F0FD
:102B50009BFB3B78002B7EF4D8AC2B681E1203F055
:102B60007F03043558F82330FEF7B3BCA4EB86048A
:102B7000204603F06FFC3B78002B7EF4C6AC2B683C
:102B80001E1203F07F03043558F82330FEF7A1BC72
:102B9000A4EB860B584603F0F3FC3B78CBF800001F
:102BA0006FF0030000FB06440434002B7EF4ADAC50
:102BB0002B681E1203F07F03043558F82330FEF70C
:102BC00088BCA4EB8604204603F0BAFB3B78002BBC
:102BD0007EF49BAC2B681E1203F07F03043558F87B
:102BE0002330FEF776BCA4EB860B584603F0C0FBFF
:102BF0003B78CBF800006FF0030000FB0644043480
:102C0000002B7EF482AC2B681E1203F07F03043588
:102C100058F82330FEF75DBCA4EB8604214630460D
:102C200001F09CFB3B78002B7EF46FAC2B681E12EE
:102C300003F07F03043558F82330FEF74ABCA4EBB9
:102C400086042146304601F0AFF93B78002B7EF434
:102C50005CAC2B681E1203F07F03043558F8233058
:102C6000FEF737BCA4EB86042146304601F0ACFAEF
:102C70003B78002B7EF449AC2B681E1203F07F03D7
:102C8000043558F82330FEF724BCA4EB8604214613
:102C9000304601F0BFFA3B78002B7EF436AC2B684F
:102CA0001E1203F07F03043558F82330FEF711BCE1
:102CB000A4EB860B5946304603F03CFD3B78CBF83D
:102CC00000006FF0030000FB06440434002B7EF488
:102CD0001CAC2B681E1203F07F03043558F8233018
:102CE000FEF7F7BBA4EB860B5946304603F02AFDEE
:102CF0003B78CBF800006FF0030000FB064404347F
:102D0000002B7EF402AC2B681E1203F07F03043507
:102D100058F82330FEF7DDBBA4EB860B594630464E
:102D200003F018FD3B78CBF800006FF0030000FBC8
:102D300006440434002B7EF4E8AB2B681E1203F02B
:102D40007F03043558F82330FEF7C3BBA4EB860B92
:102D50005946304603F044FA3B78CBF800006FF058
:102D6000030000FB06440434002B7EF4CEAB2B683A
:102D70001E1203F07F03043558F82330FEF7A9BB79
:102D8000A4EB86042146304601F038F93B78002B4D
:102D90007EF4BBAB2B681E1203F07F03043558F89A
:102DA0002330FEF796BBA4EB86042146304601F0A3
:102DB00059FA3B78002B7EF4A8AB2B681E1203F067
:102DC0007F03043558F82330FEF783BBA4EB860B52
:102DD0005946304601F0C0F93B78CBF800006FF05F
:102DE000030000FB06440434002B7EF48EAB2B68FA
:102DF0001E1203F07F03043558F82330FEF769BB39
:102E0000A4EB86042146304601F06AF93B78002B9A
:102E10007EF47BAB2B681E1203F07F03043558F859
:102E20002330FEF756BB029BE31A9B10A4EB8604EB
:102E3000CAF810302146304602F00AFD3B78002BDC
:102E40007EF463AB2B681E1203F07F03043558F841
:102E50002330FEF73EBB029BE31A9B10A4EB860BCC
:102E6000CAF810305946304602F0F2FC3B78CBF8F5
:102E700000006FF0030000FB06440434002B7EF4D6
:102E800044AB2B681E1203F07F03043558F823303F
:102E9000FEF71FBB2DE9F84F224D0023002B03F155
:102EA000FF3706DA01F0FCFA02F0FCFD02F074FFD5
:102EB00019270026DFF878803046D8F80020B24283
:102EC00015DD2B68184C01339342A8BF00232B60FB
:102ED000D5F80090F02303FB09F304EB030AE35C4D
:102EE000A346EBB1022B04D15046FEF7D3FA3B4682
:102EF000D4E7012B0ED108B900F0EEF8F02303FB64
:102F000009F39B440949DBF80420821A8A429CBFDA
:102F10000222E254F02303FB09F3E35C022BE3D02B
:102F20000136CAE700000020707A01203F420F00FE
:102F3000A00500200B4B012200211A61C3F80415E3
:102F4000C3F808150421C3F810154FF44031C3F835
:102F500004131A60044B4FF480611960034B1A701C
:102F6000704700BF00A0004000E100E0CB0500205A
:102F700004207047F8B5D1E9004514F001002DD0C8
:102F800015F001002AD064101C2C3CD81F4F6D1086
:102F900041F288363B5DAE42A8BF2E46012B05D0DC
:102FA0000121204604F09CFD01233B55184B1B7862
:102FB0000BB9FFF7BFFF002D4FF00003154A0EDCE1
:102FC000154940F2DC50FF25D65CB44204BF21F81D
:102FD0001300D5540133042BF6D10420F8BDD15C85
:102FE0008C4203D10C4A22F81360F6E70133042B1C
:102FF000F5D10023D15CFF2901D1D454F2E701338C
:10300000042BF7D1E9E70020E8E700BFAC0500207A
:10301000CB0500201C0000200E00002070B5D1E977
:10302000004514F001001BD015F0010018D0641009
:103030001D2C28BF1B24164E335D012B05D001210A
:10304000204604F04DFD01233355124B6D10A5F1C0
:1030500010029A42104B04D94FF0FF321A6004203C
:1030600070BD0E4A1C600E4B93FBF5F313800D4AA6
:10307000127812B9FFF75EFFF1E70B4A0121916464
:10308000D2F848150B449BB2C2F84035E7E700BFC1
:10309000AC05002090860100180000200C000020E4
:1030A00020A10700CB05002000A00040002802DC82
:1030B0001C20FEF7D3B90120704704207047002878
:1030C00002DC1C20FEF7CAB90B68DB0701D40D2017
:1030D000F8E7002070470000024B01221A64D3F881
:1030E000400570470080004008B5FFF7F5FF4FF43A
:1030F0007A73B0FBF3F008BD0120704700487047B9
:1031000068B700001D20704770B5054D2B5C8B42E1
:1031100004460E4602D004F0E3FC2E5570BD00BFFD
:10312000AC05002070B50024084D2646635D012BD8
:1031300008D10021204604F0FDFC0021204604F0C7
:10314000CFFC665501341D2CF0D170BDAC050020BC
:1031500070470F2070473B2070470000F8B50B68A0
:10316000DA0707460D4604D40D20FEF777F9012053
:1031700007E05B10062B05D103F008F9400040F092
:103180000100F8BDF3D80C4A0C4E52F82340335DD1
:103190002BB10021204604F0A3FC00233355012F5E
:1031A00006DD6B68042B03D10221204604F098FC55
:1031B000204604F09FFBE1E74CB70000AC0500207F
:1031C00070B50468E20702D54568EB0704D40D200A
:1031D000BDE87040FEF742B964101C2C23D8124E93
:1031E000335D012B18D00121204604F079FC012326
:1031F0001B2C335510D10D4BDA6E0D4B202AB8BF66
:103200004FF0A04302F01F0203EB8203D3F8002724
:1032100042F44072C3F80027A5F34A012046BDE8F6
:10322000704004F00BBC70BDAC05002054C700001A
:103230000003005070B50C68E30704D40D20FEF7BE
:103240000DF9012070BD64101C2C14D8012814DD68
:103250004B68042B14BF002502250A4E335DAB4298
:1032600004D02946204604F03BFC3555204604F0A6
:103270007DFC012803D00020E4E70025EDE70420D1
:10328000E0E700BFAC05002013B50A4A044692E807
:10329000030022686B46042A83E8030019464FF0B6
:1032A000020003D100F090FF02B010BD00F0B2FFA9
:1032B000FAE700BF14B7000010B5084C63792BB1D2
:1032C0000021052004F00CFC00236371052004F0AC
:1032D0004DFC00280CBF0420002010BDAC050020D0
:1032E00010B5084CE37A2BB100210B2004F0F8FB59
:1032F0000023E3720B2004F039FC00280CBF0420EB
:10330000002010BDAC05002007480849084A0123E9
:1033100043604B6053600023C0F80035C1F80035AE
:10332000C2F80035704700BF00C0014000100240E5
:10333000002002401C2870B504460D4625D8134EC7
:10334000335C012B04D0012104F0CAFB0123335567
:103350001C2C12D1FFF7D8FF0D4B1A6F0D4B202AF2
:10336000B8BF4FF0A04302F01F0203EB8203D3F873
:10337000002742F44072C3F80027291C204618BFDA
:103380000121BDE8704004F0D5BB70BDAC05002044
:1033900054C70000000300500368D90702D40D2071
:1033A000FEF75CB841680A1F514251415810FFF7BF
:1033B000C1BF0000F8B5314CD4F84031B3B100239F
:1033C000D4F84055C4F840312D4B186800280DDB67
:1033D0002C4A1178B1FA81F14909117004F0AAFB65
:1033E000294B1B882B449BB2C4F84035234AD2F8A2
:1033F0004431002B37D00021244ED2F84445C2F886
:1034000044113378224D0C3433B12B68032B03D88D
:10341000204AD05C04F08EFB2B681E4F01335A42C9
:1034200002F0030203F0030358BF53422B60002253
:10343000042B194618D00133F81810F8010CFF2896
:1034400001D10122F4E702B12960012104F072FBED
:10345000012333702A68104B33F812302344074A93
:103460009BB2C2F84435F8BD4FF0FF332B60002308
:10347000337004F58C435033F1E700BF00A00040E7
:1034800018000020CA0500200C000020C9050020FB
:10349000A80500201C0000200E000020094B0A494E
:1034A00040F2DC521A805A809A80DA80074A002360
:1034B0001370074AFF20087048708870C870136046
:1034C000704700BF0E0000201C000020C90500202E
:1034D000A8050020024B4FF0FF321A60704700BF72
:1034E00018000020024A0348062101F06DBF00BF0A
:1034F0001CB7000046BF000038B54FF4E1311D484D
:1035000003F0CEFF1C4B03210122C3F80815002451
:1035100004211A61C3F810151A60C3F804454FF06E
:1035200080430221C3F818150A209A6004F0DCF9E0
:10353000124A2346FF21995401331D2BFBD1104B16
:10354000104D01221A6000200F4A0423014614681E
:10355000002CFCD02C681160013B44EA0020F6D11D
:103560000A4B01221A6004F0F5F8BDE8384001F07A
:1035700033B800BFF079012000800040AC05002086
:1035800000D0004008D5004000D1004004D00040E9
:10359000F8B506460948094F0C4603F0C1FF8442BE
:1035A000A8BF04463546AB1B9C4205DD384603F0F8
:1035B000BDFF05F8010BF6E72046F8BDF0790120C4
:1035C0000146014803F071BFF079012010B5054CA8
:1035D000204603F077FF20464FF4E131BDE810406C
:1035E00003F05EBFF0790120C3070CD4064B1B68C3
:1035F000834208D8054B1B68984204D850F8043C15
:10360000002B18BF18467047D4050020D0050020B5
:103610000B4908B50122002341F823200133642B14
:10362000FAD1084B1A60084B084A1846002106F0E8
:103630003FFB074B40F8043F064B186008BD00BF36
:10364000C88B012008000020D80500207067010009
:10365000A09D0500CC050020034B044A1A60044BD2
:10366000044A1A60FFF7D4BFD4050020D805002013
:10367000D0050020486D0120044B1B681868C0F37A
:103680000F10023820EAE070704700BFCC05002020
:1036900000B59BB00246054901A806F063FE01A8EB
:1036A00002F0B3F802F078FBFCE700BFEFB70000D0
:1036B000C30713D4042802D812D00B4870470368FC
:1036C00003F00F03042B01D104307047092B09D0FC
:1036D000064A0748032B18BF104670470548704735
:1036E000054870470548704760B30000DAB700002E
:1036F000E3B70000C9B7000066B30000D3B700000D
:10370000064B074900201A6843F8040CC2F30F1255
:10371000023203EB82038B42F5D37047DC050020B5
:10372000486D01202F4B304A1868304B2DE9F0418D
:103730001C682F4D136803F00F01072928D8136860
:10374000C3F30F13023302EB8302AA42F2D32949D7
:10375000002251F82200FFF747FF41F82200013212
:10376000642AF6D1244A1068FFF73EFF1060234A0E
:10377000106810B1FFF738FF1060214B214C1E6814
:103780000021F0274FF03C08B14214DBBDE8F08186
:10379000C3F30F1302EB83039A42D0D01968CE070C
:1037A00007D4884205D28C4203D351F8041C01B1DE
:1037B0001960043BF0E707FB01F31A191B5D0BB915
:1037C0000131E1E71269551E08FB012204EB820278
:1037D0001832002DF4DB52F8040DFFF705FF013D10
:1037E0001060F6E7D4050020DC050020D00500209D
:1037F000486D0120C88B012008000020486D012081
:10380000A0050020707A0120C307F0B540D4214BF9
:103810001C68A0423CD3204B1D68A84238D850F801
:10382000043CABBB03680246C3F30F13012673B914
:10383000904242F8046C2BD0116851F8043C51F8C6
:103840002370176041F82320013B0A46EFE752F846
:103850002310CF0702EB830C18D48C4216D88D426C
:1038600014D351F8047C8FB90F6807F00F0EBEF126
:10387000070F08D9CCF8007042F8043C0B680A60C6
:10388000C3F30F13E1E741F8046CD0E7013BCEE747
:10389000F0BD00BFD4050020D00500200D4930B593
:1038A0000D4C0B461A6853F8045CC2F30F12901CBF
:1038B00065B18B4214BF0A46002243F8042C01EB89
:1038C000800103EB8003A342ECD330BD12011A60E8
:1038D000F7E700BFDC050020486D0120144B2DE9FF
:1038E000F041144C1E464FF000083268C2F30F1727
:1038F00012070FD07D1C9E424FEA850505D0184661
:103900002A46314606F0BBF903465A1904352B44C2
:10391000C2F80080023706EB8706A642E5D3E41A18
:10392000A410013C044A24011C601360BDE8F0812E
:10393000DC050020486D0120CC0500202DE9F04178
:103940009AB0FFF7C9FB214D0746002455F8240023
:103950000134FFF759FF642CF8D11D4B1868FFF7AD
:1039600053FF1C4B186808B1FFF74EFF1A4DDFF8E4
:1039700074800026D8F800309E4218DBFFF78EFFD7
:10398000FFF7D0FEFFF7AAFFFFF7A6FB134B144982
:103990001B681B68C3F30F13C21B023B01A806F090
:1039A000E1FC01A801F031FF1AB0BDE8F0812B78ED
:1039B00013B90136F035DDE72C69013C002CF8DB4A
:1039C00005EB84039869FFF71FFFF6E7C88B01201A
:1039D00008000020486D0120707A0120CC050020ED
:1039E000A9B70000A00500202DE9F8431B4C23686F
:1039F0001B684D1CC3F30F139D42064688461746AD
:103A0000A1460CDBFFF79AFF23681B68C3F30F1373
:103A10009D4204DB0A20BDE8F843FDF71FBD08F115
:103A20000202D9F800009B1A1B0140F82230002343
:103A300040F8043C06F00F06034646EA08169400D8
:103A400043F8046B0119083CC9F800101C44A34258
:103A500001D3BDE8F88343F8047BF8E7CC050020E8
:103A6000F8B510F0010704460E462CD1174B1B6821
:103A7000834228D8164B1B68834224D9154D2860F1
:103A80000068012200F00F00FFF7AEFF2C682F60E6
:103A90000546C0B12146043051F8042BC2F30F1281
:103AA000B242A8BF3246920006F0DEF8FFF728FEC9
:103AB00044F8045CFFF736FE2268074B44F8047CA8
:103AC000134023602C462046F8BD00BFD4050020DB
:103AD000D0050020486D0120F0FF0F00011D0022DD
:103AE000042091FBF0F1FFF77FBF38B5054608468B
:103AF0000C46FFF7F3FF50B1C21C2B46591B8C42FA
:103B000006DC002CACBF0419041C0023237138BD53
:103B100013F8011B02F8011FF0E7F0B502289BB073
:103B20000C4604DC1C20FDF799FC1BB0F0BD0868B6
:103B3000C20706D4042804D9036803F00F03042B3A
:103B400001D00E20EFE74B6813F00107F9D1042BE9
:103B5000F7D91B6803F00F03042BF2D18B68DB0746
:103B600001D40D20DFE7FFF7A3FD06466068FFF7ED
:103B70009FFDA5681AAC014604F8647D6D103046BF
:103B800002F0ACFF29466423224603F009F82046E0
:103B900006F02EFC01462046FFF7A7FFC5E7000010
:103BA00010B50446ADF5806D10B9FFF797FF0BE037
:103BB00002F0BBFE0138062827D8DFE800F008082D
:103BC00010172804230000200DF5806D10BD20463D
:103BD00002F025FF011B2046FFF787FFF4E7204690
:103BE00002F0D1FE400040F00100EDE769464FF4DD
:103BF0008062204602F0E1FE684606F0F9FB0146CD
:103C00006846E9E704210348E6E70020CDE7042001
:103C1000DAE700BF38B80000022838B50C4604DCEB
:103C20001C20BDE83840FDF719BC0868C10706D460
:103C3000042804D9036803F00F03042B01D00E20DD
:103C4000EFE76368DA07FAD4042BF8D91B6803F0AE
:103C50000F03042BF3D1A368DB0701D40D20E0E7A9
:103C6000FFF726FD05466068FFF722FDA4680146C0
:103C70006410284602F032FF214602F06EFFBDE8D4
:103C80003840FFF78DBF012838B50C4604DC1C20F6
:103C9000BDE83840FDF7E2BB0868C10706D4042838
:103CA00004D9036803F00F03042B01D00E20EFE7C3
:103CB0006368DA07FAD4042BF8D91B6803F00F0302
:103CC000042BF3D1FFF7F4FC05466068FFF7F0FC26
:103CD0000146284602F002FF02F07EFF400040F05D
:103CE000010038BD012870B505460C4604DC1C20D7
:103CF000BDE87040FDF7B2BB0868C10706D40428D0
:103D000004D9036803F00F03042B01D00E20EFE762
:103D10006368DA07FAD4042BF8D91B6803F00F03A1
:103D2000042BF3D1FFF7C4FC06466068FFF7C0FC24
:103D3000022D014615D0A468E30712D56410304661
:103D400002F0CCFE054602F0F0FD012812D1002C55
:103D500002DD0135012C07D12846BDE87040FFF790
:103D60001FBF4FF0FF34EAE7284602F066FE013C31
:103D70000546EFE70228EFD1002CEDDD0135012CDF
:103D8000EAD000221146284602F081FE02F055FEDC
:103D9000013C0546F3E70000086810B510F0010487
:103DA0001AD0441007EE904A9FED187AF8EEE77AA1
:103DB00067EE877A17EE900A05F0B8FB03F0DEFF96
:103DC0000022134B05F00AFC03F08EFF05F0B6FE4F
:103DD000400040F0010010BD042812D9036803F030
:103DE0000F03042B07D1FFF763FC0A22214606F0DC
:103DF000C3FB0446D6E7032B03D10A222146043035
:103E0000F5E70D20FDF72AFBCCE700BFD3023739D9
:103E10000000D040086808B5C30706D4042804D9B8
:103E2000036803F00F03042B04D00E20BDE8084004
:103E3000FDF714BBFFF73CFC0378232B08BF0130D0
:103E40001022002106F098FB00F10053B3F1804FDF
:103E500001D31420EAE7400040F0010008BD000053
:103E6000024A0348062101F0AFBA00BF08B80000BB
:103E700000B80000002070471E20FDF7EFBA1E209A
:103E8000FDF7ECBA1E20FDF7E9BA1E20FDF7E6BAF1
:103E90001E20FDF7E3BA1E20FDF7E0BA1E20FDF755
:103EA000DDBA1E20FDF7DABA1E20FDF7D7BA1E20B4
:103EB000FDF7D4BA1E20FDF7D1BA1E20FDF7CEBA09
:103EC0001E20FDF7CBBA1E20FDF7C8BA1E20FDF755
:103ED000C5BA1E20FDF7C2BA024A0348112101F0FB
:103EE00073BA00BF74B80000FCB80000034B012295
:103EF0001A60034B1868904010437047686D0120AA
:103F00004C6D01202DE9F041EFF31082012302F006
:103F1000010883F310881549154C0968154D164E94
:103F200001398B4003274FF00E0C4FF00B0E002B86
:103F300018D02168296018420AD072461100013950
:103F4000FDDC2168316039000139FDDC5B08EEE7FA
:103F500039000139FDDC2168316062461100013908
:103F6000FDDCF3E788F31088BDE8F0812000002035
:103F70005C6D0120080500500C05005070B5084E1E
:103F8000084D002456F824000021FFF7BDF855F82D
:103F9000240000210134FFF7B7F8052CF2D170BDE1
:103FA000E8B9000034BD000008B5054B00221A60D6
:103FB000044B1B680BB102F057FC002008BD00BF8A
:103FC000646D01205478012010B5041E0ADA002423
:103FD000074B53F8242001239340064A1360064AF6
:103FE000136010BDFFF78EF8A042F0DDF0E700BFD0
:103FF00054C700005C6D0120180500502DE9F843FE
:10400000344B1B680C461BB94FF0FF30FFF7DCFF49
:10401000246814F0010525D0C4F34743C4F34720B6
:10402000C4F3470240F2596540435B4390FBF5F10E
:1040300093FBF5F0000240EA01401346534393FB23
:10404000F5F31843244B1B68202B01BF234BC4F30B
:10405000456453F8243043EA0020FFF753FF002063
:10406000BDE8F883042CFAD9236803F00F03092B69
:10407000F5D154F8046FDFF86080DFF860907610B7
:1040800040F25967B542EADA54F8042FD3071FD536
:10409000C2F34743C2F34720C2F3470140435B43A7
:1040A00090FBF7FC93FBF7F0000240EA0C400B4654
:1040B0004B4393FBF7F31843D8F80030202B02BF93
:1040C000C2F3456259F8223043EA0020FFF71AFF95
:1040D0000135D7E75C6D012020000020D8BB00002F
:1040E00008B50B68DA074CBF5B104FF0FF330128AF
:1040F0000DDD4A68042A14BF1822202205491846FB
:104100000A60FFF725F8FFF75FFF002008BD1822BF
:10411000F4E700BF2000002010B510F0010402D029
:104120004410204610BD042812D9026802F00F0284
:10413000042A07D1FFF7BCFA0A222146BDE8104045
:1041400006F01ABA032A03D10A2221460430F5E701
:104150000D20FDF783F9E4E7086810F0010370B55E
:104160001CD0FFF7D9FF0346203B5E2B27D8154C08
:1041700003EB83030022012110462344052A1AD0B1
:104180009E5C052410252E4218BF4018013C4FEAC2
:1041900041014FEA6505F6D10132EFE70428E3D982
:1041A000026802F00F010429DED1C2F30F13002BC5
:1041B000DAD00379D8E7400040F0010070BD01205B
:1041C000FCE700BFFCB9000038B508680D46FFF7F2
:1041D000A3FF04466868FFF79FFF621E042A01469A
:1041E00012D8431E042B0FD8084803EB8303134453
:1041F0000568012202FA03F32B430360044B1B689A
:1042000013B1204602F031FB002038BD646D01205F
:104210005478012038B508680D46FFF77DFF044645
:104220006868FFF779FF621E042A014614D8431E0E
:10423000042B11D8094803EB83031344012202FA2B
:1042400003F3026822EA0302054B02601B681BB1FC
:104250000022204602F009FB002038BD646D0120D9
:10426000547801202DE9F04F054685B008680C46CA
:10427000FFF752FF022D01903CDD6068FFF74CFF15
:104280000746A068FFF748FF0446231DDFF8C8A0D3
:104290000293661E4FF00108029B9E4206F101093F
:1042A00035D006EB8602531E07F1050B3D460393FE
:1042B000AB4522D0042E19D86A1E042A16D8039BB7
:1042C000019ADAF800005919224B4FF0010C18EA54
:1042D000020E0CFA01F11B6811D00143CAF800105C
:1042E00023B162464946284602F0BFFA4FEA480821
:1042F0000135DDE701242746C7E74E46CCE720EA33
:104300000101CAF80010002BF0D07246EAE73D1D0B
:10431000042D1BD8012C19D1DFF83C80DFF8349034
:104320000026D8F8003004FA05F223EA0203C8F8A0
:104330000030D9F80030013623B100223146781D13
:1043400002F093FA052E05F10505EAD1002005B02B
:10435000BDE8F08F54780120646D0120086808B52D
:10436000C30703D5FFF7D8FE054B1860054B1B6844
:104370001BB1034B186802F079FA002008BD00BF9A
:10438000646D0120547801202DE9F3413F4D4FF435
:1043900041732C68ADF804300A238DF806305CBBFD
:1043A000FFF7ECFDDFF8F480264658F8267001216F
:1043B0003846FEF7A9FE01360021384603F0BAFB65
:1043C000052EF2D100260DF1040816F8087001211F
:1043D0003846FEF799FE01360121384603F0AAFB64
:1043E000032EF2D1FEF778FE294B186001232B60D3
:1043F000204602B0BDE8F081012C1CD1244C266877
:10440000FEF76AFE864298BF801BC72801D80024A9
:10441000EEE700210420FEF777FE00210320FEF7DF
:1044200073FE00210A20FEF76FFEFEF755FE022301
:1044300020602B60EBE7022C21D1154B1C68FEF7A6
:104440004BFE844298BF001BB0F57A6FDFD3042087
:1044500003F050FA0446032003F04CFA06460A2003
:1044600003F048FA34442044C0F53F6003230D3084
:1044700090FBF3F0074B1860012003F03BFA064A6B
:1044800000232B6013600124B2E700BF586D0120A8
:10449000606D01204C6D0120686D012034BD00006D
:1044A0002DE9F843434E326852B9434B1B683BB980
:1044B000424B1B68002B74D0BDE8F843FFF764BF84
:1044C0003F4D2C6884BB3D4B1B68002B65D13A4A9D
:1044D000336810681146002865D13A4F3A4EDFF82C
:1044E000F4800B60002157F82400FEF70DFE56F80B
:1044F000249001214846FEF707FEB9F1220F10D89B
:1045000058F82920314B1F2AD8BF4FF0A04302F0A2
:104510001F0203EB8203D3F8002742F44072C3F872
:1045200000270134052CDDD12B68264EDFF888905A
:10453000254F002BCCBF03F1FF330423002156F895
:104540002300FEF7E1FD2A68214B53F82280002466
:1045500004EB840101EB0803D9F8001057F824009C
:10456000194101F00101013403F0E4FA052CEFD107
:104570002B68012156F82300FEF7C6FD2B680021A9
:1045800056F8230003F0D6FA2B68013393FBF4F4BA
:1045900004EB84041C1B2C6003E0FFF7F5FE0028ED
:1045A00095D1BDE8F883002B97D11360BDE8F8439F
:1045B000FFF7E4BC646D0120546D0120686D01209B
:1045C000506D0120E8B9000034BD00000003005028
:1045D000D8BC000054C700004FF0FF30FFF7F4BC18
:1045E000024A0348092100F0EFBE00BFECBC000006
:1045F00048BD00004FF0805310B51A69094B0224E2
:10460000C3F8044522F00302884203D30022C3F812
:10461000042510BDD3F80044002CFBD0C3F80805D6
:104620001044F1E700E00140002815BF4FF4D2210B
:104630004FF4B4214FF4B4204FF49620FFF7DABFC3
:1046400000280CBF4FF496234FF4B4231868030ED0
:10465000532B0CBF20F07F4000207047064B0122F7
:10466000C3F80425D3F80024002AFBD000220160FF
:10467000C3F80425704700BF00E00140002821F086
:104680007F4141F0A6410CBF4FF496204FF4B42077
:10469000FFF7E4BF0A4B30B50124C3F804450029F5
:1046A00003DC0022C3F8042530BD52F8044BD3F8D4
:1046B0000054002DFBD040F8044B0139EFE700BF58
:1046C00000E0014038B54C68023405460A462146F0
:1046D000FFF7E0FF05EB840038BD0000124B1B68BC
:1046E000002B0BBF4FF4B4224FF4D2224FF4962389
:1046F0004FF4B42328B91A1DDB79522B08BF10469A
:10470000704782420DD9C378522B0AD143680233D5
:1047100000EB8300824204D9C378522B18BF0020DB
:1047200070470020704700BF6C6E01202DE9F041FA
:104730000020B4B0FFF7D2FF0024DFF8A4800546C4
:10474000274626464DBB224D2868FFF779FF3B469A
:104750003246CDE900401F4902A805F003FE02A839
:1047600001F053F81C4B1A682B68002B0CBF4FF458
:1047700096234FF4B423D21A4FF470416423534369
:10478000009193FBF1F302A8144905F0EBFD02A898
:1047900001F03BF834B0BDE8F08169682A68019106
:1047A0008B1C1F44D1B2C2F307239C42C2F30742C1
:1047B000009102A84146B8BF1C4605F0D3FD02A8EF
:1047C00001F023F82846FFF789FF01360546B9E7CF
:1047D0006C6E012052BE0000706E0120FCBD000016
:1047E0003EBE000070B50020FFF72AFF05460120FD
:1047F000FFF726FF0C4B1E68B6FA86F485424FEA97
:104800005414B8BF054620461C60FFF70DFF074A49
:10481000074B002E18BF1346064A691C2046BDE808
:1048200070401360FFF72ABF6C6E012004B00400D3
:1048300004A00500706E012070B50020FFF700FF96
:1048400002460120FFF7FCFE1F4E204C054672B9C0
:1048500068B94FF4D2214FF49620FFF7CBFE012127
:104860002846FFF70BFF1A4B3560236029E0AA4268
:1048700008DD00233360164B23604FF4B421236816
:10488000002017E001233360124B23604FF4D22144
:10489000F5E7120E522A08D000B123600E4800F04E
:1048A000B4FFBDE87040FFF79DBF5A68023203EBCA
:1048B000820301208B4205D21A68551CE9D10028D9
:1048C000D3D170BD2160FCE76C6E0120706E0120B9
:1048D00004B0040004A0050017BE000010B50020BD
:1048E000FFF7FCFE014608B9084610BD8478FFF7C3
:1048F000F5FEDA2C08BF0146F5E700002DE9F04F80
:104900004FF480729FB05F4C5F48002105F0D0F9F2
:104910004FF4807200215D4805F0CAF9D4F8009088
:10492000B9FA89F84FEA58184046FFF77DFEA246CB
:10493000574B584C0020B9F1000F08BF1C46FFF739
:10494000CDFF064638BB4846FFF77AFE524D411C64
:104950004046FFF793FECAF800802C60FEF736FE53
:10496000DAF800302A68002B0CBF4FF496234FF47E
:10497000B423D21A4FF4704164235343009193FB44
:10498000F1F305A8454905F0EDFC05A800F03DFF51
:104990001FB0BDE8F08F3568C5F30743A3F10A02E5
:1049A000092AC5F3072546D8374B595D91BB10221C
:1049B0003B48DFF8ECB005F07BF937463A68C2F3C4
:1049C00007218D4209D1C2F307410B2926D01329B3
:1049D0002BD00A2901D1CBF800703846FFF77EFEB4
:1049E00007460028EAD12E4F396881B12046FFF7EB
:1049F00069FE0123044657F8231029B1204603938A
:104A0000FFF760FE039B04460133042BF3D11E4ADB
:104A1000012353553046FFF761FE92E7D2B2022AD6
:104A2000DBDC0BEB82025760D7E7102200215846EF
:104A300005F03EF9D1E7A3F11502082AEAD8134A96
:104A4000525D002AE6D1152B0CBF314600213046BD
:104A50000368C3F30742152A0ED01D2A08BF0021A0
:104A6000FFF73CFE0028F3D119B12046FFF72AFEDC
:104A700004460123054ACCE7C3F307239D4208BF40
:104A80000146EDE76C6E01206C6D0120746E012013
:104A900004A0050004B00400706E0120E1BD000018
:104AA000588D0120FFF72ABF2DE9F84FDFF8A8B095
:104AB000274F03339246042293FBF2F6DBF80030D3
:104AC000B41C002B3B684FEA84040CBF4FF4B422A3
:104AD0004FF4D22223449A4281460D46B84614D25E
:104AE000FFF70CFFDBF80030002B3B680CBF4FF4E6
:104AF000B4224FF4D22223449A4206D2154800F041
:104B000084FE00273846BDE8F88F2D025FFA8AF14F
:104B100041F0A441ADB2D8F800700D434FEA09410D
:104B200001F47F0129433846FFF798FD07F1080596
:104B30003146381DC8F80050FFF790FD1EB10A9AA3
:104B40002846FFF7A7FD083C2544C8F80050D9E7E0
:104B5000706E0120BBBD00006C6E012030B59BB0B3
:104B6000FFF76AFE00214FF4FF621D4805F0A0F830
:104B7000FFF7B4FE1A490024A0B9194B024653F8B6
:104B8000301001B101320130FF28F8D1154901A8D8
:104B900005F0E8FB01A800F038FE134800F035FEF0
:104BA0001BB030BD0368C3F307420A2A0BD1C3F31D
:104BB0000722FF2A04D001EBC20541F832002B7115
:104BC000FFF78CFDD8E7132AFAD1C3F30723FF2B95
:104BD0001EBF01EBC30241F833401471F0E700BF80
:104BE000D083012087BE00009BBE00000A4B00223C
:104BF000C3F8002101225A60D3F80021002AFBD01B
:104C00000022C3F80C2101229A60044B0222C3F84F
:104C100080211A60704700BF0010004000E100E0F2
:104C2000074B0222C3F88020064B0022C3F8102154
:104C300001221A61D3F81021002AFBD0704700BF6F
:104C400000E100E00010004008B504490A780AB10C
:104C5000FFF7E6FF0020087008BD00BF756F012058
:104C60004FF08053586E400040F001007047000044
:104C7000024B1868400040F001007047F86F0120B7
:104C8000024B1868400040F00100704724000020EB
:104C9000024B1868400040F001007047FC6F012093
:104CA00070B504460D461646FEF71EFA4FF08053C7
:104CB00001225B6E6270E270020A23F00043A2716F
:104CC000020CE2711A0A002160716372000EA27276
:104CD0001A0C1B0E2670A17025712072E2722373CC
:104CE00070BD000010B5054C204605F081FB014663
:104CF0002046BDE81040FEF7F8BE00BF017001205D
:104D0000104B1B685A1C10B514D0CBB1012B13D01B
:104D1000022B13D0042B13D00B4C0C4A052B08BFCD
:104D20001446204605F064FB01462046BDE81040CD
:104D3000FEF7DBBE064CF4E7044CF2E7054CF0E767
:104D4000054CEEE72800002031BF000037BF00000F
:104D50002CBF0000FBB60000F4B6000010B52148DF
:104D60000278002A3DD14FF08043C3F80021012290
:104D70001A60D3F80021002AFBD01B4B1B4C0022E9
:104D80000721C3F80C25C3F808151949C3F81025E5
:104D9000C3F81C15C3F824250121C3F82C250822CB
:104DA000C3F83015C3F81425C3F818450224C3F816
:104DB00034454FF6FF74C3F83C450E4CC3F83845F4
:104DC0001824C3F85445C3F80423D3F8002242F052
:104DD0001002C3F80022084AC3F80425FFF706FFB3
:104DE000017010BD756F012000100040200004020A
:104DF0007469627521100100766F0120F8B5104BBF
:104E00001B7804460BB9FFF7A9FF0E4E3378ABB100
:104E10000D4A1278D21A02F003010C4A02EB411239
:104E200002F1200710685168254603C50832BA42CE
:104E30002C46F7D1013B33700120F8BD1846FCE742
:104E4000756F012000700120746F0120766F0120C2
:104E500030B5002889B02ADD0D6815F0010426D18F
:104E6000042D26D92B6803F00F03092B21D16B6881
:104E70003F2B1EDD6846FFF7C1FFB0B19DF8002053
:104E80000435A242A8BF1DF8043004F10104A6BFF6
:104E90005B0043F001030123202C45F8043FF0D1CF
:104EA000054BDDF809201A60042009B030BD002050
:104EB000FBE72046F9E700BFFC6F012030B5384B17
:104EC0001B788BB00BB9FFF749FF02A8FFF796FFDD
:104ED00010B900200BB030BD9DF808300B2BF8D96D
:104EE0009DF80930012BF4D19DF80B30012BF0D146
:104EF0002C4D2D4C2D4ADDF8111000232B60237012
:104F00009DF80C3013602A4A116023B9DDF8153082
:104F10002B6000230FE0012B11D1DDF815309DF837
:104F200019202B600DF11A010E239342A8BF1346DE
:104F300000229A4230D10022E2540420CAE7022B18
:104F400005D19DF8152012230DF11601EDE7042B74
:104F50000DD10AAA6B4652F8130D516803C3DDE95F
:104F6000000102F033FE04F0E9FD2860D1E7052BD3
:104F7000CFD10AAA6B4652F8130D516803C3DDE97D
:104F8000000102F023FE04F0D9FD9DF81D202860E9
:104F90000A230DF11E01C8E7885CA0540132C8E75E
:104FA000756F0120F86F012001700120280000209A
:104FB000FC6F012010B5154B1B7804460BB9FFF7A9
:104FC000CDFEFFF72DFE124B0022C3F80445C3F8B7
:104FD000002101221A60D3F80021002AFBD0002210
:104FE000C3F80C2101229A60094AD2F80C31002B37
:104FF000FBD0084B1978084B03EB4113C2F804357A
:10500000FFF70EFEBDE81040FFF7F0BD756F012001
:1050100000100040746F0120766F012000B5002859
:1050200089B01DDD0B6813F0010219D1042B17D9CB
:10503000196801F00F01092912D159683F290FDDC4
:10504000043353F8040F10F0010118BFC0F34701F7
:105050000DF802100132202AF3D16846FFF7AAFFAB
:10506000002009B05DF804FB002810B511DD0C68C4
:10507000E3070ED56410532C0BD8074B1B780BB9E4
:10508000FFF76CFEFFF7CCFD044BC3F80845FFF7B4
:10509000ADFD002010BD00BF756F01200010004065
:1050A000002810B50DDD0C68E3070AD56410FF2C4D
:1050B00007D8054B1B780BB9FFF750FE034BC3F81D
:1050C0002445002010BD00BF756F01200010004076
:1050D000002813B515DD0C68E10712D564100A4AE3
:1050E0000A4B072CCDE900230BD8094B1B780BB9D1
:1050F000FFF734FE02AB1C44064B14F9082CC3F82E
:105100000C25002002B010BDE2ECF0F4F8FC000425
:10511000756F01200010004070B5002888B020DDB8
:10512000086810F001041CD104281AD9036803F0A0
:105130000F03042B15D1FEF7BBFA064605F058F90C
:10514000122828BF1220054600F10D0202216846F0
:10515000FFF7A6FD8DF80D50A54205DC6846FFF768
:1051600029FF002008B070BD0DEB0403325D9A7377
:105170000134F1E72DE9F041012888B00D4630DD1A
:10518000086810F001042CD104282AD9036803F020
:105190000F03042B25D14B68DB0722D5FEF788FAD5
:1051A000804605F025F96D680E2828BF0E206E1088
:1051B000074600F1110201216846FFF771FD6B12ED
:1051C0008DF80D606D14360E8DF80E308DF80F5081
:1051D0008DF810608DF81170A74206DC6846FFF765
:1051E000E9FE002008B0BDE8F0810DEB040318F8DB
:1051F00004209A740134EFE730B5002889B016DD39
:105200000C68E30713D56510684610220021FFF7EC
:1052100047FD63128DF80D5064142D0E68468DF80D
:105220000E308DF80F408DF81050FFF7C3FE0020B0
:1052300009B030BD174BD3F8002122B10022C3F8CA
:10524000002101229A60D3F80C2102B30021C3F897
:105250000C11D3F80024012A0F4A19D1D3F848358C
:105260005B4213600D4A1378032B9CBF013313700C
:105270000B4A1378013303F003031370094A02EB5E
:105280004313044AC2F80435024B01229A60704766
:105290001160F9E700100040240000200070012098
:1052A000746F0120766F0120024A0348102100F03C
:1052B0008BB800BFACBE0000A3BE0000044A054985
:1052C0001368C8540133C3F309031360704700BF68
:1052D000307401203070012070B51149114A0B68FB
:1052E000834202DC00230B6017E0855CA5F1FA061F
:1052F000012E00F1010405D89C420FDAA55C013DA6
:105300001F2D01D92046EBE70446151A165D2E55D0
:105310000134A342FADC181A086070BD1570FAE770
:105320003C7801203C74012008B5FDF7D5FE074B01
:105330001A68824284BF00221A601B68C01A44F6B1
:105340002063984294BF0020012008BD2C700120EA
:1053500070B5094C094D0A4E23682A68934200D162
:1053600070BDF05CFEF72CF90028F9D023680133FA
:10537000C3F309032360EFE7347401203074012084
:105380003070012070B5074E074D044633682A6817
:105390009B1ADB43C3F30903A34200DB70BDFFF795
:1053A000D7FFF3E7307401203474012010B5FFF704
:1053B00095FA044608B9204610BD83781D2B08BF16
:1053C0000446FFF78BF9F5E7F0B5074D2B680B2B7B
:1053D00008DC064F0C245C433E19C6E90112013378
:1053E00038512B60F0BD00BF38740120688D01205A
:1053F00008B5FBF7D1FEFFF7F3F8FBF7F1FEFEF778
:1054000071F8FEF72DFDFEF767FDFFF74DFF01F088
:1054100017F801F02DFABDE8084001F061BC00006A
:1054200008B54FF416620021034804F041FC034B19
:1054300000221A6008BD00BF707A0120A00500207C
:10544000064B074A1B6812689B1ADB43C3F3090328
:105450008342D4BF00200120704700BF3074012078
:1054600034740120F8B507460E4614461D4673B93C
:105470000320FFF7E5FF10B3FA20FFF71FFFF8B294
:10548000FFF71CFFF0B2BDE8F840FFF717BF501D53
:10549000FFF7D6FF98B1FB20FFF710FFF8B2FFF738
:1054A0000DFFF0B2FFF70AFFE0B2FFF707FFC4F30A
:1054B0000720FFF703FF2E46731B9C4200DCF8BD5C
:1054C00016F8010BFFF7FAFEF6E70000F8B50C4EF0
:1054D0000C4D0024F0273368A34203DCBDE8F840FC
:1054E000FFF79EBF07FB04F359195B5D2BB1002347
:1054F0001A4649781120FFF7B5FF0134EBE700BFEA
:10550000A0050020707A0120F8B50E4C0E4E07461B
:105510000025BC4205F1010511D0237853B10023C9
:105520001A4661781120FFF79DFFF02200212046E6
:1055300004F0BEFB0A2D04F1F004EAD1F8BD356099
:10554000F8E700BF707A0120A00500202DE9F04F98
:1055500012F00106ADF54F7D82468B4617D0012330
:105560008DF8143042FA03F354128DF815305214AA
:105570001B0E8DF817208DF818308DF8164005ABEE
:105580000522FFF76FFF0DF54F7DBDE8F08F042A70
:105590002CD9116801F00F03042B38D105AD02237B
:1055A00010462B70FEF784F8044604F021FFB0F596
:1055B000487F034604F1FF31A8BF4FF448739E4271
:1055C00006F101020DD1B0F5487F06D96D4B19885F
:1055D0009B78ADF832138DF834332B46594650463C
:1055E000CFE7164611F8012FAA55E8E740F0C6802C
:1055F000A2F1040CDCF100024FF0030342EB0C02B9
:105600008DF814308DF8152005AB0222E6E7092B42
:1056100040F09180154604238DF8143055F8043F6E
:105620004FEA6308B8F1200F8DF815804FEA632325
:10563000A8BF4FF020088DF816308DF8178006AC03
:1056400003220521B04502DC05ABE21AC6E755F896
:10565000040F10F0010706D1042847D9036803F0AE
:105660000F03022B0DD14FF0010323704310637021
:1056700047121B0E4014A770E070237105340136E9
:10568000E0E7042B30D123464FF0020C03F802CBA5
:10569000CDE9012100930393FEF70AF8814604F057
:1056A000A7FE0C28DDE901210AD8009B6070874223
:1056B00001D1DC19E3E719F80740DC550137F6E7BB
:1056C00023460C2003F8010F09F1FF3009F1080906
:1056D00010F8017F03F8017F4845F9D12E23E372CA
:1056E000237363730E34CAE7012B08D12346071FC7
:1056F00003F8022B7842784160701C46BFE7092B03
:1057000009D1042323704368581060705B12A370A2
:10571000E7700434B3E7032B0AD121700368C3F3A5
:105720000F10C3F34173C3EB800363701B12EEE7EA
:1057300027700134A3E7032B7FF425AF05238DF8F1
:105740001430C1F30F13C1F34171C1EB830164291C
:105750004FEA21238DF81510A8BF64218DF816306B
:105760008DF8171003328E4205AB01DB0A1D35E7B9
:10577000334412F8010F18710136F4E7002A7FF460
:1057800002AF35E770B300000F4970B5F022002476
:1057900002FB04135D78854203D001340A2CF7D153
:1057A00070BDF0221846002104F082FA074A1368FF
:1057B000013BA34200D11460002329461A46112060
:1057C000BDE87040FFF74EBE707A0120A0050020B2
:1057D00030B5B3B032AC0223054604F8C83D04F03E
:1057E00007FEC72828BFC720691E0023984207DC90
:1057F000421C2346FE211420FFF734FE33B030BD97
:10580000013311F8012FE254F0E770B5B2B032ACB9
:105810000223054604F8C83D04F0EAFDC72828BF66
:10582000C72006460023681E9E420BDC06F13200AC
:10583000FFF7A8FD2346721CFF211420FFF712FE7C
:1058400032B070BD013310F8012FE254ECE70000D4
:105850002DE9F04F0128B9B08146884603DC1B20B2
:10586000FBF7FCFD58E00868C2072BD4042829D9AF
:10587000036803F00F03042B24D1FDF719FF05463D
:10588000D8F80400C3071FD404281DD9036803F007
:105890000F03042B18D1FDF70BFF0646214BDFF851
:1058A00090A01B6803930027039BBB420EDC00966D
:1058B0002B461D4AC82106A804F020FD06A8FFF7C4
:1058C000A4FFCCE7194DDBE7184EE7E70C2303FBF9
:1058D00007F202EB0A03294652F80A00049304F087
:1058E0007DFD049B044618B9D3E9013B9C4201DBD2
:1058F0000137D9E70BEBC40231465BF8340005935E
:10590000049204F06BFDDDE9042340B9536808F10B
:105910000801A9F10200984739B0BDE8F08F0134C1
:10592000E4E700BF3874012008C00000FFB70000A2
:10593000688D01202DE9F0411F4F204AD7F80080E3
:1059400005460023F02098450EDC0024F02000FBE3
:1059500004F15318565C8EB101340A2CF7D1184863
:10596000BDE8F041FFF751BF00FB03F15418647824
:10597000AC4201D1515CE9B90133E4E7F022314690
:10598000184604F095F90F49457051F835108570A7
:105990000222A0450270C0E90212C0E9046601DCDF
:1059A00001343C60002329461A461020BDE8F0412E
:1059B000FFF758BDBDE8F081A0050020707A0120F6
:1059C00051C40000D083012070B5FFF77FFD094E60
:1059D000FF246FF0070505FB046393F8FC37043BD5
:1059E000012B03D8E043C0B2FFF7A4FF013CF2D182
:1059F00070BD00BFD08301202DE9F8431D4E07463E
:105A00000D460024B046E3009A191279062A01D007
:105A1000032A23D158F80300836803F07F031C2B6B
:105A20001CD1C36803F07F02042A17D1026902F077
:105A30007F02192A12D11B0A00EB83001030FDF7F8
:105A400037FE0378814633B104F0D2FCA84205D179
:105A500000239D4207DCE0B2FFF76CFF0134FF2C0E
:105A6000D1D1BDE8F88319F80310FA5C9142F5D161
:105A70000133EEE7D0830120F8B5094F0546FF2436
:105A80006FF0070606FB047393F8FC37AB4203D1B3
:105A9000E043C0B2FFF74EFF013CF3D1F8BD00BFB9
:105AA000D08301202DE9F84FFDF716FB584B1A68FB
:105AB000824284BF00221A601A6842F20F71821A71
:105AC0008A420BD95349186000235A181279073AB1
:105AD000022A0FD90833B3F5FF6FF6D1BDE8F88F6E
:105AE0000720FFF7C9FF8AF800802EE00820FFF7A3
:105AF000C3FF3FE0FDF7F8FA002814BF0446012475
:105B00000020FDF7D9FB81460020FDF7E9FB424D5F
:105B1000424E0746B9F1000F17D02B68002B70D109
:105B200033682C60002B6FD0DFF8F8B0DFF8F0A0FE
:105B30009BF800304FF00108002BD1D10920FFF76E
:105B40009BFF8AF800808BF80080AFB133689BB967
:105B50002B6834601BB3DFF8C8B0DFF8C8A09BF82F
:105B600000304FF00108002BC0D10920FFF784FF5F
:105B70008BF800808AF800802B6883B1284A11785E
:105B8000904661B99C4238BF2C602B68E31A312BD8
:105B900005D90720FFF770FF012388F8003032682D
:105BA00082B1204B1978984661B9A24288BF34600F
:105BB0003368E41A312C05D90820FFF75DFF012373
:105BC00088F800302B685BB1B9F1000F08D1144C94
:105BD000227812B90720FFF74FFF00232B602370B4
:105BE0003368002B3FF47AAF002F7FF477AF0D4C72
:105BF000227812B90820FFF73FFF0023336023709B
:105C00006CE7002FA2D1B9E7002FA1D1B4E700BF04
:105C100028700120D08301201870012020700120FD
:105C20001C7001202470012037B50546FFF74EFC9B
:105C300002A8002440F8044DFDF726FB214620462B
:105C4000FEF7B2F9FEF72CFCFDF75EFBFDF726FC34
:105C5000FDF740FCFEF7C0FCFDF764FA25B1FDF747
:105C6000D7FC0248FFF7D1FD03B030BD42C40000AD
:105C7000002301461A461120FFF7F4BB07B51312A3
:105C80008DF801208DF802301314120E8DF80010DB
:105C90008DF803308DF8042001466B460522132051
:105CA000FFF7E0FB03B05DF804FB0A460146122053
:105CB000FFF74CBC70B505460C46FDF71DFA58B110
:105CC00004F13200FFF75EFB2B46224600211B2029
:105CD000BDE87040FFF7C6BB70BD10B41446034664
:105CE0000A46142021465DF8044BFFF7BBBB0000B9
:105CF00030B5084C01444FF0FF33884201D3D843FC
:105D000030BD10F8015BDAB26A4054F8222082EA12
:105D10001323F2E724C00000FE2837B5044614D848
:105D20000B4B53F8300080B1416808308900FFF711
:105D3000DFFF02AD45F8040D0920FFF723FB2B46DA
:105D4000042221461720FFF78DFB03B030BD00BFB2
:105D5000D0830120F8B50746FFF728FB4FF0FF3549
:105D600004460CB92846F8BD2668C6F30743152B30
:105D70000CD104F10801384604F030FB08B9C6F331
:105D800007252046FEF7AAFC0446EAE71D2B08BFBC
:105D90004FF0FF35F5E700002DE9F047BF4CC04D4F
:105DA0009CB0FFF7D5FA2068C0F580612844FDF764
:105DB000EFFB23680344064623607BB1B94F002EF6
:105DC0000FDC2B78FA2B40F030812368022B16DC95
:105DD000FFF7AAFA10B10120FFF77EFA1CB0BDE868
:105DE000F0872068C0F580612844FDF7D1FB236867
:105DF000034406462360FDF76FF93860DFE76878F3
:105E0000AC78831E182B00F20681DFE813F019002E
:105E10002D00310035003800410004014B008000A6
:105E20008A008E00A400E000F100040104010401D6
:105E30000401040104010401040104010401FF0040
:105E4000FF2C0FD02046FFF79FFC974A002342F813
:105E5000343002EBC40221461371132000931A461A
:105E6000FEF722FE0320B7E72046FFF763FDF9E7C0
:105E70002046FFF789FCF5E7FFF7A6FDF2E7FFF7FD
:105E800025FB0020FFF7D0FE8848FFF7BEFCE9E7BE
:105E9000632CE7D8864B214653F824201520FFF7C2
:105EA00055FBDFE7FFF782FA6FF007080446002C86
:105EB000D8D02768C7F30743152B04D02046FEF738
:105EC0000DFC0446F3E704F10806304604F090FAAE
:105ED00005460530FFF756FAFB20FFF7EFF91D20C6
:105EE000FFF7ECF9C7F30720FFF7E8F9E8B2FFF78F
:105EF000E5F9C5F30720FFF7E1F9A8EB0407F3196B
:105F00009D42DBDD16F8010BFFF7D8F9F7E7002318
:105F100000931A4619461D20FEF7C6FDFDF778FBD3
:105F2000A0E72046FFF7F8FE9CE7FDF7E7F8614A97
:105F300000906421604B03A804F0E0F9022303A859
:105F40008DF80C3004F054FA03AB02460021162001
:105F5000FFF788FA86E7544F002557F8354007EBDE
:105F6000C5035CB3D4F8048093F804A04FEA880614
:105F7000B01DFFF707FAFB20FFF7A0F9012006F19B
:105F80000109FFF79BF9E8B2FFF798F95FFA89F08A
:105F9000FFF794F9C9F30720FFF790F95046FFF790
:105FA0008DF9083404EB0609A1450BD8FFF7D0F9A9
:105FB00006EB080001F0ECFBFFF7CAF90135FF2DF5
:105FC000CBD14FE714F8010BFFF778F9ECE7002489
:105FD000FFF77CFA2246214600942346DA20FEF79A
:105FE00063FD4FF4FF6221462F4803F061FE95E701
:105FF000012C02D1FEF79AFB34E7022C02D1FEF706
:1060000051FD2FE70120FFF70FFE2BE700231A4673
:1060100021461A209CE7A0F1C803052B3FF622AFCA
:1060200000221146FBF7E6F81CE7FB2B7FF4D3AE0A
:106030002268042A7FF7CCAEB5F8037040F2F6333D
:106040009F423FF7C8AE3B1D9A427FF7C1AEEB5C63
:10605000FE2B7FF4C0AE6878AC781B2807F1FF36C2
:106060007AD02DD807285ED0082837D001282CD127
:10607000FF2C11D02046FFF787FB6D790F4B009363
:106080002146BB1E2A460A20FEF70EFD064B43F8AA
:10609000340003EBC4042571781D9DE63C78012093
:1060A0003C7401202C700120D083012024C4000006
:1060B000C88B01203BC4000036C40000427401209C
:1060C0001D285BD04DD31E2870D0A0F1C803052B2E
:1060D000E2D83F4A3146FBF78DF8DDE7632CDBD889
:1060E0006B79022B0CD0032B14D0012BD4D1D5F813
:1060F0000630384A5B0043F0010342F82430CBE716
:10610000002EC9DDB91E3448FDF7EFFC314B43F8D2
:106110002400C1E7AB79002B2E4B0CBF00220422D8
:1061200043F82420B8E7632EB6DC3246284903A89A
:1061300003F09AFD1CAB1E4403A8002306F8643C40
:10614000FFF708FE0028A7DB224B214653F820204A
:106150001520FFF7FBF99FE731461D48FFF74CFC80
:106160009AE7FF2C98D06A79022A95D81A4B0093A7
:106170002146BB1E0B20FEF797FC8DE7632EA8BFC0
:106180006326002303A9B3420BDB1CAA26EAE673AD
:106190001344002203F8642C15200091731C21463F
:1061A000E9E7EA185279CA540133ECE7012C7FF48D
:1061B00073AF002E7FF770AF6B791BB1322BA8BF86
:1061C00032231C4664235C43044B1C6064E700BF1D
:1061D00041740120C88B012042740120040000207A
:1061E000084B01221A60084A1368002BFCD0074BA9
:1061F0001868042390FBF3F00638400040F00100DB
:10620000704700BF00C0004000C1004008C500400A
:106210000120704710B5064C204600F08DFE054960
:10622000204600F0EFFE044B01221A6010BD00BFB3
:1062300078780120801A06004078012010B5064CBD
:10624000204600F079FE0549204600F0DBFE044BB5
:1062500001221A6010BD00BF34790120801A0600A7
:106260004478012010B501210D20FCF74DFF094CA9
:1062700001210E20FCF748FF00210F20FCF744FF0E
:10628000204600F09BFD20461021BDE8104000F0A4
:10629000ABBD00BF587801202DE9F8430C68E30737
:1062A00004D40D20BDE8F843FBF7D8B864102FD410
:1062B000FCF728FFA0422BDB00212046FCF724FF3F
:1062C0004FF4FA620121204601F09AFA00B3DFF898
:1062D0006C8000254FF00109002707264FF47A72E1
:1062E0000121204601F08CFA90B12828C4BF09FA98
:1062F00006F31F4316F1FF36F0D205F8087001359A
:10630000052DE9D1012206210920FDF76DFB08B911
:1063100000200FE003460B2243F8042F064900F14A
:10632000180411F8012F520042F0010243F8042F23
:106330009C42F6D1BDE8F8834778012048780120D7
:1063400010B50468E30704D40D20BDE81040FBF746
:1063500085B86410FF2C01D91720F6E7FFF782FFFC
:10636000E1B2024800F063FD002010BD5878012022
:1063700008B5FFF777FF0021034800F058FD400003
:1063800040F0010008BD00BF58780120274A82B0C4
:1063900001210023ADF80630C2F8F015C2F800154F
:1063A00019461A0102F1804202F5E0420133082B3E
:1063B000C2F81415C2F81015F3D11C4B4FF4E0626B
:1063C000C3F818250422C3F81425C3F810250DF1CD
:1063D0000602C3F82C260122C3F830261A60D3F82F
:1063E0000021002AFBD00022C3F8002101225A60BC
:1063F0000E4B1A46D3F804110029FBD00021C3F834
:10640000041101219960D2F81431002BFBD0002037
:10641000C2F81401C2F80005BDF806301BB2834271
:10642000C8BFA3F50B70400002B070470070004079
:1064300008B5FFF7ABFF400040F0010008BD0000C9
:10644000024A03480A21FEF7BFBF00BF68C400002C
:10645000B8C4000070B50668F10705D54568EA07BD
:1064600002D58468E30704D40D20BDE87040FAF734
:10647000F5BF7610802E01D91520F6E76D10FF2D9F
:1064800001D91620F1E76410FF2C01D91720ECE7A1
:106490000A4B1B680BB9FFF7BDFEF1B2084800F0CC
:1064A0002FFEE9B2064800F00FFDE1B2044800F00B
:1064B0000BFD034800F08FFE002070BD40780120E6
:1064C000787801200C4B1B6870B506460D461446C3
:1064D0000BB9FFF7B3FEF1B2084800F011FEE9B2C4
:1064E000064800F0F1FCE1B2044800F0EDFC03487E
:1064F000BDE8704000F06FBE44780120347901207F
:106500000128F8B536DD0D68EA0733D51A4B4C681B
:106510001B686D100BB9FFF77DFEE9B2174800F05C
:10652000EFFD14F001050DD0C4F34701134800F04E
:10653000CBFC124800F04FFE18B12320FAF78EFF73
:106540000020F8BD042CF4D9236803F00F03092BB5
:10655000EFD154F8046F094F7610AE42E9DD54F8DC
:10656000041FCB0704D5C1F34701384600F0ACFC4B
:106570000135F2E70120E4E7407801207878012036
:1065800038B50468E20702D54568EB0704D40D204E
:10659000BDE83840FAF762BF6410802C01D915209D
:1065A000F6E76D10FF2D01D91620F1E7124B1B689D
:1065B0000BB9FFF72FFEE4B22146104800F0A0FD12
:1065C000E9B20E4800F080FC00210C4800F0A2FD6A
:1065D00020B14042400040F0010038BD0122214678
:1065E000064800F08AFD054800F065FC0028F1D05F
:1065F000024800F063FCEDE7407801207878012044
:1066000038B5124B1B6804460D460BB9FFF716FE52
:10661000E4B221460E4800F073FDE9B20C4800F0E8
:1066200053FC0B4800F0D7FD08B1404238BD0122B1
:106630002146074800F061FD054800F03CFC0028B9
:10664000F4D00348BDE8384000F038BC447801205D
:1066500034790120F8B5354E354D376804466FB9A9
:106660000D211D20FFF7CCFF5A2816D101222A70D8
:106670002A211D20FFF726FF0123336095F9003002
:10668000022B29D0032B44D0012B45D121461D20BC
:10669000FFF7B6FF4FF0FF3424E00F211920FFF77A
:1066A000AFFF332805D102232B705F222021192050
:1066B000E0E70D211E20FFF7A3FFC7280AD103231F
:1066C0003A462A211E202B70FFF7FCFE1B222A21AE
:1066D0001E20CFE72F70CFE7012C13D129211920DD
:1066E000FFF78EFF7F28C8BFA0F580706FF07E0394
:1066F0009842B8BF1846C82358437F2390FBF3F055
:106700006043F8BD032C0BD12B211920C0E72D21AC
:10671000FBE721461E20BBE74FF0FF340020EAE7ED
:10672000052CF4D04FF0FF340020DFE75078012033
:106730002C00002008B50120FFF78CFF400040F03E
:10674000010008BD08B50320FFF784FF400040F0BA
:10675000010008BD08B50520FFF77CFF400040F0B0
:10676000010008BD38B5104B1B6813B90120FFF7B5
:1067700071FF0120FFF76EFF04460320FFF76AFF59
:1067800005460520FFF766FF6D4304FB045400FB3C
:10679000004002F0B9FE01F035FB03F0CFF94000F4
:1067A00040F0010038BD00BF507801200128F8B545
:1067B00035DD0F68FB0732D54D6815F001062ED187
:1067C000042D2CD92B6803F00F03092B27D16C68FB
:1067D000144B64101B68202CA8BF20240BB9FFF7B2
:1067E00019FDC7F3470122460F480F4F00F085FC03
:1067F0000435A64211DA0C4800F05DFB18B97000B0
:1068000040F00100F8BD384600F058FB400040F071
:10681000010045F8040F0136EBE76000F0E70120C6
:10682000F0E700BF40780120787801200020704711
:1068300001207047002070470020704700207047FB
:1068400001207047002070470020704700207047EB
:1068500000207047002070470020704700207047DC
:106860000020704700207047704770477047000055
:10687000024A03480F21FEF7A7BD00BF1CC5000058
:1068800094C500000246104601320378013B1F2BDD
:10689000F9D9704708B5FFF7F5FF0378002B39D019
:1068A000222B00F1010011D1037823B1222B00F13A
:1068B000010204D11046BDE80840FFF7E3BF5C2B9E
:1068C00002D1437803B1821C1046EDE73A2BF2D097
:1068D0002C2BF0D07B2B0BD1FFF7D4FF0378002BB0
:1068E000E9D07D2B01D10130E5E7FFF7D3FFF5E7D4
:1068F0005B2B10D00246104612F8013B002BDAD079
:10690000202BD8DD2C2B05D003F0DF015D2901D031
:10691000222BF0D108BDFFF7B5FF0378002BCAD0BA
:106920005D2BE0D0FFF7B6FFF7E708B5F0B1FFF752
:10693000A9FF0378222B1AD07B2B1AD05B2B1AD0FD
:10694000A3F13002092A05D92D2B05D14278303A1E
:10695000092A07D8032009E0742B0ED0662B0ED02D
:106960006E2B0ED0181C18BF0120404208BD042019
:10697000FCE70220FAE70120F8E70520F6E7062009
:10698000F4E70720F2E738B5FFF77CFF03782D2BFB
:1069900011D101304FF0FF34431E00210A2501E0E0
:1069A00005FB012113F8012F303AD0B20928F7D99D
:1069B00004FB01F038BD0124EEE710B51446FFF7E3
:1069C00061FF0378222B02D000230B7010BD621EE2
:1069D00001300378222BF7D0002BF5D05C2B07D0A9
:1069E000441C002AF0DD01F8013B013A2046F0E7A3
:1069F0004378622B00F1020409D0662B09D06E2B7C
:106A000009D0722B09D0742B08BF0923E9E70823AA
:106A1000E7E70C23E5E70A23E3E70D23E1E710B5F9
:106A20000446FFF737FF0346A342184604D902780D
:106A3000202A03F1FF33F7D910BD08B590B10378D0
:106A400083B1FFF71FFF037803F0DF035D2B09D04D
:106A5000FFF720FF03782C2B08BF0130BDE808406A
:106A6000FFF710BF002008BD38B50D1E0DDD0378FF
:106A70005B2B0AD10130FFF705FF0124A54205D0A9
:106A8000FFF7DBFF10B10134F8E7002038BD38B55F
:106A9000154609B100230B70F8B10378E3B1FFF795
:106AA000F1FE03782C2B044603D10130FFF7EAFEF8
:106AB000044623787D2B0FD019B12A462046FFF7D4
:106AC0007CFF2046FFF7E6FE03783A2B05D1013024
:106AD000BDE83840FFF7D6BE002038BD2DE9F041B3
:106AE0000D469AB004462F789FB32E21284603F016
:106AF00068FC804690B1461B303F092F13D82846CA
:106B0000FFF741FF01462046FFF7AEFF044604B3FE
:106B1000B8F1000F1DD001363544E4E7284603F0F4
:106B200067FC0646E8E723787B2B11D1601C6422C2
:106B300001A9FFF7ACFF044658B13246294601A827
:106B400003F05EFC0028E2D02046FFF7A3FEEEE74C
:106B5000002420461AB0BDE8F08138B50D1E044669
:106B60001CDDFFF7E2FE012807D1601C012D00D1DA
:106B700038BDFFF762FF013DF8E702280ED1002281
:106B80001146601CFFF783FF012DF1D0FFF755FF81
:106B900000221146FFF77BFF013DF5E70020E7E704
:106BA000F8B50C1E074615461E4613DDFFF7BDFE61
:106BB00002280FD132462946781CFFF768FF012CC6
:106BC00000D1F8BDFFF739FF32462946FFF75FFFD6
:106BD000013CF4E70020F4E710B50446C8B1FFF724
:106BE00051FE03787B2B0AD101300024002211468C
:106BF000FFF74DFF68B1FFF74DFE0134F6E75B2B61
:106C000006D101300024FFF718FF10B10134FAE774
:106C10000024204610BD002870B514DD0D68EB0778
:106C200011D56D10013DFDF759FE00264FF0FF34E0
:106C300060B916B3304603F0DBFB01463046BDE8D1
:106C40007040FCF752BF4FF0FF35ECE70368C3F329
:106C50000742152A0BD1C3F307239C42B8BF1C4639
:106C60009D4201D100F10806FDF738FDE0E71D2A3D
:106C700004BF00264FF0FF34F6E7601C400040F0F0
:106C8000010070BD10B508680C46FCF711FDFFF758
:106C900061F80028A2BF034B626843F8202000205F
:106CA00010BD00BFC88B012008B50868FCF700FDC7
:106CB000FFF750F80028AABF024B012053F820002C
:106CC00008BD00BFC88B012008B50868FCF7F0FCC0
:106CD000FFF740F80028ACBF0420002008BD0000EA
:106CE000024A03480421FEF76FBB00BF30C6000014
:106CF0002AC6000008B5FCF7FFFBFCF7ADFCFEF769
:106D000077FB0448FEF781FDFDF728FFBDE808404A
:106D1000FEF75ABE7FC60000FCF7BCB838B50025A8
:106D2000057329B90B4B0C4A0C48252102F02EFFA4
:106D300001600B4951F82220027151F82330837110
:106D40009DF8103051F8233043710223C3718560E0
:106D500038BD00BF97C60000F6C60000A5C60000FB
:106D600054C70000037B23B943738373036101237A
:106D70000373704784B00DF1100C0CE90E009DF800
:106D80000810026800230129C2F80035039B12D0C5
:106D90000BD303290CD0C2F85435019BC2F824351B
:106DA0000123C2F8003504B0704743F00203F2E754
:106DB00043F00403EFE743F00603ECE710B5FFF7F9
:106DC000D1FF03688279C3F808254279C3F80C25FE
:106DD0000279C3F81025034BBDE810400ECBFFF736
:106DE000C9BF00BF6C7801200A0611D43F2912D810
:106DF0001F2913D80F2914D8072915D803298CBFA8
:106E00004FF080434FF000430268C2F824357047CA
:106E10004FF00073F8E74FF08063F5E74FF0006341
:106E2000F2E74FF08053EFE74FF00053ECE70368D1
:106E3000C3F81C15D3F80821002AFBD0D3F8180595
:106E40000022C3F80821C0B27047000007B5094B03
:106E500009490A484FF080421A6000229A600222D3
:106E60001A710F2300930E220D23FFF757FF03B073
:106E70005DF804FB6C780120003002405878012056
:106E80002DE9F84380460D46174601EB02090C46F2
:106E90004C45A4EB05060BD0D8F8003014F8011BC4
:106EA0001B68404698470028F2D13046BDE8F88379
:106EB0003E46FAE77047203000F03CBA203000F040
:106EC0002BBA203000F03CBA38B5437F0D460BB9E1
:106ED000002038BD00F16804204600F039FA00288F
:106EE000F6D12046294600F008FA0120F1E700001B
:106EF0002DE9F0411E4600254FF47A73C0E9015395
:106F00000C4B044640F8203B8846174600F0ECF94D
:106F100004F1680000F0E8F99DF8183063769DF8F8
:106F20001C302676C4E90487A37665772046BDE841
:106F3000F08100BF3CC70000F0B5837E2E4C2F4D82
:106F40000121C17654F82320437E54F8233012F0F7
:106F5000200F14BF2F464FF0A04702F01F0213F07E
:106F6000200F03F01F0308BF4FF0A04502F5E072A9
:106F700003F5E07340F20C6647F8226045F82360A1
:106F800003694FF0CC72C3F8242503690622C3F8C5
:106F90000025827E036954F82220C3F80825427E2A
:106FA000036954F82220C3F80C2590F91830144ACC
:106FB0005C0903F01F03994004F1600342F82310B9
:106FC00090F91830002BBDBF03F00F0302F6FC321E
:106FD000D2189B18B5BF40234022137683F80023B4
:106FE00090F918300122590903F01F0302FA03F344
:106FF000034A42F82130F0BD54C70000000300509E
:1070000000E100E0C37EA3B103690022C3F80025BC
:107010000A4B99420ED90A4B994294BF4FF08061B6
:107020004FF0C8610369C3F8241503690622C3F849
:10703000002570474FF0CC71F4E700BFA086010037
:1070400090D003002DE9F041044688461F461546BE
:10705000002A50D000F12006304600F059F923698B
:10706000C3F88885236901221A622369C3F834654D
:107070002369C3F8385523691A602269D2F84C3164
:107080001BB9D2F82431002BF8D00023C2F84C31C0
:107090002269D2F85C311BB9D2F82431002BF8D028
:1070A0000023C2F85C3122696FB9D2F8243153B998
:1070B0000123D3612369D3F84821002AFBD00022A1
:1070C000C3F8482109E0012353612369D3F804215F
:1070D000002AFBD00022C3F804212369D3F824211D
:1070E00012B10022C3F824212369D3F83C0520669D
:1070F000C0B2BDE8F0811046FBE70123FFF7A2BF55
:1071000010B5044680F8B010683000F001F9012392
:10711000637710BDF8B500234377036990F8B0207A
:10712000C3F88825036901261E62036900F168051A
:107130000446C3F8445528460F4600F0FBF823697F
:10714000C3F8480523699E602369D3F850211AB912
:10715000D3F82421002AF8D00022C3F85021284671
:1071600000F0E8F8236930B1D3F860211AB9D3F8F8
:107170002421002AF8D00022C3F8602123696FB9C6
:10718000D3F8242152B90122DA612369D3F84821C6
:10719000002AFBD00022C3F8482109E001225A61ED
:1071A0002369D3F80421002AFBD00022C3F804216C
:1071B0002369D3F8240168B10022C3F8242123698C
:1071C000D3F8C404C3F8C404022803D004280CBFB5
:1071D00003200420F8BD0121FFF79CBF70B543696F
:1071E000D3F86421044692B10022012500F1200663
:1071F000C3F864210577304600F08AF86369C3F864
:10720000346563694022C3F8382563691D63636987
:10721000D3F86821DAB10025C3F8685104F1680693
:10722000012363772577304600F072F8D4F8B43044
:1072300003B19847636965773046C3F8446500F049
:1072400079F86369C3F84805636901225A63636981
:10725000D3F8042162B10022C3F80421237F3BB19B
:107260006369D3F83C05D4F8B830206603B1984779
:107270006369D3F8242152B10022C3F82421636941
:10728000D3F8D024C3F8D024636901225A6170BDB9
:107290000148FFF7A3BF00BF787801200148FFF73E
:1072A0009DBF00BF3479012007B514231322CDE917
:1072B00000324FF04022114604230848FFF718FE21
:1072C000074A08481E231F21CDE900310323114638
:1072D000FFF70EFE03B05DF804FB00BF78780120D5
:1072E000003000403479012008B54022002102F02E
:1072F000DFFC0022C0E9102208BD026C10B5531C4F
:10730000446C03F03F039C421CBF8154036410BDD6
:107310000023C0E910337047D0E9102393421FBF08
:10732000C25C013303F03F03436414BF10464FF0C7
:10733000FF307047D0E91030181A48BF403070470E
:10734000D0E91023934214BFC05C4FF0FF30704768
:10735000036C406C013303F03F031B1A5842584141
:10736000704700000649074A074B9B1A03DD043BA0
:10737000C858D050FBDC00F013F8F8F761FF0000AC
:10738000F8CB00000000002038020020FEE7FEE7F6
:10739000FEE7FEE7FEE7FEE7FEE7FEE7FEE7FEE7C5
:1073A000394B1A680D2A08D14FF080420021C2F8EB
:1073B0000C11C2F81011C2F838151B680D2B46D1FC
:1073C0004FF08052314BD2F80414C3F82015D2F894
:1073D0000814C3F82415D2F80C14C3F82815D2F8F1
:1073E0001014C3F82C15D2F81414C3F83015D2F8C1
:1073F0001814C3F83415D2F81C14C3F84015D2F889
:107400002014C3F84415D2F82414C3F84815D2F850
:107410002814C3F84C15D2F82C14C3F85015D2F820
:107420003014C3F85415D2F83414C3F86015D2F8E8
:107430003814C3F86415D2F83C14C3F86815D2F8B0
:107440004014C3F86C15D2F84424C3F870250E4BD1
:107450001B680D2B09D14FF08043D3F80024D207CD
:1074600044BF6FF00102C3F80024094AD2F8883003
:1074700043F47003C2F88830BFF34F8FBFF36F8FB0
:10748000044B054A1A6070473001001000C00040EC
:1074900000ED00E0300000200090D0030120704794
:1074A00003681322DB69184770470369C3F81C158A
:1074B0000369D3F81C21002AFBD00022C3F81C2149
:1074C0000120704710B490F95C30144C5909012226
:1074D000203103F01F0302FA03F344F8213003695B
:1074E0005DF8044B0421C3F8081303695A6003696B
:1074F000DA6003690022C3F8002502694FF0FF3308
:10750000C2F80C350269C2F814350269C2F80835B0
:1075100002691430C2F81035FFF7FABE00E100E04E
:107520001430FFF707BF1430FFF70ABF1430FFF71E
:10753000F3BE0000036990F85E2010B5C3F80C2577
:10754000036990F85D20C3F8142590F86120036961
:10755000012A01BF90F85F40C3F81045036990F815
:10756000604006BFC3F8084503690022B1F5966F75
:10757000C3F86C2569D9B1F5166F69D9B1F5965F75
:1075800069D9B1F5165F68D9B1F5615F67D9B1F511
:10759000964F66D9B1F5E14F65D9B1F5164F64D96B
:1075A000B1F5614F64D9B1F5963F64D9B1F5E13FCA
:1075B00063D9B1F5613F63D9364B994263D9B1F5CF
:1075C000E12F63D9B1F5612F94BF4FF070634FF095
:1075D00080530269C2F8243503690422C3F80025E8
:1075E00001690023C1F808310169C1F81C31016942
:1075F00001230B6001698B600169C1F8042390F9D4
:107600005C20510902F01F0293406031224A42F887
:10761000213090F95C30002BBDBF03F00F0302F660
:10762000FC32D2189B18B5BF60236022137683F812
:10763000002390F95C300122590903F01F0302FA7C
:1076400003F3154A42F8213010BD4FF49E23C0E7E2
:107650004FF41D23BDE7114BBBE7114BB9E7114BAD
:10766000B7E7114BB5E7114BB3E74FF41D03B0E794
:107670004FF46B03ADE70E4BABE74FF0EB73A8E7AE
:107680004FF06C73A5E74FF08063A2E74FF0E8631B
:107690009FE700BF90D0030000E100E000B01300BE
:1076A0000050270000F03A0000A04E0000C0750016
:1076B00000903A012DE9F0411E4600254FF47A73FF
:1076C000C0E901530D4B044640F8143B1746884669
:1076D000FFF70AFE0A4AC4F8108084F85C7052F87A
:1076E000263084F85D309DF8183052F8233084F845
:1076F0005E3084F861502046BDE8F081E8C70000A4
:1077000054C7000010B50369D3F8082104464AB1F4
:10771000D3F818151430C9B2FFF7EFFD2369002222
:10772000C3F8082110BD00000148FFF7EBBF00BF00
:10773000F079012007B52223009302222123034977
:107740000348FFF7B7FF03B05DF804FB00200040DB
:10775000F079012008B102F079BD70470A4B196831
:107760000A4B30B5D3F804050C060D0A44EA0002B2
:107770004FF47A712B46A2FB014501FB0355E00B48
:1077800040EA454030BD00BF547A0120001001405E
:1077900038B5044648B1FFF7E1FF054600F01AF896
:1077A000FFF7DCFF401BA042F8D338BD074B002297
:1077B000C3F8042182B0D3F80431054A0193019B38
:1077C00013680133DBB2136002B070470010014050
:1077D000547A01207047704708B500F067F8FFF74A
:1077E000FAFF0120FFF7D4FFFFF784FA034CFFF7FD
:1077F00093FA002CFBD0AFF30080F8E70000000004
:1078000038B5174B174D53F82030174813F0200F99
:107810004FF0010403F01F0304FA03F408BF4FF014
:10782000A04000292B681149B3FBF1F300F5A260D9
:1078300002FB03F321464FF00A02B3FBF2F314BF3D
:107840002246002200F014F842F2107358434FF41D
:107850007A722B68B3FBF2F3B0FBF3F038BD00BFD4
:1078600054C70000300000200003005040420F00C9
:1078700030B504680C40944206D1013B002BF8D18E
:1078800012E0013B002B0FD004680C409442F8D169
:10789000002405680D40954204D101349C42F8D182
:1078A000002002E0201C00E0181C30BD0D4BE0223F
:1078B00083F811234FF40032C3F880211A604FF08F
:1078C00080430122C3F818259A6003F5883300210C
:1078D000C3F808150221C3F80413C3F844131A604F
:1078E000704700BF00E100E0014B1860704700BF27
:1078F0004C000020222837B50CD84B4B53F82030D1
:10790000052B00F0828007D8032B12D07BD8022BE6
:1079100000F08180002074E01D2B78D003D81C2B50
:10792000F8D1052206E01E2B73D01F2BF2D10822BE
:1079300000E002223D4B196808296EDD0A296FDD3F
:107940000D29B5BF0C240E24022303233848C0F8A8
:10795000F0350123C0F8003500200546030103F18E
:10796000804303F5E04301300828C3F81455C3F8F9
:107970001055F3D12F4B18682F4B1B6800021B03C7
:1079800003F4805300F4E0601843294BC3F8180552
:10799000C3F81425C3F810250DF10602C3F82C26F0
:1079A0000122C3F830261A60D3F80021002AFBD048
:1079B0000022C3F8002101225A601D4B1A46D3F859
:1079C00004010028FBD00020C3F8040101209860C6
:1079D000D2F81431002BFBD00023C2F81431BDF9CA
:1079E00006209A42124AB8BFADF80630A142C2F84A
:1079F0000035BDF9060004D035BF611A091BC84027
:107A0000884003B030BD032294E7042292E70622A7
:107A100090E707228EE701228CE70824002395E7F0
:107A20000A24012392E700BF54C70000440000204D
:107A30000070004048000020607A0120222830B504
:107A40003CD8224B53F82000214B00221D4653F80E
:107A50002240B4F1FF3F32D11E4C45F822006FEABC
:107A600041411D4D1D4B246853F822306FEA5141AE
:107A700025F81210012101FA04F4C3F86005013C55
:107A8000C3F8640505EB4202C3F86805C3F86C054A
:107A90000020C3F80015C3F80C05C3F80405C3F8AB
:107AA0000845C3F81405C3F81005C3F82025C3F82A
:107AB0002415C3F82815C3F82C05996030BD8442FD
:107AC000CAD00132042AC2D1F8E700BF54C700006F
:107AD000340000204C000020587A012010C800001B
:107AE000222815D8114B124A53F8203013F0200FDA
:107AF00008BF4FF0A04203F01F03032908D8DFE8B6
:107B000001F00210080C03F5E073002142F8231085
:107B1000704703F5E0730C21F8E703F5E0730421E7
:107B2000F4E703F5E0730321F0E700BF54C700005A
:107B300000030050222813D80A4B53F820000A4BA8
:107B400010F0200F4FF0010200F01F0008BF4FF0AF
:107B5000A043824011B9C3F80C257047C3F808252B
:107B6000704700BF54C7000000030050222810D8FF
:107B7000094B0A4A53F8203013F0200F08BF4FF08A
:107B8000A04203F01F03D2F81005D84000F0010016
:107B900070470020704700BF54C70000000300502A
:107BA0002DE9F04106460D4601EB02080C4644451E
:107BB000A4EB050707D0336814F8011B1B68304697
:107BC00098470028F3D13846BDE8F0812DE9F0410F
:107BD000C1F30A57A7F2FF35132D82B002460B46B8
:107BE0000C464FEAD178064633DC002D4EDB3C498B
:107BF000294103EA0100104326D049080B4052EA0C
:107C000003060CD04FF48023132D24EA010143FA1C
:107C100005F444EA01040CBF4FF000460026314948
:107C200001EBC8082346D8E90045324620462946DC
:107C300001F01EFBCDE9000122462B46DDE90001E3
:107C400001F014FB02460B461046194602B0BDE88F
:107C5000F081332D07DDB5F5806FF5D101F008FB1C
:107C600002460B46F0E7A7F213474FF0FF31F94009
:107C70000842E9D049080842D1D04FF0804320EAB9
:107C8000010143FA07F741EA0706C8E721F000417E
:107C90000143D9D0C3F3130101434E420E43114DAA
:107CA0005C0C360B640406F4002305EBC80243EABF
:107CB0000401D2E900450B4602462946204601F060
:107CC000D7FACDE9000122462B46DDE9000101F09B
:107CD000CDFA21F00041024641EAC873B4E700BF83
:107CE000FFFF0F0020C80000F8B5C1F30A57A7F244
:107CF000FF35132D02460B460C4610DC002D29DB08
:107D00008C461D4929410B422AD04FF400242C41B6
:107D1000644424EA0104002621463046F8BD332D90
:107D200005DDB5F5806F1ED010461946F8BDA7F2E7
:107D300013474FF0FF3121FA07F73842F4D00123FF
:107D4000C5F1330503FA05F5461928BFE41826EAFC
:107D50000706E1E7013501F0004407D00026DBE724
:107D60000028D2D1E0E701F083FAF8BD44F07F5457
:107D700044F440140026CFE7FFFF0F0030B51F4A40
:107D800021F00043934287B01CDD1D4A934205DD7C
:107D900002460B4601F06AFA07B030BD02AA00F0B5
:107DA0008FF800F003000128DDE9042312D0022837
:107DB0001CD0A0B1DDE9020100F066FB01F1004139
:107DC00007B030BD002300930022002301F084F8A7
:107DD00007B030BDDDE9020100F056FBDCE701240D
:107DE000DDE90201009401F077F8D5E70124DDE92F
:107DF0000201009401F070F8E0E700BFFB21E93FC9
:107E0000FFFFEF7F2DE9F04F8BB004460D4600F0E9
:107E100079FA294B93F900A0BAF1FF3F06460F46C5
:107E200012D022462B462046294601F071FE834699
:107E300050B94FF000084FF000092046294642464D
:107E40004B4601F03DFE20B9304639460BB0BDE847
:107E5000F08F0122194BCDF820B00092CDE90445F6
:107E6000CDE902450193BAF1000F17D042464B46C7
:107E70004046494601F0DCFCBAF1020FCDE90601AB
:107E80000ED101F0A1FE21230360089B73B9DDE947
:107E90000667304639460BB0BDE8F08FCDE906895C
:107EA000684601F055F90028EFD1EAE701F08CFEB1
:107EB000089B0360EBE700BF5000002030C80000C3
:107EC0002DE9F047CA4B21F000479F4290B0804611
:107ED000894640F38F80C74B9F420C46924626DC72
:107EE0000029B9A3D3E9002340F38F8001F0BEF944
:107EF000C14B9F4204460D4600F04781B4A3D3E92D
:107F0000002301F0B3F902460B46CAE900232046DC
:107F1000294601F0ABF9AEA3D3E9002301F0A6F99D
:107F20000125CAE90201284610B0BDE8F087B34B2D
:107F30009F4240F38980B24B9F4200F31C813D1564
:107F4000A5F21645A7EB055319461F46064601F054
:107F5000F5FD01F0D9FA8046894642464B46304647
:107F60003946CDE90A8901F081F90022A54B01F0DB
:107F700035FB8946804601F0E1FD01F0C5FA064671
:107F80000F4632463B4640464946CDE90C6701F074
:107F90006DF900229B4B01F021FB00220023CDE96B
:107FA0000E0101F083FD002800F0608100233046BF
:107FB0003946002201F07AFD002814BF0123022374
:107FC000914A019202212A4600910AA8514600F0E6
:107FD00083FB002C054614DADAF80420DAF80C30BA
:107FE00002F1004203F100434542CAF80420CAF8F6
:107FF0000C3006E000200021C2E90089C2E902013C
:108000000025284610B0BDE8F08701F031F97A4B21
:108010009F4204460D4600F00B816DA3D3E9002377
:1080200001F026F902460B46CAE9002329462046FC
:1080300001F01CF966A3D3E9002301F019F94FF010
:10804000FF35CAE90201DCE700F0FCFF62A3D3E9D7
:1080500000238046894601F0C1FA00226B4B01F0F3
:1080600007F901F06BFD054601F04EFA56A3D3E97E
:108070000023CDE9060101F0B1FA02460B46404665
:10808000494601F0F3F852A3D3E90023804689461C
:10809000DDE90601CDE9028901F0A0FA1F2D0246B3
:1080A0000B46CDE9042340F3B380DDE90423DDE989
:1080B000020101F0DBF8804689463F15C9F30A53F7
:1080C000FB1A102B40F3B18045A3D3E90023DDE96F
:1080D000060101F083FA8046894602460B46DDE937
:1080E000020101F0C3F802460B46DDE90201CDE9C9
:1080F000082301F0BBF842464B4601F0B7F83AA31B
:10810000D3E9002380468946DDE9060101F066FADD
:1081100042464B4601F0AAF80B46CDE9040102465F
:10812000DDE9080101F0A2F8C1F30A53FF1A312F6B
:108130008046894600F39C809DED087BCAE9008952
:108140008DED027B42464B46DDE9020101F08EF8DF
:10815000DDE9042301F08AF8002CCAE90201BFF628
:1081600050AF09F1004401F100436D42CAE90084B7
:10817000CAE9020345E702460B4601F077F80025FD
:10818000CAE90201CAE900013BE715A3D3E90023CC
:1081900001F06CF814A3D3E900230D46044601F066
:1081A00065F802460B46CAE900232946204601F03D
:1081B0005DF80DA3D3E9002301F058F80125CAE9C1
:1081C00002011EE7AFF3008000004054FB21F93F9D
:1081D0003163621A61B4D03D83C8C96D305FE43F3A
:1081E0000000601A61B4D03D7370032E8A19A33B5E
:1081F000FB21E93F7BD90240FB21F93FFB213941BB
:10820000FFFFEF7F00007041B8C800000000E03FB2
:108210004046494601F02AF8394B6A1E804653F819
:108220002230BB4289463FF448AFCAE9008989E75A
:108230002BA3D3E9002301F01BF82BA3D3E90023E0
:108240000D46044601F014F802460B46CAE9002325
:108250002946204601F00AF823A3D3E9002301F0C0
:1082600007F84FF0FF35CAE90201CAE60323A7E683
:108270001FA3D3E90023DDE9060101F0AFF90646AB
:108280000F4602460B46DDE9080100F0EFFF80468D
:10829000894602460B46DDE90801CDE9028900F076
:1082A000E5FF32463B4600F0E1FF13A3D3E900238C
:1082B00006460F46DDE9060101F090F932463B46DD
:1082C00000F0D4FF02460B4640464946CDE9042360
:1082D00000F0CCFF80468946A7E700BFAFF30080DF
:1082E0000000601A61B4D03D7370032E8A19A33B5D
:1082F0000000002E8A19A33BC14920259A837B39AF
:1083000038C800005E4A8A432DE9F04104460D4614
:1083100000F0958000290B460646844656DD0F1571
:1083200000F0A580C3F31303A7F2FF3743F48013D3
:108330004FEADC72F80702EB43034FEA4C0504D521
:10834000ED0F05EB43034FEA8C0500267F10B44682
:1083500016224FF400110CEB010098424FEAD5743D
:108360004FEA450503DC1B1A00EB010C0E44013AF1
:1083700004EB43034FEA5101EDD110469646202409
:108380004FF0004209E051D05B00013C03EBD57394
:108390004FEA52024FEA450537D0634502EB0E0122
:1083A000F1DD002901EB020E0ADBE046A3EB0C0332
:1083B000A94288BF03F1FF336D1A1044C446E3E7B6
:1083C000BEF1000FF1DB0CF10108EFE721F00042F4
:1083D000024329D0002942D10146CA0A153B49056A
:1083E000002AFAD012F4801001D044E06046520016
:1083F000D40200F1010CF9D5CCF1200401FA0CFCF7
:10840000E1401F1A41EA02038CE72B4321D14408C3
:10841000731003F17F53F20703F5001348BF44F0D4
:10842000004403EB07512046BDE8F081A942ABD8D8
:10843000002901EB020EC3DB98460023BCE702468D
:108440000B4601F0CBF822462B4600F011FFBDE8A9
:10845000F081411C16BF421C01365408D8E7024681
:1084600000F004FF02460B4601F0E2F9DCE71A4691
:1084700031463B46B6E78C4620244FF0FF30BFE73D
:108480000000F07F000000002DE9F04F21F00048CF
:10849000B8F1795F85B006460F4692469B466BDA87
:1084A00001F04CFB002800F0E18032463B463046AC
:1084B000394601F093F874A3D3E9002304460D462E
:1084C00001F08CF872A3D3E9002300F0D1FE22461C
:1084D0002B4601F083F870A3D3E9002300F0C6FE19
:1084E00022462B4601F07AF86DA3D3E9002300F071
:1084F000BFFE22462B4601F071F86BA3D3E900239F
:1085000000F0B4FE22462B4601F068F868A3D3E9D8
:10851000002300F0ADFE22462B4601F05FF8CDE9C6
:1085200000010022664B2046294601F057F8DDE99C
:108530000023804689462046294601F04FF85246DE
:1085400004460D465B463046394601F047F8024680
:108550000B462046294600F089FE02460B4640465F
:10856000494600F083FE02460B460020554900F0C4
:108570007DFE05B0BDE8F08F02460B4601F02EF8F7
:1085800041A3D3E9002304460D4601F027F840A398
:10859000D3E9002300F06CFE22462B4601F01EF8C2
:1085A0003DA3D3E9002300F061FE22462B4601F0F3
:1085B00015F83BA3D3E9002300F05AFE22462B46D0
:1085C00001F00CF838A3D3E9002300F04FFE224657
:1085D0002B4601F003F836A3D3E9002300F048FE50
:1085E0002B46224600F0FAFF374B9845CDE90001B3
:1085F00097DD364B98453EDCA8F50013002200209D
:1086000030499046994600F031FECDE90201002242
:108610002B4B2046294600F0E1FF42464B4600F036
:1086200025FEDDE90023804689462046294600F0E4
:10863000D5FF524604460D465B463046394600F0AB
:10864000CDFF02460B462046294600F00FFE0246AB
:108650000B464046494600F009FE02460B46DDE95E
:10866000020100F003FE05B0BDE8F08F15490020BF
:1086700005B0BDE8F08F9FED107B4FF000088DED49
:10868000027BDFF84C90C2E7D43888BEE9FAA8BD77
:10869000C4B1B4BD9EEE213EAD529C804F7E923E51
:1086A0009015CB19A001FA3E7751C1166CC1563F07
:1086B0004C5555555555A53F000000000000E73FBB
:1086C0000000E03F0000F03F3233D33F0000E93FBD
:1086D0000000D23F000000002DE9F04FADF5197DFC
:1086E000BE4CA29EBE4D54F826600793D41E85FB57
:1086F0000475E417C4EBA50424EAE4741D46631C66
:10870000A3EB8303013D02EBC303059373190496A6
:108710000994019503900B91A4EB05071AD43B44EF
:10872000002400255E1C0DF18008DDF88C9208E025
:1087300059F8270000F0E8FE0137B742E8E80201E7
:1087400008D0002FF4DA013720462946B742E8E87E
:108750000201F6D1049B002B079B4FEAC30302934F
:108760002ADB039A20A902EB030801EB0309049B0F
:1087700072AA02EBC30B0DF5E07A019B002B4FF0C0
:1087800000064FF0000711DB039C4D4675E90223FC
:10879000F4E8020100F022FF02460B46304639465B
:1087A00000F066FD444506460F46EFD1EAE8026751
:1087B000DA4509F10809E0D1DDE902040499204411
:1087C0008B0082460BA8A3F10802C31808930CABD8
:1087D00013440A938B4698AB03EBCB03BBF1000F1A
:1087E00053E9284529DD70AB03EBCB080DF13009C7
:1087F00000227C4B2046294600F0F0FE01F09EF955
:1088000000F082FE0022784B06460F4600F0E6FE9E
:1088100002460B462046294600F028FD01F08EF95D
:1088200078E9022349F8040B3946304600F020FD70
:1088300070AB984504460D46DAD1DDF81490204619
:1088400029464A4600F088FC00224FF07F53044638
:108850000D4600F0C3FE00F0FBFB0022634B00F06E
:10886000BDFE02460B462046294600F0FFFC0D46A1
:10887000044601F063F9804600F046FE0B460246CE
:108880002946204600F0F2FC4B46002B06460F46D8
:1088900040F3E1800BF1FF320CA9C9F1180351F844
:1088A000225045FA03F101FA03F30CA8EB1A40F841
:1088B0002230C9F11705884443FA05F5002D2CDD57
:1088C000BBF1000F08F1010840F381820C9C002CE1
:1088D00040F0A780BBF1010F0AD00CA9012251F88A
:1088E000044F531C002C40F09E809B451A46F6D145
:1088F000059B002B0EDD012B00F0D980022B09D146
:108900000BF1FF320CAB0CA953F82230C3F3150363
:1089100041F82230022D00F0AF80002200233046C3
:10892000394601F0C3F8002800F05382049B0BF194
:10893000FF394B4510DC0BF180430CAA013B089832
:1089400002EB8303002253F80419834242EA010236
:10895000F9D1002A40F0B680049B0CAA013B52F8E2
:108960002330002B40F0A1800A9A012352F8041909
:1089700001330029FAD05B440BF1010999450693B4
:108980004CDC099A079909EB020801EB0B0508F189
:10899000804802EB030BA39B08F1FF3803EB880828
:1089A00070AB03EBC909A39B20A903EB8B0301EB7D
:1089B000C505029358F8040F00F0A6FD0B46019977
:1089C0000246002905F1080BC5E900234FF0000617
:1089D0004FF000071CDB039C0CE000BF00CA000046
:1089E000ABAAAA2A0000703E00007041000020409F
:1089F00075E90223F4E8020100F0F0FD02460B469F
:108A00003046394600F034FC544506460F46EFD157
:108A1000029B9845E9E802675D46CBD1DDF818B0C6
:108A2000D9E6012300220CA9C4F180749B4541F8CA
:108A300022400EDD51F8232001EB8B0001EB830374
:108A40006FF07F4100E01A688A1A43F8042B8342D2
:108A5000F9D101244CE706D10BF1FF330CAA52F8EF
:108A60002350ED152AE700227B4B01F03DF800284A
:108A700040F0A381054650E732463B460020774947
:108A800000F0F4FB06460F46002C3FF446AF059A73
:108A90007249002000F060FB02460B463046394622
:108AA00000F0E4FB06460F4637E7012363E70BF1CE
:108AB000FF320CAB0CA953F82230C3F3160341F874
:108AC000223027E70CAB059A53F82930183ACDE944
:108AD000068505926BB909F18043013B0CA901EBB6
:108AE000830353F8041909F1FF39183A0029F8D023
:108AF0000592059A5949002000F02EFBB9F1000FAC
:108B000004460D46C0F2C0814FEAC90370AA02EBC9
:108B1000030808930CAB03EB8906DFF844B14FF070
:108B2000000A08F10807043656F8040D00F0ECFCC2
:108B300022462B4600F052FD5B4667E90201524691
:108B40002046294600F04AFD0CAB9E4204460D46E5
:108B5000EAD148AB03930193CDF8149009F10103D6
:108B6000DDF810900293C3464FF0000AB9F1000FF0
:108B7000C0F22A81DFF8EC805D4635A3D3E90023FB
:108B800000260027002403E0544510DCF8E8022307
:108B9000F5E8020100F022FD02460B463046394658
:108BA00000F066FB0134A14506460F46ECDA019B56
:108BB000E3E802670193029B0AF1010A9A45ABF1CF
:108BC000080BD3D1A29BDDF81490032B39D8DFE832
:108BD00013F0D900060006004D0048AB0393B9F12D
:108BE000000F4FF000004FF0000109DB039D05EB83
:108BF000C904083474E9022300F03AFBA542F9D114
:108C0000079B002B40F01E810B9BC3E900010B4624
:108C100003990246D1E9000100F028FBB9F1000FE9
:108C20000CDD4AAD01240134F5E8022300F020FBFD
:108C3000A145F8DA079B002B40F014810B9BC3E998
:108C40000201069B03F007000DF5197DBDE8F08FCA
:108C500000000040FB21F93F0000E03F0000F03F32
:108C60000000703EC8C9000048AB0393B9F1000F83
:108C700040F32781039ACDF810904FEAC90301937E
:108C8000D318D3E900AB09F10053013B02EBC9084B
:108C90000293914678E9026752465B463046394670
:108CA00000F0E6FA04460D4602460B4630463946C9
:108CB00000F0DCFA52465B4600F0DAFAC145A24603
:108CC000AB46C8E90201C8E90045E3D1DDF81090E0
:108CD000B9F1010F40F3F580019B039A0299134407
:108CE000C900D3E9006701F1080A019192440DF52A
:108CF000947B7AE9028932463B464046494600F079
:108D0000B7FA04460D4602460B464046494600F077
:108D1000ADFA32463B4600F0ABFAD34526462F4625
:108D2000CAE90201CAE90045E3D1019C039B103462
:108D3000002000211C4403F1100574E9022300F017
:108D400097FAA542F9D1039C079ED4E90023D4E900
:108D50000245002E00F08A8003F1004701F1004334
:108D60000B99C1E90403069B2646944605F100448D
:108D700003F00700C1E900C7C1E902640DF5197DE0
:108D8000BDE8F08F089C039D0834002000212C448E
:108D900074E9022300F06CFAA542F9D1079B13B1E4
:108DA00001F1004319460B9BC3E90001069B03F048
:108DB00007000DF5197DBDE8F08FBBF1000F08F13C
:108DC000010874DD022581E500260027EFE6002476
:108DD0008EE5CDE90685059D304639466A4200F0AC
:108DE000BBF90022384B06460F4600F07DFE00B36B
:108DF0000022364B3046394600F0F0FB00F09EFE74
:108E0000044600F081FB00222F4B00F0E7FB0B46ED
:108E100002463946304600F029FA00F08FFE0BF189
:108E200001090CAB183543F82B00059543F8294090
:108E30005FE63046394600F081FE0CABD94643F878
:108E40002B0056E60B9C01F10043C4E900030B46DE
:108E500003990246D1E9000100F008FAB9F1000FC8
:108E60003FF7DFAE01F100431946E7E60B9EC6E986
:108E70000023069BC6E9040103F00700C6E902458A
:108E80000DF5197DBDE8F08FA29B032B3FF6D9AEFF
:108E900001A252F823F000BFA98E0000DB8B000076
:108EA000DB8B0000698C00000020002176E7324651
:108EB0003B460020064900F0D9F9022506460F4638
:108EC0002BE5002000213EE7000070410000703ECD
:108ED0000000F03F000000002DE9F04F21F00046B7
:108EE000B6F1795F85B004460D469046994604DA9E
:108EF00000F024FE002800F0858022462B46204604
:108F0000294600F06BFB06460F4602460B462046FC
:108F1000294600F063FB41A3D3E9002382468B4638
:108F20003046394600F05AFB3EA3D3E9002300F057
:108F30009DF932463B4600F051FB3CA3D3E90023A8
:108F400000F096F932463B4600F048FB39A3D3E9DE
:108F5000002300F08BF932463B4600F03FFB37A37D
:108F6000D3E9002300F084F90E9BCDE900019BB307
:108F70000022294B4046494600F030FBDDE9002342
:108F8000CDE902015046594600F028FB02460B4647
:108F9000DDE9020100F06AF932463B4600F01EFBB3
:108FA00042464B4600F062F919A3D3E90023064676
:108FB0000F465046594600F011FB02460B4630461C
:108FC000394600F055F902460B462046294600F086
:108FD0004DF905B0BDE8F08F02460B4630463946E4
:108FE00000F0FCFA0AA3D3E9002300F03FF952464F
:108FF0005B4600F0F3FA22462B4600F039F905B043
:10900000BDE8F08F2046294605B0BDE8F08F00BFCF
:10901000495555555555C53F0000E03F7CD5CF5AC1
:109020003AD9E53DEB9C2B8AE6E55A3E7DFEB157E9
:10903000E31DC73ED561C119A0012A3FA6F8101152
:109040001111813F21F000431946704700000000D4
:109050002DE9F041C1F30A57A7F2FF35132D02465F
:109060000B460C46884606461DDC002D3CDB364F81
:109070002F4101EA070C5CEA000C19D030A3D3E9B8
:10908000002300F0F5F80022002300F037FDC8B3FC
:10909000002C04DA4FF4801343FA05F5A84428EABB
:1090A000070400262EE0332D06DDB5F5806F2DD0A8
:1090B00010461946BDE8F081A7F213474FF0FF3C78
:1090C0002CFA07F70742F3D01DA3D3E9002300F0E1
:1090D000CFF80022002300F011FD98B1002C21DB15
:1090E00026EA070644460DE015A3D3E9002300F065
:1090F000BFF80022002300F001FD18B1002C08DBAE
:109100000026344621463046BDE8F08100F0B0F834
:10911000D0E724F000430D4A1E43002E18BF14462A
:109120000026EFE7142D08D00123C5F1340503FA1A
:1091300005F5AE1928BF9844D2E704F10108CFE73E
:109140009C7500883CE4377EFFFF0F000000F0BFF5
:109150000020704700000000F8B5C1F30A53044630
:109160000D460E4617460BBB21F00046034633431F
:109170001BD0354B002200F031FA344B9F4204469D
:109180000D4635DBC1F30A530E46363B3B4440F2F5
:10919000FE72934232DC002B11DD26F0FF4626F4EE
:1091A000E00646EA035520462946F8BD40F2FF7224
:1091B0009342EBD102460B4600F05AF8F8BD13F18A
:1091C000350F28DA4CF250339F4222462B460ADDF7
:1091D00019A1D1E9000100F03DF817A3D3E900235C
:1091E00000F0FCF9F8BD16A1D1E9000100F032F859
:1091F00013A3D3E9002300F0F1F9F8BD22462B4672
:109200000DA1D1E9000100F025F80BA3D3E900235B
:1092100000F0E4F9F8BD26F0FF4626F4E006363308
:1092200046EA0355204629460022094B00F0D6F9AC
:10923000F8BD00BFAFF300809C7500883CE4377E2A
:1092400059F3F8C21F6EA50100005043B03CFFFF68
:109250000000903C03F0004321F0004242EA030189
:10926000704700BF81F0004102E000BF83F000437F
:1092700030B54FEA41044FEA430594EA050F08BFB1
:1092800090EA020F1FBF54EA000C55EA020C7FEA75
:10929000645C7FEA655C00F0E2804FEA5454D4EBF2
:1092A0005555B8BF6D420CDD2C4480EA020281EABC
:1092B000030382EA000083EA010180EA020281EAF4
:1092C0000303362D88BF30BD11F0004F4FEA013146
:1092D0004FF4801C4CEA113102D0404261EB410155
:1092E00013F0004F4FEA03334CEA133302D05242DB
:1092F00063EB430394EA050F00F0A780A4F1010497
:10930000D5F1200E0DDB02FA0EFC22FA05F28018D0
:1093100041F1000103FA0EF2801843FA05F35941B6
:109320000EE0A5F120050EF1200E012A03FA0EFC35
:1093300028BF4CF0020C43FA05F3C01851EBE3715F
:1093400001F0004507D54FF0000EDCF1000C7EEB7C
:1093500000006EEB0101B1F5801F1BD3B1F5001FBA
:109360000CD349085FEA30004FEA3C0C04F10104D9
:109370004FEA445212F5800F80F09A80BCF1004F02
:1093800008BF5FEA500C50F1000041EB045141EA84
:10939000050130BD5FEA4C0C404141EB010111F485
:1093A000801FA4F10104E9D191F0000F04BF014630
:1093B0000020B1FA81F308BF2033A3F10B03B3F10E
:1093C00020020CDA0C3208DD02F1140CC2F10C029E
:1093D00001FA0CF021FA02F10CE002F11402D8BFFC
:1093E000C2F1200C01FA02F120FA0CFCDCBF41EAC8
:1093F0000C019040E41AA2BF01EB0451294330BD97
:109400006FEA04041F3C1CDA0C340EDC04F1140473
:10941000C4F1200220FA04F001FA02F340EA03004A
:1094200021FA04F345EA030130BDC4F10C04C4F190
:10943000200220FA02F001FA04F340EA0300294670
:1094400030BD21FA04F0294630BD94F0000F83F4BA
:10945000801306BF81F480110134013D4EE77FEA9D
:10946000645C18BF7FEA655C29D094EA050F08BFE9
:1094700090EA020F05D054EA000C04BF19461046CA
:1094800030BD91EA030F1EBF0021002030BD5FEA0E
:10949000545C05D14000494128BF41F0004130BD36
:1094A00014F580043CBF01F5801130BD01F000458A
:1094B00045F0FE4141F470014FF0000030BD7FEAFD
:1094C000645C1ABF194610467FEA655C1CBF0B46F8
:1094D000024650EA013406BF52EA033591EA030F0F
:1094E00041F4002130BD00BF90F0000F04BF002107
:1094F000704730B54FF4806404F132044FF000053A
:109500004FF0000150E700BF90F0000F04BF0021B2
:10951000704730B54FF4806404F1320410F0004518
:1095200048BF40424FF000013EE700BF42004FEA13
:10953000E2014FEA31014FEA02701FBF12F07F4390
:1095400093F07F4F81F06051704732F07F4208BF47
:10955000704793F07F4F04BF41F40021704730B54E
:109560004FF4607401F0004521F000411CE700BF9A
:1095700050EA010208BF704730B54FF000050AE01D
:1095800050EA010208BF704730B511F0004502D51E
:10959000404261EB41014FF4806404F132045FEA20
:1095A000915C3FF4D8AE4FF003025FEADC0C18BFC9
:1095B00003325FEADC0C18BF033202EBDC02C2F1BB
:1095C000200300FA03FC20FA02F001FA03FE40EA4D
:1095D0000E0021FA02F11444BDE600BF70B54FF051
:1095E000FF0C4CF4E06C1CEA11541DBF1CEA13552F
:1095F00094EA0C0F95EA0C0F00F0DEF82C4481EA97
:10960000030621EA4C5123EA4C5350EA013518BFB6
:1096100052EA033541F4801143F4801338D0A0FBA3
:1096200002CE4FF00005E1FB02E506F00042E0FB50
:1096300003E54FF00006E1FB03569CF0000F18BF56
:109640004EF0010EA4F1FF04B6F5007F64F54074FE
:1096500004D25FEA4E0E6D4146EB060642EAC62191
:1096600041EA55514FEAC52040EA5E504FEACE2EFE
:10967000B4F1FD0C88BFBCF5E06F1ED8BEF1004F01
:1096800008BF5FEA500E50F1000041EB045170BD7D
:1096900006F0004646EA010140EA020081EA0301C1
:1096A000B4EB5C04C2BFD4EB0C0541EA045170BDBD
:1096B00041F480114FF0000E013C00F3AB8014F137
:1096C000360FDEBF002001F0004170BDC4F1000480
:1096D000203C35DA0C341BDC04F11404C4F1200501
:1096E00000FA05F320FA04F001FA05F240EA02005C
:1096F00001F0004221F0004110EBD37021FA04F692
:1097000042EB06015EEA430E08BF20EAD37070BD4B
:10971000C4F10C04C4F1200500FA04F320FA05F0AA
:1097200001FA04F240EA020001F0004110EBD370AC
:1097300041F100015EEA430E08BF20EAD37070BD1C
:10974000C4F1200500FA05F24EEA020E20FA04F3F5
:1097500001FA05F243EA020321FA04F001F00041A4
:1097600021FA04F220EA020000EBD3705EEA430E15
:1097700008BF20EAD37070BD94F0000F0FD101F044
:109780000046400041EB010111F4801F08BF013C7D
:10979000F7D041EA060195F0000F18BF704703F0BB
:1097A0000046520043EB030313F4801F08BF013D42
:1097B000F7D043EA0603704794EA0C0F0CEA1355FE
:1097C00018BF95EA0C0F0CD050EA410618BF52EAB8
:1097D0004306D1D181EA030101F000414FF00000BE
:1097E00070BD50EA410606BF1046194652EA4306CC
:1097F00019D094EA0C0F02D150EA013613D195EA40
:109800000C0F05D152EA03361CBF104619460AD187
:1098100081EA030101F0004141F0FE4141F4700191
:109820004FF0000070BD41F0FE4141F4780170BD81
:1098300070B54FF0FF0C4CF4E06C1CEA11541DBFE6
:109840001CEA135594EA0C0F95EA0C0F00F0A7F8E8
:10985000A4EB050481EA030E52EA03354FEA013115
:1098600000F088804FEA03334FF0805545EA131328
:1098700043EA12634FEA022245EA111545EA1065F0
:109880004FEA00260EF000419D4208BF964244F187
:10989000FD0404F5407402D25B084FEA3202B61AA6
:1098A00065EB03055B084FEA32024FF480104FF47A
:1098B000002CB6EB020E75EB030E22BFB61A7546EE
:1098C00040EA0C005B084FEA3202B6EB020E75EB81
:1098D000030E22BFB61A754640EA5C005B084FEAE9
:1098E0003202B6EB020E75EB030E22BFB61A7546B6
:1098F00040EA9C005B084FEA3202B6EB020E75EBC1
:10990000030E22BFB61A754640EADC0055EA060E81
:1099100018D04FEA051545EA16754FEA06164FEAC4
:10992000C30343EA52734FEAC2025FEA1C1CC0D170
:1099300011F4801F0BD141EA00014FF000004FF0FD
:10994000004CB6E711F4801F04BF01430020B4F1BE
:10995000FD0C88BFBCF5E06F3FF6AFAEB5EB030C76
:1099600004BFB6EB020C5FEA500C50F1000041EB73
:10997000045170BD0EF0004E4EEA113114EB5C0440
:10998000C2BFD4EB0C0541EA045170BD41F4801113
:109990004FF0000E013C90E645EA060E8DE60CEA1B
:1099A000135594EA0C0F08BF95EA0C0F3FF43BAF38
:1099B00094EA0C0F0AD150EA01347FF434AF95EAEF
:1099C0000C0F7FF425AF104619462CE795EA0C0FD3
:1099D00006D152EA03353FF4FDAE1046194622E7A0
:1099E00050EA410618BF52EA43067FF4C5AE50EA7A
:1099F00041047FF40DAF52EA43057FF4EBAE12E76A
:109A00004FF0FF3C06E000BF4FF0010C02E000BF4A
:109A10004FF0010C4DF804CD4FEA410C7FEA6C5C2D
:109A20004FEA430C18BF7FEA6C5C1BD001B050EAD0
:109A3000410C0CBF52EA430C91EA030F02BF90EABB
:109A4000020F0020704710F1000F91EA030F58BF7A
:109A5000994208BF90422CBFD8176FEAE37040F0DC
:109A6000010070474FEA410C7FEA6C5C02D150EA7A
:109A7000013C07D14FEA430C7FEA6C5CD6D152EA35
:109A8000033CD3D05DF8040B704700BF84461046FA
:109A900062468C461946634600E000BF01B5FFF7F9
:109AA000B7FF002848BF10F1000F01BD4DF808EDC9
:109AB000FFF7F4FF0CBF012000205DF808FB00BF9A
:109AC0004DF808EDFFF7EAFF34BF012000205DF8F4
:109AD00008FB00BF4DF808EDFFF7E0FF94BF012041
:109AE00000205DF808FB00BF4DF808EDFFF7CEFF42
:109AF00094BF012000205DF808FB00BF4DF808ED81
:109B0000FFF7C4FF34BF012000205DF808FB00BF51
:109B10004FEA410C7FEA6C5C02D150EA013C0AD169
:109B20004FEA430C7FEA6C5C02D152EA033C02D15B
:109B30004FF0000070474FF0010070474FEA4102BC
:109B400012F5001215D211D56FF47873B3EB62528F
:109B500012D94FEAC12343F0004343EA505311F0B6
:109B6000004F23FA02F018BF404270474FF0000048
:109B7000704750EA013005D111F0004008BF6FF086
:109B8000004070474FF00000704700BF1FB51C46F3
:109B9000094B1B680546D86852B1084B0091CDE9C6
:109BA000013207492B46224600F028F800F0BAFDA2
:109BB000044B1A46F2E700BF5400002010CA000010
:109BC0001DCA0000FFB70000014B1868704700BFB6
:109BD0005400002008B5074B044613B10021AFF331
:109BE0000080054B1868836A03B19847204601F04E
:109BF00071FB00BF000000004CCA00000EB403B5AA
:109C0000014603AB054853F8042B0068019300F0AC
:109C100081F802B05DF804EB03B0704754000020F7
:109C200070B50D4E0D4CA41BA4100025A54209D102
:109C30000B4E0C4C01F050FBA41BA4100025A542B8
:109C400005D170BD56F8253098470135EEE756F836
:109C5000253098470135F2E7240200202402002035
:109C6000240200203402002010B5431E0A44914211
:109C700000D110BD11F8014B03F8014FF7E78842FE
:109C800010B501EB020307D8421E99420AD011F821
:109C9000014B02F8014FF8E78342F5D98118D21A37
:109CA000D34200D110BD13F8014D01F8014DF7E783
:109CB00002440346934200D1704703F8011BF9E7C1
:109CC0009368013B002B10B4936008DA9469A342B7
:109CD00001DB0A2903D15DF8044B00F063BC136873
:109CE000581C1060197008465DF8044B7047F8B5B1
:109CF00006460F461446D518AC4201D1002007E0B5
:109D00003A4614F8011B3046FFF7DAFF431CF3D143
:109D1000F8BD00002DE9F04F9DB00C4617460393A7
:109D2000064618B183690BB900F0F4FD7B4B9C42E9
:109D300057D17468A38918075DD52369002B5AD0C1
:109D40000023099320238DF8293030238DF82A3001
:109D50004FF0010BB846454615F8013B0BB1252BDA
:109D600054D1B8EB070A0BD053463A462146304649
:109D7000FFF7BDFF013000F0C280099B53440993F7
:109D800098F80030002B00F0BA8000234FF0FF322B
:109D9000CDE90523049307938DF853301A93A84611
:109DA000052218F8011B5E4800F0C2FE049B78BB38
:109DB000D90644BF20228DF853201A0744BF2B2216
:109DC0008DF853202A782A2A2AD0079AA8460020FC
:109DD0000A25414611F8013B303B092B69D960B394
:109DE00024E0504B9C4201D1B468A3E74E4B9C4207
:109DF00008BFF4689EE72146304600F025FC0028A5
:109E00009ED04FF0FF301DB0BDE8F08FA846A2E70E
:109E1000434A801A0BFA00F0184304904546BEE707
:109E2000039A111D12680391002A01DB079204E0D6
:109E3000524243F002030792049398F800302E2B0D
:109E40000ED198F801302A2B38D1039B1A1D1B68BC
:109E50000392002BB8BF4FF0FF3308F102080593BF
:109E6000324D98F800100322284600F061FE40B100
:109E70004023401B03FA00F0049B034308F1010850
:109E8000049398F800102A488DF82810062208F14B
:109E9000010700F04DFE002837D0264B1BBB039B6B
:109EA000073323F0070308330393099B4B440993BB
:109EB00050E705FB0232012088468AE7002308F1BB
:109EC0000108059319460A25404610F8012B303A3F
:109ED000092A03D9002BC3D00591C1E705FB012155
:109EE00001238046F0E703AB00932246124B04A9FE
:109EF0003046AFF30080B0F1FF3F8146D5D1A38952
:109F00005B063FF57EAF09987DE703AB00932246E1
:109F1000094B04A9304600F087F8ECE7A4CA00001A
:109F200050CA0000C4CA000084CA000056CA00001B
:109F30005ACA000000000000EF9C00002DE9F04725
:109F400091461F468A680B69DDF820809342B8BFAE
:109F50001346C9F8003091F8432006460C4612B16A
:109F60000133C9F800302368990642BFD9F80030A0
:109F70000233C9F80030256815F0060507D104F151
:109F8000190AE368D9F800209B1AAB4228DC94F840
:109F900043302268003318BF012392062DD404F108
:109FA000430239463046C047013020D02368E56877
:109FB000D9F8002003F00603042B08BFAD1AA368EC
:109FC00022690CBF25EAE57500259342C4BF9B1AA0
:109FD000ED184FF000091A344D451AD1002008E061
:109FE0000123524639463046C047013003D14FF075
:109FF000FF30BDE8F0870135C3E7E1185A1C302077
:10A0000081F84300224494F8451082F8431002334B
:10A01000C5E70123224639463046C0470130E6D025
:10A0200009F10109D8E700002DE9F04301F1430CE3
:10A030000C46097E85B06E291746064698460C9A4E
:10A0400000F0B38022D8632936D00AD8002900F066
:10A05000B980582900F0838004F1420584F8421049
:10A0600032E0642901D06929F6D120681368050619
:10A0700003F104012AD51B681160002B03DA2D229D
:10A080005B4284F843206F480A2239E0732900F0CC
:10A090009D8008D86F2920D07029DDD1236843F036
:10A0A0002003236003E0752917D07829D4D17823C1
:10A0B00084F84530644855E01368191D1B68116029
:10A0C00004F1420584F8423001238CE01B681160E2
:10A0D00010F0400F18BF1BB2CFE713682568181D9A
:10A0E0001060280601D51B6802E06806FBD51B88B6
:10A0F00054486F2914BF0A220822002184F8431013
:10A100006568A560002DC0F29580216821F00401EA
:10A110002160002B3DD1002D40F08E806546082A3D
:10A120000BD12368DB0708D5236962689A42DEBF3A
:10A13000302305F8013C05F1FF35ACEB0503236145
:10A14000CDF800803B4603AA21463046FFF7F6FED5
:10A1500001304DD14FF0FF3005B0BDE8F0833948F4
:10A1600084F84510136821681D1D1B6815600A06D8
:10A170000BD5CA0744BF41F0200121601BB92268FA
:10A1800022F0200222601022B7E74D0648BF9BB2A2
:10A19000EFE76546B3FBF2F102FB1133C35C05F850
:10A1A000013D0B460029F5D1B9E7136825686169BF
:10A1B000181D106028061B6801D5196002E06A06A8
:10A1C000FBD51980002323616546B9E71368191D83
:10A1D00011601D6862680021284600F0A9FC08B1E2
:10A1E000401B606063682361002384F84330A7E765
:10A1F00023692A4639463046C0470130AAD0236831
:10A200009B0713D4E068039B9842B8BF1846A3E7A6
:10A2100001234A4639463046C04701309AD00135BD
:10A22000E368039A9B1AAB42F2DCEBE7002504F1EA
:10A230001909F5E7002BACD1037884F8423004F11A
:10A2400042056CE761CA000072CA000038B50D4BC8
:10A250001C68A36B05467BB9182000F04DFC0A4A28
:10A260000A4BA063C0E90023094B83600B23838161
:10A2700001220023C0E90423A36B00221D615A615F
:10A2800038BD00BF540000200E33CDAB34126DE654
:10A29000ECDE050038B5134B1C68A36B7BB91820A6
:10A2A00000F02AFC104A114BA063C0E90023104BB8
:10A2B00083600B23838101220023C0E90423A16B67
:10A2C0000C480A694B690C4C504304FB0300A2FB89
:10A2D00004230344541C43F10005C1E9044525F05F
:10A2E000004038BD540000200E33CDAB34126DE673
:10A2F000ECDE05002DF451582D7F954C0CB430B593
:10A30000174B0C1E9DB01D6808DA8B232B604FF095
:10A31000FF301DB0BDE8304002B070474FF402730B
:10A32000ADF8143014BF04F1FF33234604930793B0
:10A330004FF6FF7302900690ADF81630209A21ABCD
:10A3400002A92846019300F06BFD431CBCBF8B2380
:10A350002B60002CDDD0029B00221A70D9E700BFD1
:10A36000540000200EB400B59CB01DAB02900690C6
:10A370006FF00041094807910491094953F8042BF3
:10A3800005910068019302A900F04AFD029B00229A
:10A390001A701CB05DF804EB03B070475400002045
:10A3A0000802FFFF10B503461A785C1C3AB9013B5E
:10A3B00011F8012B03F8012F002AF9D110BD234613
:10A3C000F2E7C9B2034610F8012B1AB18A42F9D15B
:10A3D00018467047002918BF0023F9E710F8012B31
:10A3E00011F8013B012A28BF9A42F7D0D01A7047D2
:10A3F000034613F8012B002AFBD1181A01387047C5
:10A4000010B56AB10139841810F8013B11F8012F19
:10A41000934203D1A04201D0002BF5D1981A10BD70
:10A420001046FCE770B50139044602B970BD2346F9
:10A4300011F8015F03F8015B561E2DB91444A342C5
:10A44000F4D003F8015BFAE71C463246EDE7F0B5BD
:10A4500003787BB1044623782046661C7BB14A1EF4
:10A46000631E12F8015F4DB113F8017FAF4234460D
:10A47000F7D0F0E70B78002B18BF0020F0BD18468E
:10A48000FCE72DE9F0478046894692461E460F4676
:10A490003D46089815F8014B00F0C6FA2044437871
:10A4A00013F0080332D12D2C32D17C78BD1C01224F
:10A4B000002E5DD0102E09D1302C07D12B7803F05F
:10A4C000DF03582B4FD16C7810260235002A14BFB9
:10A4D0004FF000416FF000410027B1FBF6FC384619
:10A4E00006FB1C1EA4F13003092B17D81C46A642FC
:10A4F00023DD7B1C07D084451CD301D1A64519DB85
:10A5000000FB0640012715F8014BEBE72F46BFE79C
:10A510002B2C04BFBD1C7C781A46C9E7A4F141036B
:10A52000192B01D8373CE2E7A4F16103192B04D8B9
:10A53000573CDCE74FF0FF37E5E77B1C08D12223CF
:10A54000C8F800300846BAF1000F07D1BDE8F0871F
:10A5500002B14042BAF1000FF8D00FB105F1FF3956
:10A56000CAF80090F2E73024002EAFD10826ADE7FC
:10A57000302CA3D00A26A9E7084B37B51C68084D34
:10A58000236A002B08BF2B46009313460A46014658
:10A590002046FFF776FF03B030BD00BF5400002017
:10A5A000B8000020F8B50E461446054618B1836978
:10A5B0000BB900F0AFF9214B9C422AD16C68A3691A
:10A5C000A360A3891A072ED5236963B32369206882
:10A5D000C01A6369F6B28342374604DC2146284636
:10A5E00000F02EF928BBA368013BA36023685A1C26
:10A5F00022601E7063690130834204D0A389DB07A7
:10A6000019D50A2E17D12146284600F019F990B124
:10A610000FE00B4B9C4201D1AC68D0E7094B9C4248
:10A6200008BFEC68CBE72146284600F00DF800286B
:10A63000CCD04FF0FF373846F8BD00BFA4CA0000A9
:10A64000C4CA000084CA0000324B70B51D680646BB
:10A650000C4625B1AB6913B9284600F05BF92E4BC7
:10A660009C420FD16C68B4F90C309AB215072CD407
:10A67000D00611D40922326043F04003A3814FF089
:10A68000FF303EE0254B9C4201D1AC68EBE7244B08
:10A690009C4208BFEC68E6E7510712D5616B41B1F7
:10A6A00004F14403994202D0304600F091FA0023AD
:10A6B0006363A38923F02403A381002363602369D8
:10A6C0002360A38943F00803A38123694BB9A389BD
:10A6D00003F42073B3F5007F03D02146304600F029
:10A6E000CBF9A28912F001030CD00023A3606369A7
:10A6F0005B42A361236953B9B4F90C3013F08000B5
:10A70000BAD170BD920758BF6369A360F2E7002019
:10A71000F7E700BF54000020A4CA0000C4CA00002C
:10A7200084CA000008B5062000F0A8FC012000F053
:10A73000D1FD00008A892DE9F041054610070C463D
:10A7400058D44B68002B05DC0B6C002B02DC00207E
:10A75000BDE8F081E66A002EF9D0002312F48052A1
:10A760002F68216A2B6032D0606DA3895A0705D506
:10A770006368C01A636B0BB1236CC01A00230246D6
:10A78000E66A216A2846B047431CA38906D1296896
:10A790001D2948D8294ACA40D60744D500226260FC
:10A7A000D9042269226004D5421C01D12B6803B967
:10A7B0006065616B2F600029C9D004F144039942A0
:10A7C00002D0284600F004FA00206063C0E70123AD
:10A7D0002846B047411CC8D12B68002BC5D01D2B83
:10A7E00001D0162B01D12F60B1E7A38943F04003BC
:10A7F000A381ADE70F69002FA9D093070E6808BFAA
:10A800004B690F6018BF0023A6EB07088B60B8F1F7
:10A81000000F9CDD43463A46216AA66A2846B047A7
:10A82000002806DCA38943F04003A3814FF0FF30EA
:10A830008EE70744A8EB0008E9E700BF01004020CD
:10A8400038B50B6905460C46DBB118B183690BB905
:10A8500000F060F80C4B9C4209D16C68B4F90C30E4
:10A860007BB121462846BDE83840FFF763BF074B60
:10A870009C4201D1AC68F1E7054B9C4208BFEC68F3
:10A88000ECE7002038BD00BFA4CA0000C4CA000025
:10A8900084CA0000002310B50446C0E90033836079
:10A8A00081814366C281C0E904338361194608226D
:10A8B0005C30FFF7FDF9054B6362054BA362054B66
:10A8C000E362054B2462236310BD00BFB5B00000F6
:10A8D000D7B000000FB1000033B10000014900F013
:10A8E00085B800BF41A8000070B54A1E68255543D1
:10A8F0000E4605F1740100F0B9F9044640B100219B
:10A90000C0E900160C30A06005F16802FFF7D0F92D
:10A91000204670BD836910B5044633BBC0E91233CD
:10A920000365124B124A1B688262984204BF0123DE
:10A93000836100F01FF86060204600F01BF8A06003
:10A94000204600F017F80022E06004216068FFF75D
:10A95000A1FF01220921A068FFF79CFF022212211A
:10A96000E068FFF797FF0123A36110BD4CCA000008
:10A97000DDA80000F8B51B4B1E68B369074613B984
:10A980003046FFF7C7FF4836D6E90134013B03D50F
:10A99000336833B13668F7E7B4F90C506DB16834F9
:10A9A000F4E704213846FFF79FFF30600028F1D11B
:10A9B0000C233B6004462046F8BD0B4B6566C4E99A
:10A9C0000055A560C4E90335C4E9055508222946A8
:10A9D00004F15C00FFF76CF9C4E90D55C4E91255A8
:10A9E000E9E700BF4CCA00000100FFFF2DE9F84372
:10A9F0008046894600F14804002614B93046BDE877
:10AA0000F883D4E90175013F01D52468F5E7AB89E6
:10AA1000012B07D9B5F90E30013303D02946404642
:10AA2000C84706436835EEE7D0F8EC00704770B5CC
:10AA30000E46B1F90E10002996B014461D4607DAED
:10AA400000232B60B3891A0610D44FF480630EE004
:10AA50006A4600F0A1FB0028F2DB019A02F4704282
:10AA6000A2F500535A425A412A60EEE740230020E3
:10AA7000236016B070BD00008B8973B59D07064634
:10AA80000C4607D504F1470323602361012363616A
:10AA900002B070BD01AB6A46FFF7C9FF00990546D9
:10AAA000304600F0E3F848B9B4F90C309A05EFD419
:10AAB00023F0030343F00203A381E3E70D4BB362EA
:10AAC000A389206043F08003A381009B6361019B05
:10AAD00020615BB1B4F90E10304600F06FFB28B175
:10AAE000A38923F0030343F00103A381A3891D433A
:10AAF000A581CDE7DDA80000024B0146186800F0F3
:10AB0000B5B800BF5400002082B001B901A942B11C
:10AB10004BB113780B601278101C18BF012002B0E3
:10AB200070471046FBE76FF00100F8E700000000F7
:10AB300001F0FF01102A2BDB10F0070F08D010F8EE
:10AB4000013B013A8B422DD010F0070F42B3F6D1F2
:10AB5000F0B441EA012141EA014122F007047FF00B
:10AB600000070023F0E80256083C85EA010586EA62
:10AB7000010685FA47F5A3FA87F586FA47F6A5FA9E
:10AB800087F68EB9EED1F0BC01F0FF0102F00702AA
:10AB900032B110F8013B013A83EA010313B1F8D155
:10ABA0000020704701387047002D06BF3546033836
:10ABB000073815F0010F07D1013015F4807F02BF6F
:10ABC000013015F4C03F0130F0BC0138704700BFC0
:10ABD00038B50546002945D051F8043C0C1F002B20
:10ABE000B8BFE41800F00CFB1F4A1368104633B9D5
:10ABF000636014602846BDE8384000F002BBA34201
:10AC00000CD921686218934204BF1A685B686360BC
:10AC100004BF521822600460ECE713465A680AB178
:10AC2000A242FAD919685818A0420BD120680144F1
:10AC3000581882421960DDD1106852685A60014488
:10AC40001960D7E702D90C232B60D3E720682118BD
:10AC50008A4204BF11685268626004BF091821600B
:10AC60005C60C7E738BD00BF647A012070B5CD1CB9
:10AC700025F0030508350C2D38BF0C25002D0646A0
:10AC800001DBA94203D90C233360002070BD00F022
:10AC9000B7FA214A1468214691B9204C23681BB9A0
:10ACA000304600F0B3F920602946304600F0AEF996
:10ACB000431C24D10C233360304600F0A2FAE4E7B1
:10ACC0000B685B1B18D40B2B0FD90B60CD50CC1825
:10ACD000304600F096FA04F10B00231D20F0070027
:10ACE000C31AD3D05A42E250D0E78C424B6816BF09
:10ACF000636013600C46EBE70C464968CCE7C41C64
:10AD000024F00304A04205D0211A304600F07EF959
:10AD10000130CFD02560DBE7647A0120687A01201A
:10AD2000F8B5074614460E4621B91146BDE8F8406D
:10AD3000FFF79CBF22B9FFF74BFF25462846F8BD19
:10AD400000F060FAA0420FD221463846FFF78EFF8E
:10AD500005460028F2D031462246FEF785FF3146EF
:10AD60003846FFF735FFE9E73546E7E72DE9F047D5
:10AD70008E689E4282460C469046994637D88A890C
:10AD800012F4906F31D0256809696F1A6569022342
:10AD900005EB450595FBF3F509F101033B449D42A5
:10ADA00038BF1D46530530D52946FFF75FFF0646DD
:10ADB00050B90C23CAF80030A38943F04003A381A3
:10ADC0004FF0FF30BDE8F0873A462169FEF74CFFAF
:10ADD000A38923F4906343F08003A3812661656116
:10ADE0003E44ED1B2660A5604E464E4500D94E46BA
:10ADF000324641462068FEF742FFA3689B1BA360D2
:10AE000023681E4426600020DCE72A46FFF788FFFF
:10AE100006460028E2D121695046FFF7D9FEC8E76F
:10AE20002DE9F04F9DB0804603938B891D060C469B
:10AE300016460FD50B696BB94021FFF717FF20604D
:10AE4000206128B90C23C8F800304FF0FF30C7E06C
:10AE5000402363610023099320238DF82930302398
:10AE60008DF82A304FF0010B37463D4615F8013B6F
:10AE70000BB1252B3ED1B7EB060A0BD05346324619
:10AE800021464046FFF772FF013000F0A480099B85
:10AE9000534409933B78002B00F09D8000234FF032
:10AEA000FF32CDE90523049307938DF853301A93AD
:10AEB0002F46052217F8011B4F48FFF739FE049B68
:10AEC000D0B9D90644BF20228DF853201A0744BFB9
:10AED0002B228DF853202A782A2A15D0079A2F463C
:10AEE00000200A25394611F8013B303B092B4DD98A
:10AEF000B8B10FE02F46B8E73F4A801A0BFA00F0CE
:10AF0000184304903D46D3E7039A111D126803913C
:10AF1000002A01DB079204E0524243F00203079249
:10AF200004933B782E2B0CD17B782A2B33D1039BB7
:10AF30001A1D1B680392002BB8BF4FF0FF33023776
:10AF400005932E4D397803222846FFF7F1FD38B1DD
:10AF50004023401B03FA00F0049B03430137049392
:10AF6000397827488DF8281006227E1CFFF7E0FD6F
:10AF7000002838D0234B13BB039B073323F0070370
:10AF800008330393099B4B4409936DE705FB023299
:10AF900001200F46A6E700230137059319460A252D
:10AFA000384610F8012B303A092A03D9002BC8D0B3
:10AFB0000591C6E705FB012101230746F0E703AB36
:10AFC00000932246104B04A94046AFF30080B0F135
:10AFD000FF3F8146D6D1A3895B063FF536AF09987E
:10AFE0001DB0BDE8F08F03AB00932246064B04A9C9
:10AFF0004046FFF719F8EAE750CA000056CA0000B9
:10B000005ACA0000000000006DAD000038B5064CC3
:10B01000002305460846236000F046F9431C02D190
:10B02000236803B12B6038BDF88D01201F2938B586
:10B0300004460D4604D9162303604FF0FF3038BD97
:10B04000426C12B152F821304BB9204600F030F872
:10B050002A4601462046BDE8384000F017B8012BCB
:10B060000AD0591C03D1162303600120E7E700240E
:10B0700042F82540284698470020E0E7024B014669
:10B080001868FFF7D3BF00BF5400002038B5074C45
:10B090000023054608461146236000F0EDF8431CE6
:10B0A00002D1236803B12B6038BD00BFF88D0120A9
:10B0B00000F0D2B810B50C46B1F90E1000F0AAF8A5
:10B0C0000028ABBF636DA3891B1823F48053ACBF6A
:10B0D0006365A38110BD2DE9F0411F468B89DB0517
:10B0E00005460C46164605D502230022B1F90E107E
:10B0F00000F074F8A389B4F90E1023F48053A381EF
:10B1000032463B462846BDE8F04100F023B810B572
:10B110000C46B1F90E1000F061F8431CA38915BF6D
:10B12000606523F4805343F48053A38118BFA38147
:10B1300010BDB1F90E1000F01FB849B1FF2A85BF4C
:10B140008A2303600A704FF0FF3098BF01207047D8
:10B150000846704738B5074C054608461146002298
:10B1600022601A4600F0AEF8431C02D1236803B1F6
:10B170002B6038BDF88D012038B5064C00230546FC
:10B180000846236000F058F8431C02D1236803B13D
:10B190002B6038BDF88D012038B5074C00230546DB
:10B1A00008461146236000F04FF8431C02D1236883
:10B1B00003B12B6038BD00BFF88D012038B5064CB7
:10B1C000002305460846236000F04EF8431C02D1D8
:10B1D000236803B12B6038BDF88D012038B5074CCA
:10B1E000054608461146002222601A4600F04CF837
:10B1F000431C02D1236803B12B6038BDF88D0120B8
:10B200007047704751F8043C181F002BBCBF0B5807
:10B21000C018704738B5074C05460846114600224D
:10B2200022601A4600F038F8431C02D1236803B1AB
:10B230002B6038BDF88D0120024B58221A604FF068
:10B24000FF307047F88D0120024B58221A604FF0F2
:10B25000FF307047F88D0120024B58221A604FF0E2
:10B26000FF307047F88D0120024B58221A600020F1
:10B27000704700BFF88D0120024B58221A604FF032
:10B28000FF307047F88D0120024B58221A604FF0B2
:10B29000FF307047F88D0120024B58221A604FF0A2
:10B2A000FF307047F88D0120044A05491368002BD0
:10B2B00008BF0B4618441060184670476C7A01208E
:10B2C000008E0120024B58221A604FF0FF30704769
:10B2D000F88D0120FEE700BFF8B500BFF8BC08BC40
:10B2E0009E467047F8B500BFF8BC08BC9E46704744
:10B2F000646174610000000074B300001D0300006D
:10B300007DB300000D04000085B30000E9090000D2
:10B310008CB30000F90A000091B30000430600005E
:10B320009CB3000077040000A1B30000350D0000BD
:10B33000ADB300004F030000B7B3000001090000E7
:10B34000C5B30000CF070000D2B300000B06000019
:10B3500072616E646F6D00616C6C006C617374007F
:10B3600066616C7365007472756500252E313573E6
:10B370002E2E2E006D616B654C69737400616464E0
:10B380004C6173740064656C657465006A6F696E06
:10B3900000636F707946726F6D546F0066696E64FA
:10B3A000006A6F696E537472696E677300756E69B7
:10B3B000636F6465417400756E69636F646553748F
:10B3C00072696E67006E6577427974654172726169
:10B3D0007900667265654D656D6F727900000000D9
:10B3E00045B40000AD1100004AB40000C7110000D0
:10B3F00085B30000CB11000050B40000B111000073
:10B400005AB40000CF11000063B40000D311000053
:10B410006DB40000D711000078B40000DB1100000B
:10B4200084B40000B51100008DB40000BF1100000D
:10B4300097B40000B9110000A2B40000C3110000CD
:10B4400066696C65006F70656E00636C6F73650094
:10B45000656E644F6646696C6500726561644C692F
:10B460006E65007265616442797465730061707025
:10B47000656E644C696E6500617070656E644279DA
:10B480007465730066696C6553697A6500737461ED
:10B4900072744C697374006E657874496E4C69738C
:10B4A000740073797374656D496E666F00000000F7
:10B4B000D8140000E8140000FC140000701500000F
:10B4C000A2150000D2150000041600002616000088
:10B4D000621600009A160000EA1600002A17000003
:10B4E00092170000D0170000F01700002418000089
:10B4F0006418000086180000B0180000DA18000078
:10B500001A190000921900005A1A0000CC1A000003
:10B51000161B0000781B0000941B0000B21B0000EB
:10B52000F01C00002C1D00009E1D0000CC1D000022
:10B53000F41D00002C1E0000901E0000F41E0000F0
:10B54000561F0000B81F00002C200000A42000009F
:10B5500004210000642100009A210000DE21000087
:10B56000242200006A220000BC22000012230000F6
:10B5700050230000C0230000F42300003A24000000
:10B5800080240000C624000000250000462500009D
:10B590008C250000E8260000B018000024180000E8
:10B5A00000260000D8140000342600005A260000AF
:10B5B0008E260000B4260000D8140000D814000025
:10B5C000D8140000D81400005E2700009E27000059
:10B5D000E2270000362800005C280000CA2800008E
:10B5E0001429000044290000D8140000D8140000D9
:10B5F0006229000094290000C6290000FA290000F1
:10B60000482A00007C2A0000A02A0000C22A00006C
:10B61000E42A0000162B0000482B00006C2B0000D1
:10B62000902B0000C22B0000E62B0000D814000075
:10B63000D8140000D8140000D8140000D81400005A
:10B64000182C00003E2C0000642C00008A2C000006
:10B65000B02C0000E42C0000182D00004C2D000040
:10B66000802D0000A62D0000CC2D0000002E000033
:10B67000D8140000D8140000D8140000D81400001A
:10B68000D8140000D8140000D8140000D81400000A
:10B69000D8140000D8140000D8140000D8140000FA
:10B6A000D8140000D8140000262E0000562E0000EA
:10B6B0005B2564206974656D206C6973745D002876
:10B6C00025642062797465732900286F626A656356
:10B6D0007420747970653A2025642900537461637D
:10B6E0006B20756E646572666C6F7700626F6F6C4D
:10B6F00065616E006E756D62657200737472696E5D
:10B7000067006C697374006279746520617272619C
:10B7100079000000070000000300000075B700007A
:10B72000712F00007DB700001D30000086B70000BB
:10B73000BB3000008FB70000752F000098B70000E5
:10B74000BF300000A0B70000AD30000000000000D6
:10B7500001000000020000000300000004000000DF
:10B760000A0000001D0000006D6963726F3A626993
:10B770007420763200686173546F6E6500706C617E
:10B7800079546F6E6500686173536572766F0073EC
:10B790006574536572766F00646163496E69740005
:10B7A000646163577269746500474320746F6F6BFF
:10B7B0002025642075736563733B20667265652080
:10B7C000256420776F726473003C496E7465676509
:10B7D000723E003C4C6973743E003C4F626A656384
:10B7E000743E003C4279746541727261793E000D8D
:10B7F0000A564D2050616E69633A2025730D0A0088
:10B800006D697363000000003DB80000153E000044
:10B8100046B80000993D00004AB80000E53C000031
:10B8200052B80000873C00005CB80000193C0000E2
:10B8300068B800001B3B00006E756C6C0068657892
:10B84000546F496E740073696E006A736F6E47655A
:10B8500074006A736F6E436F756E74006A736F6EF7
:10B8600056616C75654174006A736F6E4B65794102
:10B870007400000000B90000753E000008B9000027
:10B88000793E000012B900008B3E00001BB9000099
:10B89000913E000026B90000973E000032B900003A
:10B8A0009D3E000040B90000A33E000048B90000E2
:10B8B000A93E00004EB90000AF3E000063B9000091
:10B8C000B53E000078B90000BB3E000084B900001E
:10B8D000C13E000094B90000C73E0000A0B90000BE
:10B8E000CD3E0000ADB90000D33E0000BCB9000061
:10B8F0007F3E0000CFB90000853E00006E657400F9
:10B900006861735769466900737461727457694658
:10B91000690073746F705769466900776966695387
:10B920007461747573006D79495041646472657314
:10B9300073007374617274535349447363616E008E
:10B9400067657453534944006D794D4143006874F1
:10B95000747053657276657247657452657175656A
:10B96000737400726573706F6E64546F4874747092
:10B97000526571756573740068747470436F6E6E90
:10B9800065637400687474704973436F6E6E6563A9
:10B9900074656400687474705265717565737400C1
:10B9A00068747470526573706F6E7365007765624A
:10B9B000536F636B6574537461727400776562537F
:10B9C0006F636B65744C6173744576656E74007754
:10B9D0006562536F636B657453656E64546F436C3B
:10B9E00069656E74000000000400000003000000A0
:10B9F0000A00000007000000060000000000000030
:10BA00000008080800080A4A4000000A5FEA5FEAE6
:10BA10000ED92ED36E19324489330C924C924D08B4
:10BA20000800000004880808040804848488000AC8
:10BA3000448A4000048EC480000000048800000E88
:10BA4000C000000000080001224488100C925252ED
:10BA50004C048C84848E1C824C901E1EC244924CDA
:10BA600006CA525FE21FF01EC13E02448ED12E1F55
:10BA7000E24488100ED12ED12E0ED12EC48800089B
:10BA800000080000048004880244880482000EC07C
:10BA90000EC008048244880ED126C0040ED135B3EE
:10BAA0006C0C925ED2521C925C925C0ED010100E06
:10BAB0001C9252525C1ED01C901E1ED01C90100E68
:10BAC000D013712E12525ED2521C8808081C1FE23D
:10BAD00042524C1254981492101010101E113B75C3
:10BAE000B131113935B3710C9252524C1C925C90A9
:10BAF000100C92524C861C925C92510ED00C825CBF
:10BB00001FE4848484125252524C1131312A441160
:10BB10003135BB7112524C9252112A4484841EC496
:10BB200088101E0EC808080E10080482410EC2427A
:10BB3000424E048A400000000000001F08048000FC
:10BB400000000ED2524F10101C925C000ED0100E4E
:10BB500002424ED24E0C925C900E06C81C88080E13
:10BB6000D24EC24C10101C92520800080808024025
:10BB700002424C10149814920808080806001B751D
:10BB8000B131001C925252000C92524C001C925C3B
:10BB900090000ED24EC2000ED010100006C80498BD
:10BBA00008080EC807001252524F0011312A4400F3
:10BBB000113135BB00124C8C9200112A4498001EA2
:10BBC000C4881E06C48C8486080808080818080C57
:10BBD000881800000C8360000000000001000000D5
:10BBE0000200000003000000040000000500000047
:10BBF0000600000007000000080000000900000027
:10BC00000A0000000B0000000C0000000D00000006
:10BC10000E0000000F0000001000000012000000E5
:10BC20001400000016000000180000001A000000B8
:10BC30001C0000001E000000200000002300000087
:10BC400026000000290000002C0000002F0000004A
:10BC500032000000360000003A0000003E00000004
:10BC600042000000460000004B00000050000000B1
:10BC7000550000005A00000061000000680000004C
:10BC80006F000000760000007D00000084000000CE
:10BC90008B0000009200000099000000A00000004E
:10BCA000A7000000AE000000B5000000BC000000CE
:10BCB000C3000000CA000000D1000000D80000004E
:10BCC000DF000000E6000000ED000000F4000000CE
:10BCD000FB000000FF000000000000000200000068
:10BCE00004000000010000000300000050BD00003F
:10BCF000ED3E00005BBD00005D43000065BD00003F
:10BD0000A93F000072BD0000C941000079BD0000DC
:10BD10001542000082BD0000654200008EBD00009B
:10BD2000594100009FBD0000FD3F0000ACBD000078
:10BD3000E1400000150000001600000017000000A0
:10BD40001800000019000000646973706C617900CC
:10BD50006C696768744C6576656C006D62446973E4
:10BD6000706C6179006D62446973706C61794F66C3
:10BD700066006D62506C6F74006D62556E706C6F12
:10BD800074006D62447261775368617065006D6222
:10BD90005368617065466F724C6574746572006EAD
:10BDA000656F506978656C53656E64006E656F50A1
:10BDB0006978656C53657450696E004E6F742065C8
:10BDC0006E6F75676820726F6F6D206576656E2087
:10BDD000616674657220636F6D70616374696F6E04
:10BDE00000436F6D70616374656420466C617368B5
:10BDF00020636F64652073746F72650A2564206226
:10BE00007974657320757365642028256425252958
:10BE1000206F6620256400426164207265636F7242
:10BE20006420666F756E6420647572696E67206940
:10BE30006E697469616C697A6174696F6E002564FA
:10BE40002025642025642028256420776F72647380
:10BE500029002564207265636F7264732C20256449
:10BE600020776F7264732C206D61784944202564BB
:10BE70002C20636F6D70616374696F6E20637963EA
:10BE80006C657320256400526573746F726564205D
:10BE900025642073637269707473005374617274E3
:10BEA000656400726164696F000000003CBF0000BF
:10BEB000494C000049BF0000BD4E000059BF0000C2
:10BEC000514E000067BF00001D50000072BF00000F
:10BED000714C000082BF0000014D000096BF0000C1
:10BEE000E54C0000A5BF0000F9510000B1BF000003
:10BEF00075510000BABF000019510000C5BF000015
:10BF000069500000D0BF0000A1500000D9BF000060
:10BF1000D1500000E2BF0000814C0000F1BF0000E2
:10BF2000614C0000FABF0000914C00006E6F6E651E
:10BF3000006F746865720070616972006469736192
:10BF4000626C65526164696F006D657373616765EA
:10BF50005265636569766564007061636B657452F0
:10BF6000656365697665007061636B657453656EC2
:10BF700064007265636569766564496E74656765BA
:10BF8000720072656365697665644D657373616798
:10BF9000655479706500726563656976656453748C
:10BFA00072696E670073656E64496E746567657269
:10BFB0000073656E64506169720073656E645374DA
:10BFC00072696E67007365744368616E6E656C00BC
:10BFD00073657447726F757000736574506F776521
:10BFE00072007369676E616C537472656E67746812
:10BFF000006465766963654944006C6173744D65DE
:10C000007373616765494400556E6B6E6F776E2080
:10C010007072696D6974697665205B25733A257362
:10C020005D00000000000000963007772C610EEEE6
:10C03000BA51099919C46D078FF46A7035A563E97F
:10C04000A395649E3288DB0EA4B8DC791EE9D5E0A6
:10C0500088D9D2972B4CB609BD7CB17E072DB8E7A5
:10C06000911DBF906410B71DF220B06A4871B9F3FA
:10C07000DE41BE847DD4DA1AEBE4DD6D51B5D4F433
:10C08000C785D38356986C13C0A86B647AF962FD98
:10C09000ECC9658A4F5C0114D96C0663633D0FFAE5
:10C0A000F50D088DC8206E3B5E10694CE44160D5EB
:10C0B000727167A2D1E4033C47D4044BFD850DD2D5
:10C0C0006BB50AA5FAA8B5356C98B242D6C9BBDBE8
:10C0D00040F9BCACE36CD832755CDF45CF0DD6DCE3
:10C0E000593DD1ABAC30D9263A00DE518051D7C88A
:10C0F0001661D0BFB5F4B42123C4B3569995BACF15
:10C100000FA5BDB89EB802280888055FB2D90CC635
:10C1100024E90BB1877C6F2F114C6858AB1D61C1AE
:10C120003D2D66B69041DC760671DB01BC20D298CD
:10C130002A10D5EF8985B1711FB5B606A5E4BF9F5A
:10C1400033D4B8E8A2C9077834F9000F8EA809964D
:10C1500018980EE1BB0D6A7F2D3D6D08976C6491B8
:10C16000015C63E6F4516B6B62616C1CD8306585D1
:10C170004E0062F2ED95066C7BA5011BC1F40882AE
:10C1800057C40FF5C6D9B06550E9B712EAB8BE8BEF
:10C190007C88B9FCDF1DDD62492DDA15F37CD38C78
:10C1A000654CD4FB5861B24DCE51B53A7400BCA376
:10C1B000E230BBD441A5DF4AD795D83D6DC4D1A4A8
:10C1C000FBF4D6D36AE96943FCD96E34468867AD7F
:10C1D000D0B860DA732D0444E51D03335F4C0AAA1E
:10C1E000C97C0DDD3C710550AA41022710100BBE21
:10C1F00086200CC925B56857B3856F2009D466B968
:10C200009FE461CE0EF9DE5E98C9D9292298D0B09C
:10C21000B4A8D7C7173DB359810DB42E3B5CBDB749
:10C22000AD6CBAC02083B8EDB6B3BF9A0CE2B603CA
:10C230009AD2B1743947D5EAAF77D29D1526DB047F
:10C240008316DC73120B63E3843B64943E6A6D0DCA
:10C25000A85A6A7A0BCF0EE49DFF099327AE000A15
:10C26000B19E077D44930FF0D2A3088768F2011EA8
:10C27000FEC206695D5762F7CB67658071366C193F
:10C28000E7066B6E761BD4FEE02BD3895A7ADA1060
:10C29000CC4ADD676FDFB9F9F9EFBE8E43BEB71741
:10C2A000D58EB060E8A3D6D67E93D1A1C4C2D838CB
:10C2B00052F2DF4FF167BBD16757BCA6DD06B53F31
:10C2C0004B36B248DA2B0DD84C1B0AAFF64A033670
:10C2D000607A0441C3EF60DF55DF67A8EF8E6E31EF
:10C2E00079BE69468CB361CB1A8366BCA0D26F2538
:10C2F00036E2685295770CCC03470BBBB916022285
:10C300002F260555BE3BBAC5280BBDB2925AB42B99
:10C31000046AB35CA7FFD7C231CFD0B58B9ED92CAE
:10C320001DAEDE5BB0C2649B26F263EC9CA36A7513
:10C330000A936D02A906099C3F360EEB85670772CA
:10C3400013570005824ABF95147AB8E2AE2BB17B31
:10C35000381BB60C9B8ED2920DBED5E5B7EFDC7CB8
:10C3600021DFDB0BD4D2D38642E2D4F1F8B3DD680F
:10C370006E83DA1FCD16BE815B26B9F6E177B06F0A
:10C380007747B718E65A0888706A0FFFCA3B0666F7
:10C390005C0B0111FF9E658F69AE62F8D3FF6B6184
:10C3A00045CF6C1678E20AA0EED20DD75483044E26
:10C3B000C2B30339612667A7F71660D04D476949B4
:10C3C000DB776E3E4A6AD1AEDC5AD6D9660BDF40C7
:10C3D000F03BD83753AEBCA9C59EBBDE7FCFB2477A
:10C3E000E9FFB5301CF2BDBD8AC2BACA3093B3535F
:10C3F000A6A3B4240536D0BA9306D7CD2957DE5468
:10C40000BF67D9232E7A66B3B84A61C4021B685D40
:10C41000942B6F2A37BE0BB4A18E0CC31BDF055AB9
:10C420008DEF022D416C6C207461736B73207374FB
:10C430006F707065640076313039002025732025D7
:10C4400073004D656D6F727920636C656172656410
:10C45000004E6F2066726565207461736B20656E97
:10C460007472696573000000C0C400006567000055
:10C47000CDC40000E1610000D9C4000035670000B0
:10C48000DFC4000045670000E5C4000055670000F8
:10C49000EBC4000011620000F5C40000AD670000AD
:10C4A000FDC400000165000006C50000996200009F
:10C4B0000EC500003164000073656E736F72730007
:10C4C000616363656C65726174696F6E0074656D3C
:10C4D00070657261747572650074696C745800746B
:10C4E000696C74590074696C745A00746F75636870
:10C4F0005265616400693263526561640069326348
:10C5000057726974650072656164444854006D69CE
:10C5100063726F70686F6E650000000098C5000060
:10C520002D680000A6C500003D680000B3C50000EE
:10C5300031680000BCC5000041680000C6C50000AD
:10C5400045680000CFC5000049680000D4C5000060
:10C550004D680000D9C5000051680000E5C5000025
:10C5600055680000ECC5000059680000F5C50000E2
:10C570005D680000FAC500006168000005C60000A3
:10C58000656800000FC600003568000019C600008D
:10C590003968000074667400656E61626C65446998
:10C5A00073706C6179007365744261636B6C696769
:10C5B00068740067657457696474680067657448D7
:10C5C000656967687400736574506978656C006CA0
:10C5D000696E65007265637400726F756E64656480
:10C5E0005265637400636972636C6500747269619B
:10C5F0006E676C65007465787400746674546F754A
:10C600006368656400746674546F75636858007479
:10C610006674546F7563685900746674546F7563FB
:10C62000685072657373757265007661727300008D
:10C6300050C60000C96C00005AC60000A96C00007A
:10C6400063C60000856C00006FC60000176C000018
:10C65000766172457869737473007661724E616DAC
:10C660006564007365745661724E616D6564007631
:10C6700061724E616D65466F72496E6465780057F0
:10C68000656C636F6D6520746F204D6963726F42D6
:10C690006C6F636B732100705F73706920213D20A4
:10C6A0004E554C4C002F686F6D652F6769742F2EA7
:10C6B000706C6174666F726D696F2F7061636B610E
:10C6C0006765732F6672616D65776F726B2D61722E
:10C6D0006475696E6F6E6F726469636E7266352F12
:10C6E0006C69627261726965732F5350492F5350A0
:10C6F000492E63707000535049436C6173733A3A2A
:10C70000535049436C617373284E52465F535049EE
:10C710005F547970652A2C2075696E74385F742CAB
:10C720002075696E74385F742C2075696E74385F7B
:10C73000742900000000000000000000C96E000025
:10C74000816E0000B76E0000BD6E0000C36E000079
:10C75000B56E0000020000000300000004000000AD
:10C760001F0000001C0000000E000000250000005B
:10C770000B0000000A000000090000001E0000007D
:10C78000170000000C000000110000000100000074
:10C790000D00000022000000FFFFFFFFFFFFFFFF72
:10C7A0001A00000020000000150000001600000024
:10C7B0000F0000001800000013000000240000001B
:10C7C0000000000014000000050000001000000040
:10C7D000080000001900000028000000060000000A
:10C7E0000000000000000000AB740000A17B00000E
:10C7F000217500002D75000027750000A974000048
:10C80000A174000035750000C57400009D7400001F
:10C8100000C00140001002400020024000D0024051
:10C82000000000000000304300000000000030C3A2
:10C830007371727400000000FB21F93FFB21094075
:10C840007CD91240FB2119407A6A1F407CD92240D2
:10C85000BBFD2540FB2129403A462C407A6A2F40F7
:10C860005C4731407CD932409C6B3440BBFD354045
:10C87000DB8F3740FB2139401BB43A403A463C40FD
:10C880005AD83D407A6A3F404C7E40405C47414028
:10C890006C1042407CD942408CA243409C6B444087
:10C8A000AC344540BBFD4540CBC64640DB8F4740DE
:10C8B000EB584840FB21494083F9A200444E6E00EA
:10C8C000FC291500D1572700DD34F50062DBC000DC
:10C8D0003C999500419043006351FE00BBDEAB00E4
:10C8E000B761C5003A6E2400D24D42004906E0000F
:10C8F00009EA2E001C92D100EB1DFE0029B11C009C
:10C90000E83EA700F535820044BB2E009CE9840078
:10C91000B4267000417E5F00D69139005383390000
:10C920009CF439008B5F840028F9BD00F81F3B00A0
:10C93000DEFF97000F980500112FEF000A5A8B00B9
:10C940006D1F6D00CF7E360009CB2700464FB70024
:10C950009E663F002DEA5F00BA277500E5EBC70031
:10C960003D7BF100F739070092528A00FB6BEA0029
:10C970001FB15F00085D8D00300356007BFC460050
:10C98000F0AB6B0020BCCF0036F49A00E3A91D0089
:10C990005E619100081BE60085996500A0145F00A8
:10C9A0008D40680080D8FF0027734D0006063100D7
:10C9B000CA561500C9A873007BE260006B8CC000EA
:10C9C00000000040FB21F93F000000002D44743EB0
:10C9D000000000809846F83C0000006051CC783B95
:10C9E00000000080831BF0390000004020257A38C9
:10C9F000000000802282E336000000001DF369354C
:10CA00000200000003000000040000000600000017
:10CA10002C2066756E6374696F6E3A2000617373C3
:10CA2000657274696F6E2022257322206661696CBD
:10CA300065643A2066696C6520222573222C206C7F
:10CA4000696E65202564257325730A00580000204F
:10CA5000232D302B2000686C4C00656667454647E7
:10CA6000003031323334353637383941424344456A
:10CA700046003031323334353637383961626364D9
:10CA800065660000000000000000000000000000DB
:10CA90000000000000000000000000000000000096
:10CAA0000000000000000000000000000000000086
:10CAB0000000000000000000000000000000000076
:10CAC0000000000000000000000000000000000066
:10CAD0000000000000000000000000000000000056
:10CAE00000000000504F5349580000202020202013
:10CAF000202020202828282828202020202020200E
:10CB000020202020202020202020208810101010FD
:10CB10001010101010101010101010040404040451
:10CB2000040404040410101010101010414141417D
:10CB30004141010101010101010101010101010165
:10CB40000101010101011010101010104242424277
:10CB50004242020202020202020202020202020235
:10CB60000202020202021010101020000000000059
:10CB700000000000000000000000000000000000B5
:10CB800000000000000000000000000000000000A5
:10CB90000000000000000000000000000000000095
:10CBA0000000000000000000000000000000000085
:10CBB0000000000000000000000000000000000075
:10CBC0000000000000000000000000000000000065
:10CBD0000000000000000000000000000000000055
:10CBE0000000000000000000000000000000000045
:08CBF0005036FF7F0100000038
:10CBF800FFFFFFFFE803000001000000E803DC0579
:10CC0800DC05DC05DC050000FFFFFFFFFFFFFFFF81
:10CC18001800000019FCFFFFFFFFFFFFFF000000E6
:10CC28000090D003FFFFFFFFFFFFFFFFFFFFFFFFA5
:10CC3800FFFFFFFF0A0000000100000008000000DD
:10CC4800010000005800002000000000A4CA0000F5
:10CC5800C4CA000084CA00000000000000000000F0
:10CC680000000000000000000000000000000000BC
:10CC780000000000000000000000000000000000AC
:10CC8800000000000000000000000000000000009C
:10CC9800000000000000000000000000000000008C
:10CCA8000000000000000000430000000000000039
:10CCB800000000000000000000000000000000006C
:10CCC8000000000000000000430000000000000019
:10CCD800000000000000000000000000000000004C
:10CCE80000000000000000004300000000000000F9
:10CCF800000000000000000000000000000000002C
:10CD080000000000000000004300000000000000D8
:10CD1800000000000000000000000000000000000B
:10CD280000000000000000004300000000000000B8
:10CD380000000000000000000000000000000000EB
:10CD48000000000000000000430000000000000098
:10CD580000000000000000000000000000000000CB
:10CD68000000000000000000430000000000000078
:10CD780000000000000000000000000000000000AB
:10CD880000000000000000003BB1000009AB0000FB
:10CD980000000000EACA000072B30000FFB70000FC
:10CDA800FFB70000FFB70000FFB70000FFB70000A3
:10CDB800FFB70000FFB70000FFB70000FFB7000093
:10CDC800FFFFFFFFFFFFFFFFFFFFFFFFFFFF000069
:10CDD80001004153434949000000000000000000E1
:10CDE800000000000000000000000000000000003B
:10CDF80000004153434949000000000000000000C2
:10CE0800000000000000000000000000000000001A
:10CE180000000000250200004D6E0000A97200000D
:08CE2800357700000102000053
:040000030000736521
:00000001FF
